:100000000C9417120C9448120C9448120C94481239
:100010000C9448120C9448120C9448120C944812F8
:100020000C9448120C9448120C9448120C944812E8
:100030000C9448120C9448120C9448120C944812D8
:100040000C9448120C940D840C9448120C94481291
:100050000C9448120C948A850C94B0840C9428ABB0
:100060000C9448120C94E2850C940C860C94481263
:100070000C9448120C9448120C9448120C94481298
:100080000C9448120C9448120C9448120C94481288
:100090000C9448120C9448120C9448120C9437A9F2
:1000A0000C9448120C9448120C9448120C94481268
:1000B0000C9448120C9448120C9448120C94481258
:1000C0000C9448120C9448120C9448120C94481248
:1000D0000C9448120C9448120C9448120C94481238
:1000E0000C9448128F6FA66FA66FA66FA66FA66FAF
:1000F000A66FA66FA66FA66FA66FA66FA66FA66F58
:10010000A66FA66FA66FA66FA66FA66FA66FA66F47
:10011000A66FA66FA66FA66F7E6F306F3A6FB46E34
:10012000A66F606F6A6FA66FA66FC56EA26EA66F90
:10013000566FA66F746F4C6F446FA66FA66FA66F55
:10014000126F1C6F266FA66FA66FA66FA66FA66FA5
:10015000A66FA66FA66FA66F7E6F306F3A6FB46EF4
:10016000A66F606F6A6FA66FA66FC56EA26EA66F50
:10017000566FA66F746F4C6F446FA66FA66FA66F15
:10018000126F1C6F266F88AA8DAA92AA9CAAA6AA93
:100190001FABB0AAB8AAC0AACAAAD4AADEAAEDAA5E
:1001A000F7AA1FAB01AB0BAB15AB4AAC4DAC3CACEB
:1001B00040AC46AC84AC51AC55AC5BAC5FAC63AC12
:1001C00069AC6DAC71AC84AC77AC7BAC7FAC0763D5
:1001D0004236B79BD8A71A39685618AEBAAB558CB9
:1001E0001D3CB7CC5763BD6DEDFD753EF617723102
:1001F000BF000000803F05A84CCDB2D44EB93836C0
:10020000A9020C50B9918688083CA6AAAA2ABE0069
:100210000000803F436F6C64206578747275736969
:100220006F6E20646973616C6C6F77656400436FF7
:100230006C6420657874727573696F6E20616C6C84
:100240006F776564004175746F7265747261637471
:100250003A0053657474696E67206D6F746F722015
:1002600063757272656E742E2E2E00536574204D68
:100270006963726F7374657070696E670054726938
:1002800067676572696E67207761746368646F671A
:100290002E204966206163746976617465642C2040
:1002A000746865207072696E7465722077696C6C11
:1002B0002072657365742E0053657474696E6720CF
:1002C0005468726573686F6C6420546F3A00494ECD
:1002D000542050494E3A20004D32353120002074D0
:1002E0006F200053657420766F6C756D657472694C
:1002F0006320657874727573696F6E20666F722003
:100300006578747275646572200044697361626C0B
:10031000656420766F6C756D6574726963206578AD
:1003200074727573696F6E20666F7220657874726F
:100330007564657220004D313134200050696E20A3
:1003400063616E206E6F7420626520736574206235
:1003500079204D34322C206D617920696E20696ED0
:1003600076616C6964206F7220696E207573652EEA
:100370002000496C6C6567616C20532076616C7558
:100380006520666F72204D3432005A2028432920A0
:10039000746F77657220666C6F6F7220736574205E
:1003A000746F3A2000592028422920746F776572B3
:1003B00020666C6F6F722073657420746F3A200032
:1003C000582028412920746F77657220666C6F6F02
:1003D000722073657420746F3A2000526F6420524B
:1003E00061646975732073657420746F3A200047E7
:1003F0003133342000506F7346726F6D53746570E3
:10040000733A00436F6D7044656C74613A004361E8
:100410006C6962726174696F6E206D6F76656D656F
:100420006E74206973206C696D6974656420746FE3
:100430002031306D6D2E004669727374206D6F76B9
:100440006520746F20746F75636820617420782C48
:10045000793D302C3020746F206175746F2D736579
:1004600074207261646975732E0043616C696272F5
:100470006174696F6E206D6F76656D656E7420694D
:1004800073206C696D6974656420746F2031306D00
:100490006D2E0043616E6E6F7420736574207261FF
:1004A0006469757320616E6420666C6F6F72206181
:1004B000742073616D652074696D652E0043616CF5
:1004C0006962726174696F6E20636F64652069731D
:1004D000206C696D6974656420746F20626F747438
:1004E0006F6D20313025206F66205A20686569675E
:1004F00068740052656C617469766520706F736909
:1005000074696F6E696E67004162736F6C757465B4
:1005100020706F736974696F6E696E670047363952
:1005200020005A3A2000593A2000583A20004F46FD
:100530004653455453204F464620425920544F4F6E
:10054000204D554348205F20545259494E47204181
:100550004741494E3A200053657474696E672050D4
:10056000726F62652053656E736974697669747918
:1005700020546F3A005A2070726F6265206661697C
:100580006C6564206F6E2073656E7369746976693B
:1005900074793A200053657474696E672050726FE5
:1005A00062652053656E7369746976697479205445
:1005B0006F3A005A2070726F6265206661696C65DF
:1005C00064206F6E2073656E7369746976697479DF
:1005D0003A200053657474696E672050726F6265CB
:1005E0002053656E736974697669747920546F3A23
:1005F000005A2070726F6265206661696C656420C4
:100600006F6E2073656E73697469766974793A20C8
:100610000068656865004E6577205261646975738E
:100620003A20004F6C64205261646975733A20006F
:1006300043616C63756C61746564205261646975B3
:100640007320697320626164203A00536574746991
:100650006E672050726F62652053656E73697469AE
:100660007669747920546F3A005A2070726F62650F
:10067000206661696C6564206F6E2073656E7369B6
:100680007469766974793A200053657474696E6789
:100690002050726F62652053656E73697469766964
:1006A000747920546F3A005A2070726F6265206628
:1006B00061696C6564206F6E2073656E736974691F
:1006C000766974793A2000473332200050524F4205
:1006D000452D5A4F46465345543A00473330005350
:1006E000657474696E672050726F62652053656E21
:1006F000736974697669747920546F3A0050726F27
:1007000062657320646F206E6F74206D617463681E
:100710002E204F6666206279200047333020004D3E
:100720003131372043414C4942524154494F4E20C8
:10073000434F4D504C4554450068656865004E6513
:100740007720486F72697A6F6E74616C20526164B1
:100750006975733A20004F6C6420486F72697A6F34
:100760006E74616C205261646975733A2000436154
:100770006C63756C61746564205261646975732083
:100780006973206261643A20004D31313720434162
:100790004C4942524154494F4E204641494C4544F0
:1007A0000043616C6962726174696F6E20466169B1
:1007B0006C65640053657474696E672050726F6273
:1007C000652053656E736974697669747920546F16
:1007D0003A005A2070726F626520284852202D20FE
:1007E0005A20746F77657229206661696C65642090
:1007F0006F6E2073656E73697469766974793A20D7
:10080000004E6577205A204865696768743A004F42
:100810006C64205A204865696768743A004D31312C
:10082000372043414C4942524154494F4E204641A2
:10083000494C45440043616C6962726174696F6E32
:10084000204661696C65640053657474696E672045
:1008500050726F62652053656E736974697669744E
:100860007920546F3A005A2070726F6265202848D0
:1008700052202D2043656E74657220506F696E742E
:1008800029206661696C6564206F6E2073656E73E4
:10089000697469766974793A200047363920005ABC
:1008A0003A2000593A2000583A20004D3131372083
:1008B000456E6473746F70204F666673657420456F
:1008C00072726F72004F464653455453204F46464E
:1008D00020425920544F4F204D5543482E2041620D
:1008E0006F7274696E672E2053656E7369746976D2
:1008F0006974793A20004D3131372043414C4942E7
:10090000524154494F4E204641494C4544004361B1
:100910006C6962726174696F6E204661696C6564AE
:100920000053657474696E672050726F626520535E
:10093000656E736974697669747920546F3A005AE8
:100940002070726F626520285A20546F7765722973
:10095000206661696C6564206F6E2073656E7369D3
:100960007469766974793A20004D313137204341FA
:100970004C4942524154494F4E204641494C45440E
:100980000043616C6962726174696F6E20466169CF
:100990006C65640053657474696E672050726F6291
:1009A000652053656E736974697669747920546F34
:1009B0003A005A2070726F626520285920546F7770
:1009C000657229206661696C6564206F6E207365AD
:1009D0006E73697469766974793A20004D313137E4
:1009E0002043414C4942524154494F4E20464149CF
:1009F0004C45440043616C6962726174696F6E209A
:100A00004661696C65640053657474696E67205053
:100A1000726F62652053656E736974697669747963
:100A200020546F3A005A2070726F62652028582057
:100A3000546F77657229206661696C6564206F6EFA
:100A40002073656E73697469766974793A2000451C
:100A50006E6473746F70287329206E6F7420776FC3
:100A6000726B696E672070726F7065726C79005A74
:100A700020005920005820004572726F723A200001
:100A80004D31313720454E4453544F50204552523A
:100A90004F52004D3130342053300A4D3134302024
:100AA00053300A4D313037004D3131372049324310
:100AB000204572726F722E2041626F7274696E6788
:100AC00000493243204572726F72202D2043616CC1
:100AD0006962726174696F6E2041626F72746564DD
:100AE00000456E6473746F70287329206E6F7420D4
:100AF000776F726B696E672070726F7065726C7958
:100B0000005A20005920005820004572726F723A36
:100B100020004D31313720454E4453544F5020452D
:100B200052524F52006578656375746547436F6430
:100B300065202F20717565756544656C74614D6F16
:100B400076652072657475726E73206572726F724D
:100B50000069697332646820616363656C65726FF4
:100B60006D6574657220696E697469616C697A6912
:100B70006E672E2E2E00616363656C65726F6D6506
:100B800074657220693263207265637620666169DC
:100B90006C65642E00616363656C65726F6D65746E
:100BA00065722077726974652069326320666169B5
:100BB0006C65642E00616363656C65726F6D65744E
:100BC00065722073656E6420693263206661696CAA
:100BD00065642E0000000100250030001D000C009F
:100BE0001E00240031001C000B00180023002F0001
:100BF0001B000A0017000D0047000300040022003C
:100C00002B001A0041004200000002003500206461
:100C100065672E204300206D6561737572656420E1
:100C2000004572726F723A436F756C64206E6F7418
:100C300020686F6C642074656D7065726174757284
:100C4000652000206D730020616674657220004588
:100C500072726F723A54656D702E2072616973659D
:100C60006420746F20736C6F772E20526973652037
:100C70003D20004739310A4731452D31383046365D
:100C80003030300A473930004D31313720457874E3
:100C9000727564657220300A54300A4D3834205021
:100CA000340A4739310A4731453137324636303018
:100CB000300A47314535463530300A473930001C57
:100CC000151C140000002243141F1FD3107F100FA7
:100CD00010BF0F000000000000370F2B0EDB0D5F70
:100CE0000DE30C0400081D900058091C01B007A872
:100CF00001C80634023006C002C0054C036805D89E
:100D00000318056404D004F00498047C056004080A
:100D1000063004940600042007D003AC07A803386B
:100D2000088003C408580350093003DC090803682D
:100D30000AD802F40AB002800B88020C0C600298F8
:100D40000C3002240DF801B00DC0013C0E8001C82A
:100D50000E3001540FB800B40F2800E00F0000045B
:100D600000401D900060091C01B007A801D00634A6
:100D7000023806C002C8054C036805D8031805648C
:100D800004D804F00498047C056004080630049438
:100D90000600042007D003AC07A80338088003C46A
:100DA00008580350093003DC090803680AE002F41C
:100DB0000AB802800B88020C0C6002980C300224E6
:100DC0000DF801B00DC0013C0E8001C80E30015479
:100DD0000FB800B40F2800E00F000004000016D880
:100DE00000C006AC0178058002C004540348042802
:100DF00004E803FC049803D0055003A40618037804
:100E000007D8024C08A80220097002F4093802C869
:100E10000A08029C0BD001700C9001440D5001187F
:100E20000EF800EC0E8800C00F00000400681D4C96
:100E300000500B94005809DC0050082401A8076CEE
:100E4000012807B401C006FC017006440228068C84
:100E500002F005D402B8051C03880564035805ACEC
:100E6000033005F40310053C04E8048404C804CCF2
:100E700004A804140590045C057004A4055804EC4F
:100E8000053804340620047C060804C406F0030C6C
:100E900007D8035407C8039C07B003E40798032C42
:100EA00008800374087003BC085803040948034C05
:100EB00009300394091803DC090803240AF0026CC2
:100EC0000AE002B40AC802FC0AB002440BA0028C79
:100ED0000B8802D40B70021C0C5802640C4002AC4C
:100EE0000C2802F40C10023C0DF001840DD801CC4A
:100EF0000DB801140E98015C0E7001A40E4801ECAF
:100F00000E1801340FD8007C0F8800C40F0800FCB5
:100F10000F000000000000000000000000000000C2
:100F200000000000000000000000000000000000C1
:100F3000000000000000000000401F450060094F55
:100F40000010095C00C0086B0070087D002008924A
:100F500000D007AC008007CC003007DE00E006239D
:100F60000190065E014006A601F005FF01A0056D97
:100F7000025005F30200059603B0045A04600440D1
:100F80000510044806C0036E077003A8082003EB91
:100F900009D002230B8002410C3002390DE001041C
:100FA0000E9001A20E4001170FF000690FA000A2E1
:100FB0000F5000C60F0000DD0FB0FFEB0F60FF0405
:100FC00000700DD8004804AC0158038002D80254C8
:100FD00003800228043802FC040002D005C801A4E2
:100FE000069801780770014C08480120091801F49F
:100FF00009F000C80AC8009C0BA000700C700044E7
:101000000D3800180E0000EC0EA8FFC00FE8FE041B
:1010100000001B54006009640010097400C00884BB
:101020000070089C002008B800D007D80080070096
:101030000130072C01E00668019006AC0140060073
:1010400002F0056802A005E00250057403000524C3
:1010500004B004F0046004DC051004E406C00304DA
:1010600008700330092003780B8002600DE001A8AE
:101070000E4001680FA000C00F0000E80F60FF04E1
:1010800000801AD8009808AC01200780025006544E
:1010900003C80528045805FC040005D005B004A4C5
:1010A000066804780728044C08E8032009B003F414
:1010B000097003C80A38039C0BF802700CB0024494
:1010C0000D6802180E0802EC0E8801C00F8800F0AF
:1010D0000F00000000A00F5C006009690010097992
:1010E00000C0088C007008A2002008BD00D007DEF8
:1010F000008007050130073401E0066D019006B25B
:101100000140060702F0056D02A005E80250057BCC
:101110000300052B04B004F8046004EB06C003359B
:101120000920037F0B8002650DE001B00E40011D18
:101130000FF000480FC8006C0FA000ED0F60FFFE1D
:101140000F48FE004D617854656D703A0044696146
:101150006D657465723A00416363656C65726174B4
:10116000696F6E3A004D617853706565643A004A64
:1011700065726B3A004D617842656454656D703AF2
:10118000005072696E746572547970653A44656C8A
:101190007461005A54726176656C416363656C3AA0
:1011A000005954726176656C416363656C3A00580E
:1011B00054726176656C416363656C3A005A507293
:1011C000696E74416363656C3A00595072696E745C
:1011D000416363656C3A00585072696E7441636391
:1011E000656C3A005A53697A653A005953697A65D1
:1011F0003A005853697A653A005A4D61783A005975
:101200004D61783A00584D61783A005A4D696E3A0E
:1012100000594D696E3A00584D696E3A004A657240
:101220006B58593A005072696E746C696E6543610F
:101230006368653A00454550524F4D3A0041757418
:101240006F6C6576656C3A005A50726F62653A0051
:10125000436173654C69676874733A0053757070C5
:101260006F72744C6F63616C46696C616D656E740E
:101270006368616E67653A00537570706F7274478A
:1012800031304731313A005A486F6D654469723ADE
:101290000059486F6D654469723A0058486F6D6532
:1012A0004469723A00536F667477617265506F7764
:1012B00065725377697463683A004C43443A004658
:1012C000616E3A005344436172643A004865617448
:1012D00065644265643A004D6978696E6745787463
:1012E00072756465723A004E756D457874727564F6
:1012F00065723A00496E7075744275666665723A39
:101300000042617564726174653A004E6F206361DA
:101310007365206C6967687473004D313134200047
:1013200064656C6179203130306D732E00686F6DAB
:1013300065417869732000686F6D65417869732035
:101340002F20717565756544656C74614D6F7665A8
:101350002072657475726E73206572726F720050C0
:1013600072696E7465723A3A736574757020006DB7
:101370006F7665546F5265616C202F2071756575AD
:101380006544656C74614D6F766520726574757225
:101390006E73206572726F72006D6F7665546F2088
:1013A0002F20717565756544656C74614D6F766548
:1013B0002072657475726E73206572726F72006947
:1013C00073506F736974696F6E416C6C6F7765648D
:1013D0002000457874722E00436F6E6669673A008C
:1013E0004F6E6520686561746572207365656D7305
:1013F000206465636F75706C65642066726F6D2024
:10140000746865726D6973746F72202D20646973DE
:1014100061626C696E6720616C6C20666F7220730C
:1014200061666574792100616476616E6365204C44
:10143000205B303D6F66665D00657874727564652B
:101440007220636F6F6C6572207370656564205BDA
:10145000302D3235355D0064697374616E636520CB
:10146000746F2072657472616374207768656E2092
:1014700068656174696E67205B6D6D5D0074656D94
:10148000702E20666F722072657472616374696F6A
:101490006E207768656E2068656174696E67205B91
:1014A000435D0074656D702E2073746162696C69B0
:1014B0007A652074696D65205B735D00592D6F66D8
:1014C00066736574205B73746570735D00582D6F6F
:1014D0006666736574205B73746570735D00504954
:1014E00044206D61782076616C7565205B302D320B
:1014F00035355D0050494420442D6761696E0050C8
:10150000494420492D6761696E0050494420502D9F
:101510006761696E2F646561642D74696D65005043
:101520004944206472697665206D696E00504944B3
:10153000206472697665206D617800686561742049
:101540006D616E61676572205B302D335D00616394
:1015500063656C65726174696F6E205B6D6D2F736E
:101560005E325D00737461727420666565647261D9
:101570007465205B6D6D2F735D006D61782E206644
:1015800065656472617465205B6D6D2F735D0073BA
:101590007465707320706572206D6D00436F727298
:1015A0002E20646961676F6E616C2043205B6D6DF6
:1015B0005D00436F72722E20646961676F6E616CAB
:1015C0002042205B6D6D5D00436F72722E20646956
:1015D00061676F6E616C2041205B6D6D5D004D61D8
:1015E00078207072696E7461626C652072616469E2
:1015F0007573205B6D6D5D00546F776572205A20A6
:10160000656E6473746F70206F6666736574205BBB
:1016100073746570735D00546F776572205920652F
:101620006E6473746F70206F6666736574205B738D
:10163000746570735D00546F776572205820656E15
:101640006473746F70206F6666736574205B737467
:101650006570735D005365676D656E74732F7320DD
:10166000666F722074726176656C005365676D6594
:101670006E74732F7320666F72207072696E746956
:101680006E6700486F72697A6F6E74616C20726F5A
:10169000642072616469757320617420302C30207D
:1016A0005B6D6D5D00446961676F6E616C20726F88
:1016B00064206C656E677468205B6D6D5D00486FBB
:1016C0006D696E67206665656472617465205B6D27
:1016D0006D2F735D004D61782E20666565647261C3
:1016E0007465205B6D6D2F735D005374657073209E
:1016F000706572206D6D0054726176656C20616357
:1017000063656C65726174696F6E205B6D6D2F73BC
:101710005E325D00416363656C65726174696F6E12
:10172000205B6D6D2F735E325D004D61782E206AF7
:1017300065726B205B6D6D2F735D005A206D617853
:10174000206C656E677468205B6D6D5D0059206D5F
:101750006178206C656E677468205B6D6D5D005804
:10176000206D6178206C656E677468205B6D6D5DBF
:10177000005A20686F6D6520706F73205B6D6D5D22
:10178000005920686F6D6520706F73205B6D6D5D13
:10179000005820686F6D6520706F73205B6D6D5D04
:1017A0000053746F70207374657070657220616689
:1017B00074657220696E6163746976697479205BFF
:1017C0006D732C303D6F66665D004D61782E20692B
:1017D0006E6163746976652074696D65205B6D73F5
:1017E0002C303D6F66665D005072696E74657220C4
:1017F000616374697665205B735D0046696C616D39
:10180000656E74207072696E746564205B6D5D0036
:10181000416476616E636564205573657200426150
:10182000756472617465004550523A33200045502A
:10183000523A3220004550523A3120004550523A37
:1018400030200050726F746F636F6C207665727316
:10185000696F6E206368616E6765642C20757067C0
:10186000726164696E6700436F6E66696775726165
:1018700074696F6E20726573657420746F2064657F
:101880006661756C74732E00436F6E66696775725E
:101890006174696F6E206C6F616465642066726F3D
:1018A0006D20454550524F4D2E00436F6E6669675F
:1018B00075726174696F6E2073746F7265642074E1
:1018C0006F20454550524F4D2E004175746F6C6529
:1018D00076656C206163746976652028312F302924
:1018E000005A2D70726F6265205933005A2D707244
:1018F0006F6265205833005A2D70726F62652059EF
:1019000032005A2D70726F6265205832005A2D7065
:10191000726F6265205931005A2D70726F626520B6
:101920005831005A2D70726F626520782D792D73B1
:1019300070656564205B6D6D2F735D005A2D70724C
:101940006F6265207370656564205B6D6D2F735DDC
:10195000005A2D70726F6265206F66667365742021
:1019600079205B6D6D5D005A2D70726F6265206F1E
:1019700066667365742078205B6D6D5D004D6178DF
:101980002E207A2D70726F6265202D206265642092
:10199000646973742E205B6D6D5D005A2D70726FDB
:1019A000626520686569676874205B6D6D5D0077AE
:1019B000616974005072696E746572206865696748
:1019C00068743A005A2D70726F6265206661696CA6
:1019D0006564005472616E73666F726D6174696FD5
:1019E0006E206D61747269783A004175746F6C6530
:1019F00076656C696E672064697361626C6564000A
:101A00004175746F6C6576656C696E6720656E6193
:101A1000626C6564004175746F6C6576656C206DF1
:101A2000617472697820726573657400004732389A
:101A30002F6E47315A32352F6E005A2D70726F62F9
:101A4000652073746174653A005265736574205A39
:101A500020686569676874005A2D70726F6265202E
:101A600061766572616765206865696768743A00C8
:101A7000205374657020566172696174696F6E20BD
:101A800066726F6D2050726F626520746F206265A0
:101A9000642044697374616E63653A005A2D7072F4
:101AA0006F62653A005072696E7465722073657476
:101AB00020696E746F206472792072756E206D6F6C
:101AC000646520756E74696C2072657374617274DC
:101AD00021003A20776F726B696E67003A20746557
:101AE0006D702073656E736F7220646566656374D4
:101AF00000657874727564657220004D54454D50D0
:101B00003A00504944204175746F74756E652066C3
:101B1000696E6973686564202120506C616365207B
:101B2000746865204B702C204B6920616E64204BDB
:101B30006420636F6E7374616E747320696E2074B9
:101B4000686520436F6E66696775726174696F6E50
:101B50002E68206F7220454550524F4D0050494429
:101B6000204175746F74756E65206661696C65647B
:101B7000212074696D656F7574005049442041756A
:101B8000746F74756E65206661696C65642120549C
:101B9000656D706572617475726520746F20686917
:101BA000676800204B643A2000204B693A200020EF
:101BB0004B703A200020436C617373696320504975
:101BC00044002054753A2000204B753A2000206DC7
:101BD00061783A2000206D696E3A200020643A2036
:101BE0000020626961733A200050494420417574B5
:101BF0006F74756E652073746172740054617267DE
:101C0000657445787472004E6F206D6F766520693B
:101C10006E2064656C7461207365676D656E7420F9
:101C200077697468203E2031207365676D656E7436
:101C30002E20546869732073686F756C64206E651C
:101C40007665722068617070656E20616E64206DCB
:101C5000617920636175736520612070726F626CB9
:101C6000656D210044656C7461205261646975730F
:101C700020432830293A0044656C74612052616425
:101C800069757320422830293A0044656C746120DC
:101C900052616469757320412830293A00416C70A3
:101CA00068612043283930293A00416C706861200E
:101CB0004228333330293A00416C70686120412852
:101CC000323130293A00546F77657220333A00542C
:101CD0006F77657220323A00546F77657220313A1F
:101CE00000496E76616C69642064656C7461206380
:101CF0006F6F7264696E617465202D206D6F7665FB
:101D00002069676E6F726564006C696E6561722030
:101D10004C3A00454550524F4D20757064617465D2
:101D200064002C2073706565643D00206C696E65ED
:101D300061722073746570733A004A65726B3A0081
:101D40007A5F6D61783A00795F6D61783A00785F0B
:101D50006D61783A004C2000482000206973200013
:101D600020746F2000536574206F75747075743A19
:101D700020004D53312C4D53322050696E73004575
:101D8000313A0045303A005A3A00593A0020002CC6
:101D900000206D696E0020686F75727320002064EA
:101DA00061797320006D20005072696E74696E67EE
:101DB0002074696D653A005072696E7465642066BE
:101DC000696C616D656E743A0046616E737065652D
:101DD000643A00466C6F774D756C7469706C793A33
:101DE0000053706565644D756C7469706C793A0068
:101DF000202F003A0020403A00543A0020453A0093
:101E0000205A3A0020593A0020583A00583A0046E1
:101E10007265652052414D3A00556E6B6E6F776E5C
:101E200020636F6D6D616E643A00536F6674776105
:101E30007265205265736574005761746368646FDE
:101E4000672052657365740042726F776E206F75FC
:101E5000742052657365740045787465726E616CA8
:101E600020526573657400506F776572557000730A
:101E70007461727400424C4B2000736B69702000D7
:101E800020676F7420004572726F723A65787065D2
:101E900063746564206C696E652000205200204ADE
:101EA000002049002050002053002046002045001B
:101EB000205A00205900205800466F726D6174202E
:101EC0006572726F720057726F6E67206368656328
:101ED0006B73756D004563686F3A00526573656E8C
:101EE000643A005761726E696E673A00496E666FB8
:101EF0003A004572726F723A00494E46004E414EAA
:101F0000006F6B004649524D574152455F4E414D5F
:101F1000453A52657065746965725F302E39322EAC
:101F200032204649524D574152455F444154453A4B
:101F30003230313731313133204D414348494E45FC
:101F40005F545950453A455249532044656C746179
:101F50002000000000000000000000000000000061
:101F6000000024F403D950C38EB1C2A23D96828BE7
:101F70003582127AE372816CCB66A861015DC75825
:101F8000EB546151204E1E4B5648C14559431A41EE
:101F9000013F093D2F3B7139CD374036C934653398
:101FA0001432D430A32F802E6B2D632C672B752A0F
:101FB0008E29B028DC2710274B268F25D9242B24E7
:101FC0008223E0224322AC211A218D200420801F8D
:101FD000001F841E0C1E971D261DB81C4E1CE61BE0
:101FE000821B201BC11A641A0A1AB2195D190A1938
:101FF000B9186A181C18D11788174017FA16B516A1
:1020000073163116F115B31576153A150015C71468
:102010008F1458142214EE13BA1388135613251371
:10202000F612C71299126C1240121512EB11C1115F
:102030009811701148112111FB10D610B1108D109C
:102040006910461024100210E10FC00FA00F800F7E
:10205000610F420F230F060FE80ECB0EAF0E930E4B
:10206000770E5C0E410E270E0D0EF30DDA0DC10D2D
:10207000A80D900D780D600D490D320D1B0D050D4D
:10208000EF0CD90CC30CAE0C990C850C700C5C0CCD
:10209000480C350C210C0E0CFB0BE80BD60BC40BBB
:1020A000B20BA00B8E0B7D0B6B0B5A0B4A0B390B33
:1020B000290B180B080BF80AE90AD90ACA0ABB0A45
:1020C000AC0A9D0A8E0A800A710A630A550A470AF9
:1020D000390A2C0A1E0A110A040AF709EA09DD095D
:1020E000D009C409B709AB099F09920987097B097F
:1020F0006F09630958094C09410936092B09200960
:1021000015090A090009F508EB08E008D608CC080B
:10211000C208B808AE08A4089A08900887087D0885
:1021200074086B08610858084F0846083D083408D1
:102130002C0823081A08120809080108F807F007F4
:10214000E807E007D807D007C807C007B807B007F7
:10215000A807A1070000420FA1071605D0030D0331
:102160008B022E02E801B2018601630145012C01B8
:1021700017010401F400207A3A0020793A0020780F
:102180003A00696E20717565756544656C74614DC2
:102190006F766520746F2063616C63756C61746524
:1021A00044656C74615375625365676D656E7473D5
:1021B0002072657475726E73206572726F722E0074
:1021C000432068697420666C6F6F720043706F7390
:1021D000207820737175617265200043706F7320E1
:1021E00078207374657073200043706F73207920BA
:1021F000737175617265200043706F73207920736D
:10220000746570732000422068697420666C6F6F7B
:10221000720042706F73207820737175617265204F
:102220000042706F732078207374657073200042D1
:10223000706F732079207371756172652000427030
:102240006F73207920737465707320004120686972
:102250007420666C6F6F720041706F73207820730A
:102260007175617265200041706F732078207374FE
:10227000657073200041706F7320792073717561F0
:102280007265200041706F732079207374657073DC
:1022900020006D6F766552656C617469766544697E
:1022A0007374616E6365496E5374657073202F207B
:1022B000717565756544656C74614D6F76652072E6
:1022C000657475726E73206572726F720000000A19
:1022D0000B02090C0D0E08070304010000000000AA
:1022E00000000000000000000000000000000000EE
:1022F00000000000000000000012111000000000AB
:1023000000000000000000000000000000000000CD
:10231000000000010210202008081020401020407A
:102320008002010201080402010102040810204099
:1023300080804020100804020180040201804020B7
:1023400010080402010804020101020408102040E0
:1023500080010204081020408005050505070508D6
:10236000080808020202020A0A0808040404040118
:10237000010101010101010303030303030303043A
:102380000707070C0C0C0C0C0C0C0C0202020206CA
:10239000060606060606060B0B0B0B0B0B0B0B00BB
:1023A0000020002300260029002C002F003200000E
:1023B0000100000301060109010000220025002898
:1023C000002B002E0031003400020100000501083E
:1023D000010B0100002100240027002A002D0030FD
:1023E00000330001010000040107010A014E414EC3
:1023F000494E495459494E46CDCCCC3D0AD7233C91
:1024000017B7D13877CC2B329595E6241FB14F0AF8
:10241000000020410000C84200401C4620BCBE4CC9
:10242000CA1B0E5AAEC59D74006ABC8658A81124FA
:102430001FBECFEFD1E2DEBFCDBF00E00CBF13E087
:10244000A0E0B2E0EAEEFBE601E00BBF02C00790BD
:102450000D92AC31B107D9F729E1ACE1B3E001C08D
:102460001D92A53CB207E1F714E2CEE2D4E200E00F
:1024700006C022970109FE010BBF0E94CBB1C832F2
:10248000D10780E00807A9F70E9444AD0C94F3B58A
:102490000C940000CF93DF9300D01F92CDB7DEB72E
:1024A00044E050E0BC01CE0101960E94AFB56981C5
:1024B0007A818B819C810F900F900F900F90DF910C
:1024C000CF910895179A0895169A0895159A089528
:1024D00080B182FB882780F9089580B1869581704C
:1024E000089588E493E0D6CFCF92DF92EF92FF92E7
:1024F000CF93DF9300D01F921F92CDB7DEB76B0151
:102500007C016093EF047093F0048093F104909346
:10251000F2040E94B34EC982DA82EB82FC8244E06C
:1025200050E065E773E0CE0101960E94D1B523E04B
:10253000B701A6018BED93E00E9410750E9482788E
:10254000682F88E690E06D830E94BFB56D816817A3
:1025500021F088E690E00E94DAB50F900F900F907E
:102560000F900F90DF91CF91FF90EF90DF90CF9081
:102570000895CF93DF931F92CDB7DEB7BC018DE7EF
:1025800093E00E94EDB50E948278682F88E690E083
:1025900069830E94BFB56981681739F088E690E0C9
:1025A0000F90DF91CF910C94DAB50F90DF91CF911E
:1025B0000895CF93DF931F92CDB7DEB7BC018FE7AD
:1025C00093E00E94EDB50E948278682F88E690E043
:1025D00069830E94BFB56981681739F088E690E089
:1025E0000F90DF91CF910C94DAB50F90DF91CF91DE
:1025F0000895CF93DF931F92CDB7DEB7BC0181E87A
:1026000093E00E94EDB50E948278682F88E690E002
:1026100069830E94BFB56981681739F088E690E048
:102620000F90DF91CF910C94DAB50F90DF91CF919D
:10263000089580912D048823A1F010922D040E940A
:10264000AA4A80919002815080939002811109C022
:1026500080919102833010F40E94514A85E080936A
:102660009002089580919207882329F00E94F971C1
:1026700080E0DFDFF7CF08954F925F926F927F92F5
:102680008F929F92AF92BF92CF92DF92EF92FF9282
:102690000F931F93CF93DF9300D01F92CDB7DEB778
:1026A0008C018091690590916A05A0916B05B091AC
:1026B0006C0589839A83AB83BC83C0906D05D090F1
:1026C0006E05E0906F05F090700580907105909018
:1026D0007205A0907305B09074059C01AD01BC011A
:1026E000CD010E940AB181110FC149805A806B80CF
:1026F0007C80E89477F82FEF3FEF4FE75FE7C30167
:10270000B2010E940AB181110BC02FEF3FEF4FE7DA
:102710005FE7C301B2010E94B7AD18160CF4F4C014
:10272000A7019601C701B6010E940AB18111ECC050
:1027300026013701E89477F82FEF3FEF4FE75FE787
:10274000C301B2010E940AB181110BC02FEF3FEF0C
:102750004FE75FE7C301B2010E94B7AD18160CF452
:10276000D3C0A5019401C501B4010E940AB1811131
:10277000CBC024013501E89477F82FEF3FEF4FE706
:102780005FE7C301B2010E940AB181110BC02FEFB4
:102790003FEF4FE75FE7C301B2010E94B7AD1816E4
:1027A0000CF4B2C02091410530914205409143059F
:1027B0005091440569817A818B819C810E9453AD3F
:1027C0002B013C012091450530914605409147057C
:1027D00050914805C701B6010E9453AD6B017C01C1
:1027E0002091490530914A0540914B0550914C0587
:1027F000C501B4010E9453AD4B015C018091C90534
:10280000882329F020E732E441E25DE304C020E0C0
:1028100030E040E85FE3C301B2010E945FB0AB016A
:10282000BC0122E08CE09EE10E944D758091C905BB
:10283000882329F020E732E441E25DE304C020E090
:1028400030E040E85FE3C701B6010E945FB0AB0132
:10285000BC0122E084E09EE10E944D758091C90593
:10286000882329F020E732E441E25DE304C020E060
:1028700030E040E85FE3C501B4010E945FB0AB0106
:10288000BC0123E080E09EE10E944D7560918105CE
:102890007091820580918305909184050E948AAE93
:1028A0002091C5053091C6054091C7055091C805D6
:1028B0000E945FB02091C905222329F020E732E46D
:1028C00041E25DE304C020E030E040E85FE30E94C5
:1028D0005FB0AB01BC0124E08CEF9DE10F900F9045
:1028E0000F900F90DF91CF911F910F91FF90EF907C
:1028F000DF90CF90BF90AF909F908F907F906F9020
:102900005F904F900C941075C8010E9448734ACF95
:10291000CF92DF92EF92FF92CF93DF93EC01893158
:1029200091053CF0C53F81E0D8072CF0C4EFD1E021
:1029300002C0C9E1D0E0BE01882777FD8095982FBD
:102940000E948AAE6B017C016091790470917A04D7
:10295000882777FD8095982F0E948AAE9B01AC0155
:10296000C701B6010E94BEAD9B01AC0160917B0422
:1029700070917C0480917D0490917E040E945FB0F0
:1029800060937B0470937C0480937D0490937E0419
:10299000D0937A04C0937904BE0181EE9DE1DF916A
:1029A000CF91FF90EF90DF90CF900C94F8738F92BF
:1029B0009F92AF92BF92CF92DF92EF92FF92CF930E
:1029C000DF93EC018931910534F0893C91052CF0BD
:1029D000C8ECD0E002C0C9E1D0E0D0937804C09345
:1029E0007704E0911C03F0911D03E258FF4FC08073
:1029F000D180E280F38020E030E0A901C701B60178
:102A00000E94B7ADAE01662757FD6095762F181668
:102A10005CF0CB01BA010E948AAE2AE037ED43E2B6
:102A20005CE30E945FB024C0CB01BA010E948AAE71
:102A30002AE037ED43E25CE30E945FB020E030E043
:102A400040E850E40E945FB04B015C01A701960191
:102A5000C701B6010E945FB02BED3FE049E450E4AE
:102A60000E945FB09B01AC01C501B4010E94BEADE4
:102A700060939602709397028093980290939902C4
:102A8000BE0183ED9DE1DF91CF91FF90EF90DF904C
:102A9000CF90BF90AF909F908F900C94F873CF938E
:102AA000DF9320913D0597FD0DC0EC018F3F91050F
:102AB00019F014F0CFEFD0E0209721F02860209398
:102AC0003D0505C0277F20933D05C0E0D0E06111A2
:102AD000C9DD8091EB1890E0C817D90729F0BE0135
:102AE00089EC9DE10E94F873C093EB18DF91CF91C0
:102AF00008954F925F926F927F928F929F92AF92C2
:102B0000BF92CF92DF92EF92FF92CF93DF9300D0EC
:102B10001F92CDB7DEB72FE632E143E85AE360916A
:102B200061047091620480916304909164040E9436
:102B30005FB06B017C0181E890E0ACDC9B01AC01F3
:102B4000C701B6010E9453ADAB01BC0122E087EB87
:102B50009DE10E944D7585EA9DE10E940F73E09111
:102B60000A02F0910B0220E030E040E751E4638577
:102B70007485858596850E94EBAF18160CF46BC0A2
:102B800020E030E0A9018DE790E029833A834B8370
:102B90005C830E94C7B54B015C0129813A814B815E
:102BA0005C81820E931EA41EB51EC501B40120E8EF
:102BB00031E541E050E00E947EB160E87EEA8EEFB0
:102BC0009FEF0E9426B16B017C01C80CD91CEA1C46
:102BD000FB1CBA01A90188EA9DE10E941E74C7018D
:102BE000B60120E13EE040E050E00E947EB14901A4
:102BF0005A01BA01A9018EE99DE10E941E74A0EF5D
:102C0000B1EFA50194010E94C7B16C0D7D1D8E1D11
:102C10009F1D2CE330E040E050E00E947EB1BA01FD
:102C2000A90186E99DE10E941E7481E99DE10F9052
:102C30000F900F900F90DF91CF91FF90EF90DF906A
:102C4000CF90BF90AF909F908F907F906F905F904C
:102C50004F900C9427730E9472ABC0906504D09083
:102C60006604E0906704F09068046C197D098E0991
:102C70009F0928EE33E040E050E00E945CB183CF32
:102C8000811102C08EE207C0813011F48DE203C0D1
:102C9000823019F48CE20C9465AA0895EAE0F1E020
:102CA0008081886080838081806180838081806270
:102CB000808364E170E08EE20E9465AA64E170E0C6
:102CC0008DE20E9465AA62E870E08CE20E9465AA2B
:102CD000E1E2F1E08081887F81608083089567FD73
:102CE00043C08230E9F028F4882341F0813061F05C
:102CF0003BC0833009F1843059F136C0662311F0AE
:102D0000A19A69C0A19867C080910801662311F05B
:102D1000806801C08F778093080147FF3AC05FC089
:102D200080910801662311F0806401C08F7B80933D
:102D3000080147FF34C055C080910801662311F097
:102D4000886001C0877F8093080147FF32C046C07A
:102D500080910501662311F0806401C08F7B809310
:102D6000050147FF2EC03CC047FD3BC08230B9F093
:102D700028F4882341F0813061F008958330C9F050
:102D80008430F9F00895442311F0A09A0895A09892
:102D90000895442311F0A29A0895A298089580916D
:102DA0000801442311F0806201C08F7D80930801E7
:102DB000089580910801442311F08061F7CF8F7E40
:102DC000F5CF80910501442311F0806401C08F7B11
:102DD00080930501089547FFD6CF0895089508957B
:102DE00008950895643079F028F4613041F062303C
:102DF00041F00895683051F0603141F0089540E0AD
:102E000003C040E004C041E060E002C041E061E096
:102E100066CFCF93DF9382E79DE10E94277362B371
:102E20006695617070E08CE09EE10E94EC7362B385
:102E3000617070E08FE89DE10E94F873C6E0D1E018
:102E40008881992787FD9095692F661F6627661FE1
:102E500070E08AE89DE10E94EC7362B362FB662732
:102E600060F970E08FE89DE10E94F873688166FB6D
:102E7000662760F970E087E89DE10E94EC73688145
:102E800065FB662760F970E08FE89DE10E94F873AA
:102E9000688163FB662760F970E083E89DE10E942A
:102EA000EC7368816295617070E08FE89DE10E942B
:102EB000F873C3E0D1E0688166FB662760F970E0D3
:102EC0008FE79DE10E94EC73688166FB662760F9DD
:102ED00070E08FE89DE1DF91CF910C94F873FF9241
:102EE0000F931F93CF93DF9300D01F921F92CDB704
:102EF000DEB785E0E7EFF2E0DE01119601900D927A
:102F00008A95E1F7989A9A9A809107018062809356
:102F1000070180910701806180930701809104017E
:102F20008064809304018E010F5F1F4FF12CF80124
:102F300061918F018F2D56DFF394F5E0FF12F7CFEB
:102F40000F900F900F900F900F90DF91CF911F91E6
:102F50000F91FF9008950C94A5830E949083209177
:102F60000802309109028217930724F49093090212
:102F7000809308020895609108027091090280917F
:102F80000602909107026817790744F470930702CC
:102F9000609306028FE09EE10C94F8730895CF933E
:102FA000C82F69E170E086EF98E10E9443A86C2F7A
:102FB00086EF98E10E94E4A760E086EF98E10E9426
:102FC00044A8882329F085EB9BE0CF910C942773CC
:102FD000CF910895CF93DF93D82FC62F69E170E08A
:102FE00086EF98E10E9443A86D2F86EF98E10E943A
:102FF000E4A76C2F86EF98E10E94E4A786EF98E1A2
:103000000E9456A8882331F085E99BE0DF91CF919B
:103010000C942773DF91CF910895C1DF41E050E018
:1030200069E170E086EF98E10E9437A886EF98E1A9
:103030000E948DA7892B31F086EF98E10E9495A719
:1030400081E0089586E79BE00E94277380E0089561
:1030500081E59BE00E94277386EF98E10E9422A8F9
:103060008FE0DBDF81E3D9DF80E2D7DF6CE980E24C
:10307000B1DF80E2D2DF82E2D0DF60E482E2AADF69
:1030800082E2CBDF85E2C9DF60E085E2A3DF85E293
:10309000C4DF83E2C2DF60E383E29CDF83E2BDDF63
:1030A00084E2BBDF6AE484E295DF84E2B6DF80E39A
:1030B000B4DF60E280E38EDF80E3AFDF81E3ADDF8A
:1030C00082E3ABDF69E182E385DF82E3A6DF83E3AE
:1030D000A4DF60E083E37EDF83E39FDF84E39DDFA3
:1030E00060E084E377DF84E398DF86E396DF62E3E2
:1030F00086E370DF86E391DF87E38FDF60E087E3BD
:1031000069DF87E38ADF88E388DF60E188E362DFE5
:1031100088E383DF89E381DF8AE37FDF62E38AE399
:1031200059DF8AE37ACFCF9381E377DFC82F85E336
:1031300074DF811101C0C0E089E36FDF811101C03C
:10314000C0E08DE26ADF811101C0C0E08C2FCF9119
:1031500008956DE080EA96E00E9444826AE080EA89
:1031600096E00C944482E0911C03F0911D0342A967
:1031700053A964A975A922E089EF9DE10E944D75CC
:10318000E0911C03F0911D0346A957A960AD71ADF4
:1031900020E080EF9DE10E944D75E0918F02EF3FAE
:1031A00029F4E0911C03F0911D03E081F0E0E85167
:1031B000F74E608170E085EF9DE10E94EC73C9CF0E
:1031C0002F923F924F925F926F927F928F929F9237
:1031D000AF92BF92CF92DF92EF92FF920F931F9325
:1031E000CF93DF93CDB7DEB729970FB6F894DEBF44
:1031F0000FBECDBF5C01DC0116968D919C91179797
:103200008C3C910511F40C94FC2108F098C08A368E
:10321000910509F427C708F04FC08335910509F4DB
:1032200046C278F58A32910509F4A3C158F4813178
:10323000910509F49BC1429711F00C94852642D95F
:1032400043D9C4C28135910509F422C208F02BC2CA
:103250008035910511F00C94852604DA0E9472AB3A
:103260006093F2187093F3188093F4189093F51804
:103270009B9A80913F05806480933F05A3980C94AE
:10328000BC268C35910509F416C350F4843591059C
:1032900009F412C28535910509F4E9C20C9485261A
:1032A0008836910509F4BCC308F0A4C4833691059F
:1032B00009F465C30C9485268537910511F40C94A7
:1032C000BC26F0F48F36910509F4FEC650F48B3617
:1032D000910509F4D8C68D36910509F4ADC40C9456
:1032E00085268337910509F41EC708F076C6823714
:1032F000910511F00C94852686E393E00C94BD2390
:10330000883C910509F474C770F48C38910509F470
:103310001DC48E3B910509F455C68737910511F000
:103320000C9485261EC7F501208131818A3C9105C8
:1033300011F40C94A82108F4AEC70C94EC218E3241
:10334000F1E09F0711F40C944A2408F09AC08F3DD5
:10335000910511F40C942C23E0F58F3C910511F4A8
:103360000C94722228F58D3C910511F40C9458228E
:103370008E3C910511F00C948526C50129960FB657
:10338000F894DEBF0FBECDBFDF91CF911F910F919B
:10339000FF90EF90DF90CF90BF90AF909F908F9075
:1033A0007F906F905F904F903F902F900C94D37EC2
:1033B0008C3D910511F40C94D9228D3D910511F4A9
:1033C0000C940123813D910511F00C9485260C94F9
:1033D000BA22843031E0930711F40C94D72390F58E
:1033E000893E910511F40C9441238B3F910511F412
:1033F0000C947A23883E910511F00C9485266091F7
:10340000F0187091F1188BE29DE10E94EC734091ED
:10341000EC185091ED186091EE187091EF1822E0C1
:1034200082E29DE10E9410751092F1181092F0183E
:103430001092EC181092ED181092EE181092EF18EE
:103440000C94BC26863051E0950711F40C9413249B
:1034500010F40C94F1238931914011F00C948526DD
:103460008DE792E00E943E7380E00E94634E68EC1C
:1034700070E080E090E00E94A1AB8FB7F8940C94CC
:1034800049248836E1E09E0711F40C94B12568F5D3
:10349000813421E0920711F40C94BC2480F48F3223
:1034A00041E0940711F40C9489248034914011F088
:1034B0000C94852681E00E948E610C94D1248E3577
:1034C000A1E09A0711F40C94FA248336B1E09B072B
:1034D00011F40C946B258234914011F00C948526E4
:1034E00080E00E94DA650C94D124843FF1E09F07CC
:1034F00011F40C94152650F5813931E0930711F43D
:103500000C94CB25823941E0940711F40C94E52505
:103510008039914011F00C94852629960FB6F894C5
:10352000DEBF0FBECDBFDF91CF911F910F91FF90F6
:10353000EF90DF90CF90BF90AF909F908F907F9053
:103540006F905F904F903F902F908CC8863FA1E086
:103550009A0711F40C94402610F40C941B268C3816
:10356000934011F40C945A260C94852617981698BB
:1035700054C2D5012D913C91119733FD02C00C949A
:10358000BC2692961C919297E12E9396FC90E4EDC6
:10359000FBE0449150E04E155F0509F45DC03296A2
:1035A000BCE0E834FB07A9F7F7FC56C032FF2BC09C
:1035B000F501468D578D60A171A14F3F5105610501
:1035C000710509F0E8F461E0812F0E9485ACD50116
:1035D0005E966C91812F0E94BEACF501668D778D51
:1035E000812F0E9465AAB70185E69DE10E94EC73D8
:1035F000D5015E966D917C915F9780E69DE112C04A
:1036000082E793E02BC062E0812F0E9485ACB70176
:1036100080E69DE10E94EC73812F0E94F3ACBC0117
:103620008BE59DE129960FB6F894DEBF0FBECDBFA6
:10363000DF91CF911F910F91FF90EF90DF90CF908E
:10364000BF90AF909F908F907F906F905F904F90C2
:103650003F902F900C94F8738CE393E029960FB66B
:10366000F894DEBF0FBECDBFDF91CF911F910F91B8
:10367000FF90EF90DF90CF90BF90AF909F908F9092
:103680007F906F905F904F903F902F900C94487375
:103690000E9432139B9A80913F058F7B80933F0558
:1036A000A39A0C94BC26109285050C94BC2681E04C
:1036B000809385050C94BC26F5018081918192FF51
:1036C00012C0268D378D40A151A1A8EEB3E00E9413
:1036D000BBB16093EF027093F0028093F10290937C
:1036E000F2020C94BC2693FFA5C0F50182A193A120
:1036F000A4A1B5A182309105A105B10509F466C068
:103700002CF50097A105B10509F446C00197A10564
:10371000B10511F00C94BC2629960FB6F894DEBFC3
:103720000FBECDBFDF91CF911F910F91FF90EF9012
:10373000DF90CF90BF90AF909F908F907F906F90D1
:103740005F904F903F902F900C94641283309105BE
:10375000A105B10509F454C00497A105B10511F004
:103760000C94BC2629960FB6F894DEBF0FBECDBFD1
:10377000DF91CF911F910F91FF90EF90DF90CF904D
:10378000BF90AF909F908F907F906F905F904F9081
:103790003F902F900C94E44229960FB6F894DEBF28
:1037A0000FBECDBFDF91CF911F910F91FF90EF9092
:1037B000DF90CF90BF90AF909F908F907F906F9051
:1037C0005F904F903F902F900C94621229960FB605
:1037D000F894DEBF0FBECDBFDF91CF911F910F9147
:1037E000FF90EF90DF90CF90BF90AF909F908F9021
:1037F0007F906F905F904F903F902F900C94661247
:1038000029960FB6F894DEBF0FBECDBFDF91CF91E2
:103810001F910F91FF90EF90DF90CF90BF90AF90EE
:103820009F908F907F906F905F904F903F902F90E0
:103830000C94D6420E94321381E029960FB6F89478
:10384000DEBF0FBECDBFDF91CF911F910F91FF90D3
:10385000EF90DF90CF90BF90AF909F908F907F9030
:103860006F905F904F903F902F900C94634ED501D6
:103870008D919C91119792FF14C05E962D913D9170
:103880004D915C919197A8EEB3E00E94BBB160931B
:10389000F3027093F4028093F5029093F6020C9475
:1038A000BC261092F3021092F4021092F5021092CC
:1038B000F6020C94BC26F501808183FF0CC0828542
:1038C0009385A485B5858093D8029093D902A0935F
:1038D000DA02B093DB02D5018C9184FF0EC01E96F4
:1038E0008D919D910D90BC91A02D8093DC029093C1
:1038F000DD02A093DE02B093DF02F501808185FF37
:103900000CC082899389A489B5898093E002909341
:10391000E102A093E202B093E3020E94B34ED5010C
:103920008C9186FD02C00C94BC2620911C03309122
:103930001D0356968D919D910D90BC91A02DF9017E
:1039400081879287A387B487808129960FB6F894E0
:10395000DEBF0FBECDBFDF91CF911F910F91FF90C2
:10396000EF90DF90CF90BF90AF909F908F907F901F
:103970006F905F904F903F902F900C941B41D5011A
:10398000ED91FC911197F2FF0DC05E962D913D9146
:103990004D915C919197A8EEB3E00E94BBB16B0191
:1039A0007C0106C040E1C42E47E2D42EE12CF12C6C
:1039B000E3FD0E946212F501808184FD0E94641281
:1039C000D5018C9185FD0E9466120E9472AB2B017D
:1039D0003C014C0C5D1C6E1C7F1C0E9472ABA30151
:1039E0009201261B370B480B590BDA01C901803AAB
:1039F0009648A140B10518F40E94A953EECFD50115
:103A00008C9183FD1798F501808184FD1698D5016E
:103A10008C9185FD02C00C94BC2615980C94BC2694
:103A20000E94824A81110C94BC260E9472AB609362
:103A3000F2187093F3188093F4189093F51880910E
:103A40009B0283FF02C00C94BC26F501808191810A
:103A500093FF02C00C94A82692FF0AC0868D978D12
:103A6000A0A1B1A1892B8A2B8B2B11F40C94A82631
:103A7000D5018D919C91119792FD02C00C94BC26AA
:103A80009C012227317091FF23C0232B89F011E084
:103A900020E030E0A9015A966D917D918D919C9125
:103AA0005D970E94EBAF18160CF010E0212F01C0BB
:103AB00020E085010C5A1F4FF501668D778D80A19E
:103AC00091A129870E948AAE2985D8014C9124C0F2
:103AD000232B81F011E020E030E0A901F501628D97
:103AE000738D848D958D0E94EBAF18160CF010E04D
:103AF000212F01C020E000911C0310911D03D5016E
:103B00005E966D917D918D919C91919729870E94F0
:103B10008AAE2985F801408129960FB6F894DEBF58
:103B20000FBECDBFDF91CF911F910F91FF90EF900E
:103B3000DF90CF90BF90AF909F908F907F906F90CD
:103B40005F904F903F902F900C944A460E94824A7B
:103B500081110C94BC260E9472AB6093F218709392
:103B6000F3188093F4189093F51880919B0283FFCB
:103B700002C00C94BC26D5018D919C91119792FDA9
:103B800002C00C94BC2690FF11C011E020E030E090
:103B9000A9015A966D917D918D919C915D970E949E
:103BA000EBAF18160CF010E0412F01C040E0F5011A
:103BB000668D778D80A191A149870E948AAE498543
:103BC00029960FB6F894DEBF0FBECDBFDF91CF911F
:103BD0001F910F91FF90EF90DF90CF90BF90AF902B
:103BE0009F908F907F906F905F904F903F902F901D
:103BF0000C94D542D5018D919C9133E09695879593
:103C00003A95E1F7817029960FB6F894DEBF0FBEA2
:103C1000CDBFDF91CF911F910F91FF90EF90DF907B
:103C2000CF90BF90AF909F908F907F906F905F905C
:103C30004F903F902F9097CA0E94824A81110C9416
:103C4000BC260E9472AB6093F2187093F3188093B5
:103C5000F4189093F51880919B0283FF02C00C9496
:103C6000BC260E94321320901C0330901D03F501E6
:103C70008081918191FF09C0EC5AFF4F2081211171
:103C800004C02CE0222E22E0322E92FF1EC090FFB4
:103C90000FC011E020E030E0A901D5015A966D91E6
:103CA0007D918D919C915D970E94EBAF18160CF061
:103CB00010E0F501668D778D80A191A10E948AAEFA
:103CC000212FD1014C910E944A46F10126A937A922
:103CD00040AD51AD62A973A984A995A90E9452ADC6
:103CE0002B013C0120E030E0A9010E94EBAF181647
:103CF00064F420E030E040EA50E4C301B2010E94E5
:103D0000B7AD87FF0EC00C94BC2620E030E040EA3F
:103D100050ECC301B2010E94EBAF181614F40C94DE
:103D2000BC2699249394D101D0962D913C91D197A2
:103D30009E968D919C919F97821793070CF0912CE2
:103D40000E9472AB6D837E838F83988710E0412C35
:103D5000512C32010E9472AB69837A838B839C83DE
:103D60006093F2187093F3188093F4189093F518F9
:103D7000DC01CB012D813E814F815885821B930B45
:103D8000A40BB50B893E9340A105B10550F080E02E
:103D9000EAD989819A81AB81BC818D839E83AF836F
:103DA000B88781E00E94191380911C0390911D0334
:103DB0002816390609F062C0D1019396ED90FC9067
:103DC00094971E141F040CF059C0111156C099206D
:103DD00009F475C091966D917C919297882777FD33
:103DE0008095982F0E948AAE9B01AC01F10162A9D7
:103DF00073A984A995A90E94EBAF18160CF0B5C75A
:103E0000662777276E197F09882777FD8095982F79
:103E10000E948AAE2091E4023091E5024091E602D0
:103E20005091E7020E945FB00E9457AE1F921F920E
:103E3000D10152962C9152972F9351962C915197D4
:103E40002F9350962C9150972F931F962C912F9330
:103E50005B016C01E12CF12C870120E030E0A9012D
:103E600060E070E0CB010E94AE9F0F900F900F902A
:103E70000F900F900F9011E078C711E0411451049A
:103E80006104710409F050C09920F1F020E030E0A5
:103E900040E85FE3F10166A977A980AD91AD0E948A
:103EA00052AD9B01AC01D101D2966D917D918D9166
:103EB0009C91D5970E94EBAF87FF1FC048CF41145C
:103EC00051046104710481F520E030E040E85FE3D3
:103ED000F10166A977A980AD91AD0E9453AD9B0118
:103EE000AC01D101D2966D917D918D919C91D59728
:103EF0000E94B7AD18160CF42ACFF101A78DB0A11E
:103F000028EE33E00E94B5B12B013C0129813A81B2
:103F10004B815C81420E531E641E751E4114510478
:103F20006104710409F416CFD301C20129813A81D9
:103F30004B815C81821B930BA40BB50B81159449BB
:103F4000A543B74708F406CF1123E1F180911C0384
:103F500090911D0328163906A9F5D10193966D910C
:103F60007C919497882777FD8095982F0E948AAE40
:103F70002091E4023091E5024091E6025091E7027F
:103F80000E945FB00E9457AE1F921F92F1012289DA
:103F90002F9321892F9320892F9327852F935B01BE
:103FA0006C01E12CF12C870120E030E0A90160E0F8
:103FB00070E0CB010E94AE9F0F900F900F900F907A
:103FC0000F900F900E9472AB6093F2187093F318E9
:103FD0008093F4189093F518CFC680919B0283FDCF
:103FE000CBC60E9472AB4B015C010E9472AB681998
:103FF00079098A099B09693E73408105910530F072
:1040000080E0B1D80E9472AB4B015C0181E00E945C
:10401000191300910A0210910B02D8011B964D90C2
:104020005D906D907C901E9720E030E040EF51E471
:10403000C301B2010E94EBAF18160CF09DC6F80147
:104040002781308541855285C301B2010E9452AD5E
:104050009F7720E030E040E85FE30E94EBAF181666
:1040600024F28AC6D5018D919C91119793FB662706
:1040700060F992FF05C05E968D919C915F970AC092
:104080008FEF90E007C0F501618163FB662760F95F
:1040900080E090E029960FB6F894DEBF0FBECDBF4A
:1040A000DF91CF911F910F91FF90EF90DF90CF9014
:1040B000BF90AF909F908F907F906F905F904F9048
:1040C0003F902F900C944F15D5018D919C91119795
:1040D00092FF04C05E962C9120939B0293FF12C026
:1040E000F50182A193A1A4A1B5A120919B0218166C
:1040F00019061A061B0614F4822B02C08150822373
:1041000080939B0280919B0283FF36C620E040E0B3
:1041100060E070E0CB010E944A4620E040E060E0B1
:1041200070E0CB01F9CC84E09FE10E9427732996CF
:104130000FB6F894DEBF0FBECDBFDF91CF911F91B8
:104140000F91FF90EF90DF90CF90BF90AF909F9036
:104150008F907F906F905F904F903F902F900C9436
:1041600079150E9432138EE49DE10E940F733799F6
:1041700003C085E59DE102C088E59DE10E940F73C3
:1041800087E49DE10E940F730E946812882319F052
:1041900088E59DE102C085E59DE10E940F7380E402
:1041A0009DE10E940F730E946D12882319F088E52B
:1041B0009DE102C085E59DE10E940F7329960FB62F
:1041C000F894DEBF0FBECDBFDF91CF911F910F914D
:1041D000FF90EF90DF90CF90BF90AF909F908F9027
:1041E0007F906F905F904F903F902F900C94A91804
:1041F000E0911C03F0911D032081D5018D919C91CC
:1042000091FF06C0F501EC5AFF4F8081882311F021
:10421000822F01C080E0F501928192FF05C046A483
:1042200057A460A871A803C0412C512C320193FF00
:1042300007C0D501D2964D905D906D907C90D5973A
:10424000082F10E0B3E88B9FF0011124E657FD4FD3
:104250004082518262827382821306C08091770409
:10426000909178040E94D71420E030E0A901C301A6
:10427000B2010E94B7ADB801811103C08AE093E09A
:10428000D1C983EE92E00E94EC7322E0B301A20157
:104290008EED92E055C123FF0DC0F5018285938517
:1042A000A485B5858093AC029093AD02A093AE0235
:1042B000B093AF02D5018C9184FF0EC01E968D91F4
:1042C0009D910D90BC91A02D8093B0029093B1026E
:1042D000A093B202B093B302F501808185FF0CC0B8
:1042E00082899389A489B5898093B4029093B50299
:1042F000A093B602B093B702D5018C9186FF0EC091
:1043000056968D919D910D90BC91A02D8093B802F1
:104310009093B902A093BA02B093BB0229960FB64C
:10432000F894DEBF0FBECDBFDF91CF911F910F91EB
:10433000FF90EF90DF90CF90BF90AF909F908F90C5
:104340007F906F905F904F903F902F900C94B34E62
:1043500023FF0DC0F50182859385A485B5858093E3
:104360009C0290939D02A0939E02B0939F02D50160
:104370008C9184FF0EC01E968D919D910D90BC91E5
:10438000A02D8093A0029093A102A093A202B093CB
:10439000A302F501808185FF0CC082899389A489DD
:1043A000B5898093A4029093A502A093A602B0932E
:1043B000A702D5018C9186FFB1CF56968D919D9124
:1043C0000D90BC91A02D8093A8029093A902A09378
:1043D000AA02B093AB02A2CF32FFCEC4F501868D04
:1043E000978DA0A1B1A1181619061A061B060CF488
:1043F000C3C480939102C0C4E0911C03F0911D03DB
:10440000BB96D5012D913C91119732FF0DC05E9660
:104410008D919D910D90BC91A02D892B8A2B8B2B7A
:1044200009F0AAC4E7E3F2E023FF0BC0D5011A9616
:104430004D915D916D917C911D97428F538F648F4B
:10444000758FD5018C9184FF0AC01E964D915D91A8
:104450006D917C915197468F578F60A371A3D501C1
:104460008C9185FF0AC052964D915D916D917C9122
:10447000559742A353A364A375A3CF0129960FB602
:10448000F894DEBF0FBECDBFDF91CF911F910F918A
:10449000FF90EF90DF90CF90BF90AF909F908F9064
:1044A0007F906F905F904F903F902F900C94D540ED
:1044B00029960FB6F894DEBF0FBECDBFDF91CF9126
:1044C0001F910F91FF90EF90DF90CF90BF90AF9032
:1044D0009F908F907F906F905F904F903F902F9024
:1044E0000C948080F501208123FF0CC08285938588
:1044F000A485B5858093730490937404A093750488
:10450000B093760426FF11C020911C0330911D0347
:10451000F50186899789A08DB18DF901878B908FE0
:10452000A18FB28F80810E941B41409173045091F2
:104530007404609175047091760422E08AE39DE131
:1045400029960FB6F894DEBF0FBECDBFDF91CF9195
:104550001F910F91FF90EF90DF90CF90BF90AF90A1
:104560009F908F907F906F905F904F903F902F9093
:104570000C941075D5018D919C91119792FFFCC3FD
:1045800061E05E968D919D910D90BC91A02D209142
:104590003E05892B8A2B8B2B21F460E0822F8D7FA7
:1045A00002C0822F826080933E0570E085E492E035
:1045B00039C8F5018081918192FF05C0868D978D64
:1045C000A0A1B1A104C084E690E0A0E0B0E02996EB
:1045D0000FB6F894DEBF0FBECDBFDF91CF911F9114
:1045E0000F91FF90EF90DF90CF90BF90AF909F9092
:1045F0008F907F906F905F904F903F902F900C9492
:104600008814D5018D919C91119792FF07C05E96F9
:104610008D919D910D90BC91A02D04C084E690E0F9
:10462000A0E0B0E029960FB6F894DEBF0FBECDBF74
:10463000DF91CF911F910F91FF90EF90DF90CF907E
:10464000BF90AF909F908F907F906F905F904F90B2
:104650003F902F900C94D714F5018081918192FFA7
:104660008BC34FB7F8948091CA059091CB05268DE6
:10467000378D820F931F9093CB058093CA054FBF50
:104680007BC3F501808120911C0330911D0384FFC1
:1046900009C086859785A089B189F90185A396A36C
:1046A000A7A3B0A7D90195964D915D916D917C918D
:1046B000989722E089E09DE10E944D750E94A9181B
:1046C00029960FB6F894DEBF0FBECDBFDF91CF9114
:1046D0001F910F91FF90EF90DF90CF90BF90AF9020
:1046E0009F908F907F906F905F904F903F902F9012
:1046F0000C94994E2091710530917205409173058B
:1047000050917405609183047091840480918504B4
:10471000909186040E9452AD609383047093840448
:10472000809385049093860410927D0510927E05F7
:1047300010927F05109280050E94B34E69E875E0E3
:1047400085E795E00E94949480E00E94B75A4091DA
:10475000830450918404609185047091860422E062
:1047600084EB99E10E94107580E00E94997883E1C2
:104770009DE10E94277388ED92E029960FB6F89488
:10478000DEBF0FBECDBFDF91CF911F910F91FF9084
:10479000EF90DF90CF90BF90AF909F908F907F90E1
:1047A0006F905F904F903F902F900C943C13299600
:1047B0000FB6F894DEBF0FBECDBFDF91CF911F9132
:1047C0000F91FF90EF90DF90CF90BF90AF909F90B0
:1047D0008F907F906F905F904F903F902F900C94B0
:1047E000281880E10E94F3ACBC018EEC92E00E949C
:1047F000F87329960FB6F894DEBF0FBECDBFDF91D8
:10480000CF911F910F91FF90EF90DF90CF90BF90CD
:10481000AF909F908F907F906F905F904F903F9060
:104820002F900C94931882E30E940D18F50180815B
:10483000918192FFA1C2468D578D60A171A188EB35
:1048400092E00E943674D5015E966C9182E30E94DC
:10485000EA17F501668D8AE30E94EA1782E329963A
:104860000FB6F894DEBF0FBECDBFDF91CF911F9181
:104870000F91FF90EF90DF90CF90BF90AF909F90FF
:104880008F907F906F905F904F903F902F900C94FF
:104890000D18FFCFD5018D919C91119792FF0EC0FD
:1048A00021E05E968D919D910D90BC91A02D892B5C
:1048B0008A2B8B2B09F420E0822F01C081E090919C
:1048C0003F05882311F0906801C09F7790933F05C2
:1048D000882319F08EE292E002C084E192E02996EA
:1048E0000FB6F894DEBF0FBECDBFDF91CF911F9101
:1048F0000F91FF90EF90DF90CF90BF90AF909F907F
:104900008F907F906F905F904F903F902F900C947E
:104910002773F5010081118112FF03C0668D778D29
:1049200002C066E970E013FF0CC0D5019296ED90CD
:10493000FC9093971E141F0434F4EE24E394F12C9E
:1049400002C0E12CF12CA3E016950795AA95E1F79A
:104950000170882777FD8095982F0E948AAEAB0161
:10496000BC01F701EE0FFF1FE65FFD4F2E2D80818A
:1049700091810E94264700C280E00E948E61D5018D
:104980008D919C91119792FFF7C15E968D919D91AB
:104990000D90BC91A02D0097A105B10509F0DCC1D7
:1049A000EBC1F5018081918192FFE6C1868D978DE3
:1049B000A0A1B1A1892B8A2B8B2B09F4DDC180E04A
:1049C00029960FB6F894DEBF0FBECDBFDF91CF9111
:1049D0001F910F91FF90EF90DF90CF90BF90AF901D
:1049E0009F908F907F906F905F904F903F902F900F
:1049F0000C9499788BE692E00E942773D5018D91F3
:104A00009C9192FD0FC0F501808183FF16C0F501D6
:104A100062857385848595850E945CAE80E00E94E6
:104A2000F2160BC010E0D5015E966C91812F0E94AA
:104A3000F2161F5F1530B9F7E6CFD5018C9184FFD0
:104A40000BC01E966D917D918D919C9151970E9406
:104A50005CAE81E00E94F216F501808185FF09C0FD
:104A600062897389848995890E945CAE82E00E9484
:104A7000F216D5018C9186FF0BC056966D917D91F3
:104A80008D919C9159970E945CAE83E00E94F21632
:104A9000F5018081918193FF04C062A184E00E94AE
:104AA000F21629960FB6F894DEBF0FBECDBFDF9188
:104AB000CF911F910F91FF90EF90DF90CF90BF901B
:104AC000AF909F908F907F906F905F904F903F90AE
:104AD0002F900C940917D5018D919C91119792FFFD
:104AE00026C081E05E964D915D916D917C9191978C
:104AF000452B462B472B09F480E029960FB6F894F6
:104B0000DEBF0FBECDBFDF91CF911F910F91FF9000
:104B1000EF90DF90CF90BF90AF909F908F907F905D
:104B20006F905F904F903F902F900C94FB69299667
:104B30000FB6F894DEBF0FBECDBFDF91CF911F91AE
:104B40000F91FF90EF90DF90CF90BF90AF909F902C
:104B50008F907F906F905F904F903F902F900C942C
:104B6000FC6929960FB6F894DEBF0FBECDBFDF916A
:104B7000CF911F910F91FF90EF90DF90CF90BF905A
:104B8000AF909F908F907F906F905F904F903F90ED
:104B90002F900C940A6A29960FB6F894DEBF0FBEC8
:104BA000CDBFDF91CF911F910F91FF90EF90DF90DC
:104BB000CF90BF90AF909F908F907F906F905F90BD
:104BC0004F903F902F900C945A60F5018081918115
:104BD00090FF05C0E28CF38C048D158D08C0E09029
:104BE0007B04F0907C0400917D0410917E049C0174
:104BF00046E0369527954A95E1F72170AC0165E0CE
:104C0000569547956A95E1F74170BC01E4E07695C9
:104C10006795EA95E1F76170F3E096958795FA95C7
:104C2000E1F781700E94BB60A7C080E00E94997884
:104C30008AEA98E10BC00E94E67AE0911C03F091A9
:104C40001D0380810E941B4188E898E129960FB6D8
:104C5000F894DEBF0FBECDBFDF91CF911F910F91B2
:104C6000FF90EF90DF90CF90BF90AF909F908F908C
:104C70007F906F905F904F903F902F900C943E7379
:104C800029960FB6F894DEBF0FBECDBFDF91CF914E
:104C90001F910F91FF90EF90DF90CF90BF90AF905A
:104CA0009F908F907F906F905F904F903F902F904C
:104CB0000C94CC7682E592E00E942773D5018D9109
:104CC0009C9188279C7081159C4009F055C0F50186
:104CD000668D778D82A129960FB6F894DEBF0FBE40
:104CE000CDBFDF91CF911F910F91FF90EF90DF909B
:104CF000CF90BF90AF909F908F907F906F905F907C
:104D00004F903F902F900C94401680919B0282FF11
:104D100033C089E19EE10E940F73C50129960FB649
:104D2000F894DEBF0FBECDBFDF91CF911F910F91E1
:104D3000FF90EF90DF90CF90BF90AF909F908F90BB
:104D40007F906F905F904F903F902F900C941C71CC
:104D50000E9432130C94381D0397A105B10509F088
:104D60002ECE80E00E94DA652ACE411451046104FF
:104D7000710409F48BC8D8C829960FB6F894DEBF21
:104D80000FBECDBFDF91CF911F910F91FF90EF909C
:104D9000DF90CF90BF90AF909F908F907F906F905B
:104DA0005F904F903F902F9008952F923F924F9297
:104DB0005F926F927F928F929F92AF92BF92CF92AB
:104DC000DF92EF92FF920F931F93CF93DF93CDB7B4
:104DD000DEB7EC970FB6F894DEBF0FBECDBF1C0157
:104DE000DC0118968D919C9119978032910509F4F8
:104DF00036C458F58531910509F45EC198F48430C4
:104E0000910509F41BC128F4029708F4ECC00C9436
:104E10007336449711F00C94733681E08093C90582
:104E20000C947E368D31910509F4AEC128F44C976F
:104E300009F446C10C9473368E31910509F41EC3F2
:104E40004F9709F4F9C30C9473368C35910511F41E
:104E50000C94A03248F58534910511F40C948E2FF2
:104E6000B8F48434910511F00C94733680917B046E
:104E700090917C04A0917D04B0917E048D879E87E3
:104E8000AF87B88B49E1442E512C612C712C71C62F
:104E90008A35910511F40C9485328B35910511F406
:104EA0000C9491320C9473368438910511F40C945F
:104EB000373508F05DC08436910511F40C948233C7
:104EC0008338910511F00C947336609169057091E7
:104ED0006A0580916B0590916C0520916D0530916C
:104EE0006E0540916F0550917005E0907105F0904E
:104EF0007205009173051091740540907B045090E9
:104F00007C0460907D0470907E0410926F04109277
:104F10007004109271041092720410926B0410923B
:104F20006C0410926D0410926E04E091BF02EF9336
:104F3000E091BE02EF93E091BD02EF93E091BC02DD
:104F4000EF93E0EFAE2EE3E2BE2EE4E7CE2EE9E4EF
:104F5000DE2E0E94FA5740927B0450927C046092AD
:104F60007D0470927E0480E00E94B75A0C94323522
:104F70008538910511F40C94BE358638910511F0F1
:104F80000C9473364091890550918A0560918B0588
:104F900070918C0583E094E00E941E7440918D0511
:104FA00050918E0560918F05709190058FE89DE17D
:104FB0000E941E7440919105509192056091930555
:104FC000709194058FE89DE10E94367480E00E9404
:104FD000B75A85EF93E00E940F738FEE93E00E9423
:104FE0003C130C947E36F1018081918192FF11C0B7
:104FF000868D978DA0A1B1A120913F05892B8A2B89
:105000008B2B19F0822F806202C0822F8F7D8093BC
:105010003F05C1010E942E5C882311F40C947E365A
:1050200041E061E081E00E947B9A81110C947E3620
:1050300085E29BE00E9434730C947E360E9432130A
:10504000D1018D919C91119793FF07C092968D90FD
:105050009D90AD90BC90959703C0812C912C5401EC
:1050600092FF0BC0F101268D378D40A151A1A8EE12
:10507000B3E00E94BBB14B015C010E9472AB6B01BB
:105080007C01C80CD91CEA1CFB1C0E9472ABA70156
:105090009601261B370B480B590BDA01C901811504
:1050A0009449A543B74710F00C947E360E94F971DD
:1050B00081E00E941913E9CF1092C9050C947E3645
:1050C000D1018D919C91AC01487355274115510533
:1050D00051F49C0166E0369527956A95E1F7B1E0B9
:1050E0002B27217001C020E086FF08C010928105A7
:1050F000109282051092830510928405211117C029
:10510000452BD1F0AC0125E0569547952A95E1F75E
:10511000BC0134E0769567953A95E1F753E09695B2
:1051200087955A95E1F761704170817003C061E025
:1051300041E081E00E94A86180E00E94B75A37995F
:1051400002C00C94A13682E19BE00E94D86F8AE0F5
:105150009BE00E940F73379B04C087E09BE00E9496
:105160000F730E946812882321F084E09BE00E9464
:105170000F730E946D12882321F081E09BE00E9452
:105180000F7381EE9AE083C00E949318811111C0C1
:105190006AEF70E080E090E00E94A1AB0E9493185B
:1051A000811107C081EC9AE00E94277388EA9AE097
:1051B00061C183E99AE00E94D86F20917B0430910D
:1051C0007C0440917D0450917E04298F3A8F4B8F4F
:1051D0005C8F80E090E00E94B91280E090E00E9435
:1051E000D91280E090E00E94F91280E00E94997844
:1051F0000E94E67A80E090E4A7EEB4E48093A402F3
:105200009093A502A093A602B093A7020E94B34E6A
:1052100089E190E0A0E0B0E0898B9A8BAB8BBC8BEE
:105220008BE1482E512C612C712C1DA229893A89C1
:105230004B895C892D873E874F87588B41E061E021
:1052400081E00E94A861379902C00C94AC3680E8D6
:105250009AE00E94D86F88E79AE00E940F73379B0C
:1052600004C085E79AE00E940F730E9468128823A9
:1052700021F082E79AE00E940F730E946D1288234A
:1052800021F08FE69AE00E940F738FE49AE00E946B
:1052900027730C947E3684EF99E00E9427738CED7F
:1052A00099E00E94D86F84EC99E10E944873EDA1C7
:1052B000E1110C947E3681E00E94B75A298D3A8D17
:1052C0004B8D5C8D20937B0430937C0440937D0454
:1052D00050937E048AE998E00E943C138CE29AE1A4
:1052E0000E94D86F212C312C8091EF049091F00412
:1052F000A091F104B091F204898B9A8BAB8BBC8B9B
:1053000080E00E9499780E94E67A81E00E948E6196
:1053100041E061E081E00E94A86180E00E948E612E
:105320008DE29AE10E94D86F0E9471129F938F9331
:105330007F936F93B0EFAB2EB3E2BB2EB4E7CB2ECF
:10534000B9E4DB2E8601750120E030E0A901CA0135
:10535000B9010E94655F20E041E060E081E00E94C9
:105360002F626B017C0120E041E060E081E00E945F
:105370002F624B015C019B01AC01C701B6010E9489
:1053800052AD2B013C010F900F900F900F902DEC20
:105390003CEC4CEC5DE30E94EBAF181614F00C945F
:1053A000CD394D855E856F85788986E698E00E94C7
:1053B00036742D853E854F85588928323105410543
:1053C000510514F00C94D93982E30E940D188D8593
:1053D0009E85AF85B8890296A11DB11D8D879E87D8
:1053E000AF87B88BAC01BD0188E498E00E943674A9
:1053F0006D8582E30E94EA176D858AE30E94EA17B1
:1054000082E30E940D18B4E02B1631040CF46CCF2B
:1054100080E090E0A8ECB3E48093A4029093A5020E
:10542000A093A602B093A7020E94B34E81E00E940F
:105430008E6181E00E94B75A89E397E00E943C1395
:105440008CE29AE10E94D86F298D3A8D4B8D5C8D4C
:1054500020937B0430937C0440937D0450937E041E
:1054600041E061E081E00E94A86180E00E949978BB
:105470008FE197E00E94D86F0C947E36D1018D9118
:105480009C91119792FD02C00C94B73B5E968D9152
:105490009D910D90BC91A02D0297A105B10511F031
:1054A0000C94B73B80917B0490917C04A0917D0487
:1054B000B0917E048D879E87AF87B88BF101808184
:1054C000918192FF0AC0868D978DA0A1B1A102970C
:1054D000A105B10511F40C94513C41E061E081E07B
:1054E0000E94A8618DE29AE10E94D86F80E00E943C
:1054F0008E610E9471129F938F937F936F93F0EF51
:10550000AF2EF3E2BF2EF4E7CF2EF9E4DF2E8601B3
:10551000750120E030E0A901CA01B9010E94655F70
:1055200020E041E060E081E00E942F624B015C01DD
:1055300020E041E060E081E00E942F626B017C018D
:105540009B01AC01C501B4010E9452AD2B013C018D
:105550000F900F900F900F902DEC3CEC4CEC5DE316
:105560000E94EBAF181654F02DEC3CEC4CEC5DEBCC
:10557000C301B2010E94B7AD87FF05C084EC99E179
:105580000E9448739BCFA5019401C701B6010E94F8
:1055900053AD20E030E040E05FE30E945FB06B017C
:1055A0007C0120E030E040E85FE30E94B7AD87FD7A
:1055B00085CFD1018D919C91119792FF0CC05E9681
:1055C0008D919D910D90BC91A02D892B8A2B8B2BB9
:1055D00011F00C94643C2D853E854F8558892093AD
:1055E0007B0430937C0440937D0450937E0481E0DF
:1055F0000E948E61D1018D919C91119792FF0CC0F8
:105600005E968D919D910D90BC91A02D0297A10564
:10561000B10511F40C94883C81E00E94B75A8AE1EC
:1056200097E00E943C138CE29AE10E94D86F2D858E
:105630003E854F85588960C78AE39AE10E940F73BF
:105640008091000181FD02C068E401C06CE480EA41
:1056500096E00E9444820E94A9180C947E368DE246
:105660009AE10E94D86F1092490510924A05109253
:105670004B0510924C05109245051092460510926C
:10568000470510924805109241051092420510926C
:1056900043051092440580E00E948E6120917B04B6
:1056A00030917C0440917D0450917E0429A33AA35B
:1056B0004BA35CA30E947112162F072FF82EE92E20
:1056C00084E393E00E944A129B01AC0180E393E0E3
:1056D00029AF3AAF4BAF5CAF0E944A12EF92FF92F4
:1056E0000F931F9350EFA52E53E2B52E54E7C52E0E
:1056F00059E4D52E8601750129AD3AAD4BAD5CADAF
:105700000E94655F20E041E060E081E00E942F623E
:105710002B013C010F900F900F900F9020E030E094
:10572000A9010E94B7AD87FF02C00C947E360E948B
:105730007112162F072FF82EE92E8CE393E00E94AA
:105740004A129B01AC0188E393E029AF3AAF4BAF1B
:105750005CAF0E944A12EF92FF920F931F93860153
:10576000750129AD3AAD4BAD5CAD0E94655F21E09E
:1057700041E060E080E00E942F626D877E878F8726
:10578000988B0F900F900F900F9020E030E0A901C0
:105790000E94B7AD87FF02C00C947E360E94711242
:1057A000162F072FF82EE92E84E493E00E944A1268
:1057B0009B01AC0180E493E029AF3AAF4BAF5CAF03
:1057C0000E944A12EF92FF920F931F938601750178
:1057D00029AD3AAD4BAD5CAD0E94655F21E041E083
:1057E00061E080E00E942F624B015C010F900F90FE
:1057F0000F900F9020E030E0A9010E94B7AD87FF25
:1058000002C00C947E36850174012D853E854F853E
:105810005889C301B2010E94CD678091150590910E
:105820001605A0911705B09118058D879E87AF8743
:10583000B88B2091290530912A0540912B05509174
:105840002C05298B3A8B4B8B5C8BC0901D05D0901F
:105850001E05E0901F05F090200580912105909194
:105860002205A0912305B09124058D8B9E8BAF8BD3
:10587000B88F2091790530917A0540917B05509140
:105880007C052DA33EA34FA358A78091BD05909101
:10589000BE05A091BF05B091C00589A79AA7ABA787
:1058A000BCA72091250530912605409127055091F0
:1058B00028052D8F3E8F4F8F58A380911905909109
:1058C0001A05A0911B05B0911C05898F9A8FAB8F8B
:1058D000BC8F2091750530917605409177055091E8
:1058E00078052DA73EA74FA758AB8091B905909199
:1058F000BA05A091BB05B091BC0589AB9AABABAB27
:10590000BCAB10927F04109280041092810410921C
:105910008204D1018D919C91119792FFDCC05E961B
:105920008D919D910D90BC91A02DAC01BD01415078
:10593000510961097109423051056105710548F04D
:105940000397A105B10509F0C6C080E00E949978CF
:10595000C2C029893A894B895C896D857E858F858E
:1059600098890E945FB02B013C012D893E894F89A7
:10597000588DC701B6010E945FB09B01AC01C30105
:10598000B2010E9452AD2B013C016DA17EA18FA1FD
:1059900098A50E948AAE9B01AC01C301B2010E948E
:1059A0005FB029A53AA54BA55CA50E945FB02B016D
:1059B0003C012D8D3E8D4F8D58A1C701B6010E942F
:1059C0005FB06B017C0129893A894B895C89698DBB
:1059D0007A8D8B8D9C8D0E945FB09B01AC01C701BD
:1059E000B6010E9452AD6B017C016DA57EA58FA50D
:1059F00098A90E948AAE9B01AC01C701B6010E9422
:105A00005FB029A93AA94BA95CA90E945FB09B018C
:105A1000AC01C301B2010E9453AD6B017C01F7FAE6
:105A2000F094F7F8F0942D893E894F89588D698D4F
:105A30007A8D8B8D9C8D0E945FB02B013C012D8D4A
:105A40003E8D4F8D58A16D857E858F8598890E94EA
:105A50005FB09B01AC01C301B2010E9452AD9B013A
:105A6000AC01C701B6010E94BEAD9B01AC01C501EE
:105A7000B4010E9453AD209171053091720540919F
:105A80007305509174050E9452AD209183043091AA
:105A9000840440918504509186040E9453ADAB016B
:105AA000BC014093830450938404609385047093F5
:105AB000860422E084EB99E10E94107581E00E9447
:105AC0008E61F101868D978DA0A1B1A10297A105EC
:105AD000B10509F43ACF81E00E948E610E94B34E75
:105AE00081E00E94B75A87EC96E00E943C1341E0A7
:105AF00061E081E00E94A86129A13AA14BA15CA1CB
:105B000020937B0430937C0440937D0450937E0467
:105B10000C947E362DEC3CEC4CEC5DEBC701B601F1
:105B20000E94B7AD87FF85C0B301A20187EA96E066
:105B30000E94367438E24316510461047104CCF4B7
:105B400082E30E940D1842E0440E511C611C711C3E
:105B5000B301A20189E896E00E943674642D82E3C5
:105B60000E94EA17642D8AE30E94EA1782E30E94EA
:105B70000D182091EF043091F0044091F104509100
:105B8000F204298F3A8F4B8F5C8F80E00E949978C6
:105B90000E94E67A41E061E081E00E94A8618DE226
:105BA0009AE10E94D86F80E00E948E610E9471127B
:105BB0009F938F937F936F9330EFA32E33E2B32E97
:105BC00034E7C32E39E4D32E8601750120E030E09E
:105BD000A901CA01B9010E94655F20E041E060E0CF
:105BE00081E00E942F62698B7A8B8B8B9C8B20E0EB
:105BF00041E060E081E00E942F626D8B7E8B8F8B95
:105C0000988F9B01AC0169897A898B899C890E9454
:105C100052AD6B017C010F900F900F900F902DEC07
:105C20003CEC4CEC5DE30E94EBAF18160CF072CF2D
:105C30007BCF0E947112162F072FF82EE92E84E4D5
:105C400093E00E944A129B01AC0180E493E029AFEB
:105C50003AAF4BAF5CAF0E944A12EF92FF920F93A4
:105C60001F9320EFA22E23E2B22E24E7C22E29E4B6
:105C7000D22E8601750129AD3AAD4BAD5CAD0E94C7
:105C8000655F21E041E061E080E00E942F624B010E
:105C90005C0121E041E061E080E00E942F626B0145
:105CA0007C019B01AC01C501B4010E9452AD6D8F16
:105CB0007E8F8F8F98A30F900F900F900F902DECE9
:105CC0003CEC4CEC5DE30E94EBAF181664F02DEC5D
:105CD0003CEC4CEC5DEB6D8D7E8D8F8D98A10E9420
:105CE000B7AD87FF13C0B301A20189E696E00E9419
:105CF000367482E30E940D1852E0450E511C611C5F
:105D0000711CB301A2018BE496E026CF29893A8960
:105D10004B895C896D897E898F89988D0E9453ADEE
:105D200020E030E040E05FE30E945FB0698B7A8B57
:105D30008B8B9C8B20E030E0A9010E94B7AD87FDE2
:105D400018CFA5019401C701B6010E9453AD20E010
:105D500030E040E05FE30E945FB09B01AC016989E5
:105D60007A898B899C890E9452AD20E030E040EA1C
:105D700052E40E945FB06B017C0120E030E0A90199
:105D80000E94B7AD87FF31C0F7FAF094F7F8F094AE
:105D900022E0B701A60188E59AE10E9410752091E2
:105DA000EF043091F0044091F1045091F204C701E6
:105DB000B6010E94BEAD9B01AC010E9453AD6B01C8
:105DC0007C0122E0AB01BC0188E59AE10E941075DC
:105DD000A70196016091EF047091F0048091F104A5
:105DE0009091F2040E9452AD18C08090EF04909000
:105DF000F004A090F104B090F204A5019401C70151
:105E0000B6010E94BEAD9B01AC010E9453AD9B0147
:105E1000AC01C501B4010E9453AD6093EF047093CF
:105E2000F0048093F1049093F20420E030E042E823
:105E300052E46091EF047091F0048091F10490912C
:105E4000F2040E94BEAD6B017C012DEC3CEC4CE8F1
:105E50005FE30E94EBAF181654F026E636E646E6FE
:105E60005FE3C701B6010E94B7AD87FF12C080E0B3
:105E700090E0A2E8B2E48093EF049093F004A09342
:105E8000F104B093F20422E0AC01BD0180E396E09E
:105E900014C022E0498D5A8D6B8D7C8D83E296E093
:105EA0000E9410754091EF045091F0046091F1044C
:105EB0007091F20422E086E196E00E9410758D85D3
:105EC0009E85AF85B88980937B0490937C04A093D2
:105ED0007D04B0937E0481E00E948E6181E00E9487
:105EE000B75A81E196E00E943C138CE29AE10E944D
:105EF000D86F2D853E854F85588920937B0430933C
:105F00007C0440937D0450937E0441E061E081E095
:105F10000E94A86180E00E949978F0C680917B047D
:105F200090917C04A0917D04B0917E048D8F9E8F12
:105F3000AF8FB8A329E130E040E050E02D873E87E5
:105F40004F87588BD1018D919C91119792FF0CC076
:105F50005E968D919D910D90BC91A02D0297A1050B
:105F6000B10511F40C94D83C41E061E081E00E945D
:105F7000A8618DE29AE10E94D86F80E00E948E6154
:105F80000E947112162F072FF82EE92E84E393E05A
:105F90000E944A129B01AC0180E393E029AF3AAF23
:105FA0004BAF5CAF0E944A12EF92FF920F931F9388
:105FB00000EFA02E03E2B02E04E7C02E09E4D02E9D
:105FC0008601750129AD3AAD4BAD5CAD0E94655FB0
:105FD00020E041E060E081E00E942F62698F7A8FCB
:105FE0008B8F9C8F20E041E060E081E00E942F6277
:105FF00069A37AA38BA39CA39B01AC01698D7A8DC5
:106000008B8D9C8D0E9452AD6B017C010F900F9087
:106010000F900F902DEC3CEC4CEC5DE30E94EBAF4D
:10602000181654F02DEC3CEC4CEC5DEBC701B601BE
:106030000E94B7AD87FF2BC04D855E856F8578893F
:1060400081EF95E00E9436742D853E854F855889F5
:1060500028323105410551050CF074CF82E30E94CE
:106060000D18D1018D919C9192FF6CCF2D853E85AD
:106070004F8558892E5F3F4F4F4F5F4F2D873E878B
:106080004F87588BBA01A90183ED95E086C08DE753
:1060900093E00E94CCB59A8B898B0E947112162FC7
:1060A000072FF82EE92E8CE393E00E944A129B0101
:1060B000AC0188E393E029AF3AAF4BAF5CAF0E94ED
:1060C0004A12EF92FF920F931F9310EFA12E13E24B
:1060D000B12E14E7C12E19E4D12E8601750129AD28
:1060E0003AAD4BAD5CAD0E94655F21E041E060E000
:1060F00080E00E942F626DA37EA38FA398A721E06A
:1061000041E060E080E00E942F6269A77AA78BA738
:106110009CA79B01AC016DA17EA18FA198A50E94B7
:1061200052AD6B017C010F900F900F900F902DECF2
:106130003CEC4CEC5DE30E94EBAF181654F02DECF8
:106140003CEC4CEC5DEBC701B6010E94B7AD87FF9C
:1061500032C04D855E856F85788983EB95E00E941E
:1061600036748D859E85AF85B8898897A105B10560
:106170000CF0E8CE82E30E940D182D853E854F85F8
:1061800058892E5F3F4F4F4F5F4F2D873E874F8778
:10619000588BBA01A90185E995E00E9436746D8596
:1061A00082E30E94EA176D858AE30E94EA1782E380
:1061B0000E940D18C7CE8FE793E00E94CCB59E8B4E
:1061C0008D8B0E947112162F072FF82EE92E84E472
:1061D00093E00E944A129B01AC0180E493E029AF56
:1061E0003AAF4BAF5CAF0E944A12EF92FF920F930F
:1061F0001F93B0EFAB2EB3E2BB2EB4E7CB2EB9E4C6
:10620000DB2E8601750129AD3AAD4BAD5CAD0E9428
:10621000655F21E041E061E080E00E942F624B0178
:106220005C0121E041E061E080E00E942F626B01AF
:106230007C019B01AC01C501B4010E9452AD2B0150
:106240003C010F900F900F900F902DEC3CEC4CEC1C
:106250005DE30E94EBAF181654F02DEC3CEC4CECD7
:106260005DEBC301B2010E94B7AD87FF25C04D852C
:106270005E856F85788985E795E00E9436748D8507
:106280009E85AF85B8898897A105B1050CF05ACED7
:1062900082E30E940D182D853E854F8558892E5F1B
:1062A0003F4F4F4F5F4F2D873E874F87588BBA0127
:1062B000A90187E595E071CFA5019401C701B60159
:1062C0000E9453AD20E030E040E05FE30E945FB009
:1062D0006DA77EA78FA798AB81E893E00E94CCB50D
:1062E0008C01D1018D919C91119792FF0CC05E960B
:1062F0008D919D910D90BC91A02D892B8A2B8B2B7C
:1063000011F00C94EB3C298D3A8D4B8D5C8D69A17D
:106310007AA18BA19CA10E9453AD20E030E040E027
:106320005FE30E945FB0698F7A8F8B8F9C8F2D8D7A
:106330003E8D4F8D58A120937B0430937C04409375
:106340007D0450937E0481E00E948E61D1018D9185
:106350009C91119792FFABC05E968D919D910D908F
:10636000BC91A02D0297A105B10509F0A0C020E0C5
:1063700030E040EA52E4698D7A8D8B8D9C8D0E94CD
:106380005FB020E030E048EC54E40E9452AD0E943F
:1063900057AE6B017C0129893A89442737FD409526
:1063A000542F298B3A8B4B8B5C8B2DA13EA14FA197
:1063B00058A569A57AA58BA59CA50E9453AD20E0A0
:1063C00030E040E05FE30E945FB020E030E040EA70
:1063D00052E40E945FB020E030E048EC54E40E94B8
:1063E00052AD0E9457AE2B013C018D899E89AA2790
:1063F00097FDA095BA2F8D8B9E8BAF8BB88F20E029
:1064000030E040EA52E46DA57EA58FA598A90E94D0
:106410005FB020E030E048EC54E40E9452AD0E94AE
:1064200057AE4B015C01222717FD2095322FC41473
:10643000D504E604F70414F00C94033DC814D90401
:10644000EA04FB0414F00C942B3D4C185D086E0814
:106450007F088D899E89AF89B88D480E591E6A1EA6
:106460007B1E8C189D08AE08BF08800E911EA21ED0
:10647000B31EC2010E94D912C4010E94F912C12C9C
:10648000D12C7601A1E94A16A1E05A0661047104F3
:1064900014F00C945F3DB1E98B16B1E09B06A104AA
:1064A000B10414F00C945F3D80E00E94997820E0E4
:1064B00030E0A901698D7A8D8B8D9C8D0E94B7ADDE
:1064C00087FD40CD20E030E0A9016DA57EA58FA518
:1064D00098A90E94B7AD87FD35CD81E00E94B75ADB
:1064E0008DE195E00E943C138CE29AE10E94D86F06
:1064F0002D8D3E8D4F8D58A120937B0430937C04CD
:1065000040937D0450937E04E8C310928605F10108
:10651000EB5AFF4F8081882309F4F0C388E095E0AF
:106520000CC081E080938605F101EB5AFF4F80811A
:10653000882309F4E3C383EF94E00E943E73DEC333
:106540008090410590904205A0904305B09044058D
:10655000409045055090460560904705709048056D
:10656000C0904905D0904A05E0904B05F0904C054D
:10657000D1011C9113FF2BC01A96EC911A971B9610
:10658000FC911B971C960C911C971D96BC908091BA
:10659000C905882361F023E333E34BEC51E4BF01E9
:1065A000802F9B2D0E945FB0FB01DC0102C0A02F59
:1065B000BB2D2091690530916A0540916B05509182
:1065C0006C05BF01CD010E9452AD4B015C0114FF6F
:1065D0002CC0D1011E96EC911E971F96FC911F971F
:1065E00050960C91509751967C908091C9058823C4
:1065F00061F023E333E34BEC51E4BF01802F972D8F
:106600000E945FB0FB01DC0102C0A02FB72D2091DA
:106610006D0530916E0540916F0550917005BF0179
:10662000CD010E9452AD2B013C0115FF2CC0D101C0
:106630005296EC9152975396FC91539754961C9115
:10664000549755960C918091C905882361F023E3F6
:1066500033E34BEC51E4BF01812F902F0E945FB0D8
:10666000FB01DC0102C0A12FB02F209171053091F8
:1066700072054091730550917405BF01CD010E94D0
:1066800052AD6B017C0187017601A3019201C50126
:10669000B4010E948853F101808186FF2FC3E689EF
:1066A000D1015796FC91579758961C915897599637
:1066B0000C918091C905882361F023E333E34BEC0F
:1066C00051E4BF01812F902F0E945FB0FB01DC01DC
:1066D00002C0A12FB02F2091E4023091E502409139
:1066E000E6025091E702BF01CD010E945FB00E9417
:1066F00057AE6093810570938205809383059093D4
:106700008405FCC28090710590907205A09073057D
:10671000B0907405209183043091840440918504E5
:1067200050918604C501B4010E94BEAD2DEC3CEC35
:106730004CEC5DE30E94EBAF18162CF48DEB94E06B
:106740000E944873DBC2F10122818081918122FF86
:106750000CC083FF02C00C947B3D80739927892B6A
:1067600011F00C947B3D0C94813D83FF6FC0C2847B
:10677000D384E484F58420E030E0A901C701B601A8
:106780000E94EBAF181664F420E030E040E251E4E0
:10679000C701B6010E94B7AD18160CF459C00AC063
:1067A00020E030E040E251ECC701B6010E94EBAFBF
:1067B00087FD4EC0A5019401C701B6010E9453ADEB
:1067C0009B01AC0160918F047091900480919104C1
:1067D000909192040E9453AD60938F047093900443
:1067E00080939104909392040E94B34E40918F0441
:1067F00050919004609191047091920423E080EC98
:1068000093E00E94107580918F0490919004A09164
:106810009104B091920489879A87AB87BC8744E042
:1068200050E065E870E0CE0109960E94D1B50E9463
:106830008278682F88E690E069AF0E94BFB569ADA5
:10684000681721F088E690E00E94DAB510E001C0F8
:1068500011E0F101808184FF71C0C684D784E08893
:10686000F18820E030E0A901C701B6010E94EBAF3A
:10687000181664F420E030E040E251E4C701B601AC
:106880000E94B7AD18160CF458C00AC020E030E0E2
:1068900040E251ECC701B6010E94EBAF87FD4DC04D
:1068A000A5019401C701B6010E9453AD9B01AC0143
:1068B00060918704709188048091890490918A0482
:1068C0000E9453AD60938704709388048093890479
:1068D00090938A040E94B34E40918704509188049B
:1068E0006091890470918A0423E085EA93E00E9414
:1068F00010758091870490918804A0918904B091CB
:106900008A048D839E83AF83B88744E050E069E8B2
:1069100070E0CE0105960E94D1B50E948278682F62
:1069200088E690E069AF0E94BFB569AD681731F0A5
:1069300088E690E00E94DAB501C011E0D1018C91A7
:1069400085FF74C05296CD90DD90ED90FC905597E8
:1069500020E030E0A901C701B6010E94EBAF181694
:106960005CF420E030E040E251E4C701B6010E944F
:10697000B7AD18165CF00EC020E030E040E251ECFC
:10698000C701B6010E94EBAF87FF04C08EE094E020
:106990000C947D3DA5019401C701B6010E9453AD41
:1069A0009B01AC0160917F0470918004809181040F
:1069B000909182040E9453AD60937F047093800491
:1069C00080938104909382040E94B34E40917F048F
:1069D00050918004609181047091820423E08AE8E0
:1069E00093E00E94107580917F0490918004A091A3
:1069F0008104B091820489839A83AB83BC8344E091
:106A000050E06DE870E0CE0101960E94D1B50E9481
:106A10008278682F88E690E069AF0E94BFB569ADC3
:106A2000681721F088E690E00E94DAB51111AECF28
:106A300089E48F9384E78F9383E28F9380EF8F9322
:106A4000F0EFAF2EF3E2BF2EF4E7CF2EF9E4DF2E06
:106A5000E12CF12C00E411E4A6019501C601B50179
:106A60000E94655F0F900F900F900F9047C180E0DC
:106A70000E948E61109241051092420510924305CA
:106A80001092440510924505109246051092470554
:106A9000109248051092490510924A0510924B0534
:106AA00010924C056091C4027091C5028091C6029B
:106AB0009091C7020E9407548091BF049091C00436
:106AC000A091C104B091C2044091B7045091B804A0
:106AD0006091B9047091BA04C090BB04D090BC041A
:106AE000E090BD04F090BE045A01F62FE72F48173E
:106AF00059076A077B071CF45C01FA2FEB2F85010D
:106B00002F2F3E2F0C151D052E053F0514F4970160
:106B10008601480159018C189D08AE08BF0868011C
:106B20007901C41AD50AE60AF70A28013901481A78
:106B3000590A6A0A7B0AB501A40188ED9CE10E940A
:106B40003674B701A6018FEC9CE10E943674B30144
:106B5000A20186EC9CE10E943674F1018081918152
:106B600092FFBBC0868D978DA0A1B1A11816190602
:106B70001A061B0614F40C942D3EAFC0709040050D
:106B800075FA772470F880E00E948E611092750586
:106B9000109276051092770510927805109279057B
:106BA00010927A0510927B0510927C0510927D055B
:106BB00010927E0510927F0510928005109241057B
:106BC000109242051092430510924405109245051B
:106BD00010924605109247051092480510924905FB
:106BE00010924A0510924B0510924C05109289059F
:106BF00010928A0510928B0510928C0510928D05CB
:106C000010928E0510928F051092900510929105AA
:106C10001092920510929305109294056091C4020F
:106C20007091C5028091C6029091C7020E940754DC
:106C30000091A3041091A4042091A5043091A6040E
:106C40008091970490919804A0919904B0919A042E
:106C5000081B190B2A0B3B0B08511C4F2F4F3F4FA2
:106C60008091B7049091B804A091B904B091BA048E
:106C700048015901881A990AAA0ABB0A8091BF04DF
:106C80009091C004A091C104B091C204680179013F
:106C9000C81AD90AEA0AFB0A8091BB049091BC0485
:106CA000A091BD04B091BE04B901A801481B590BC5
:106CB0006A0B7B0B88ED9CE10E943674B501A40140
:106CC0008FEC9CE10E943674B701A60186EC9CE132
:106CD0000E943674872D0E948E6141E061E081E060
:106CE0000E94A8610BC080919B0282FF07C089E1CE
:106CF0009EE10E940F73C1010E941C710E9472AB41
:106D00006093F2187093F3188093F4189093F51829
:106D1000EC960FB6F894DEBF0FBECDBFDF91CF91DA
:106D20001F910F91FF90EF90DF90CF90BF90AF90A9
:106D30009F908F907F906F905F904F903F902F909B
:106D400008950E94681281110C94A3280E946D126C
:106D500081110C94A328D2CF0E94681281110C9447
:106D600027290E946D1281110C9427298DE29AE146
:106D70000E94D86F80E00E948E610E947112162FCF
:106D8000072FF82EE92E84E393E00E944A129B011C
:106D9000AC0180E393E029AF3AAF4BAF5CAF0E9408
:106DA0004A12EF92FF920F931F9350EFA52E53E2DA
:106DB000B52E54E7C52E59E4D52E8601750129ADAF
:106DC0003AAD4BAD5CAD0E94655F20E041E060E014
:106DD00081E00E942F626DA77EA78FA798AB20E06D
:106DE00041E060E081E00E942F6269A77AA78BA74B
:106DF0009CA79B01AC016DA57EA58FA598A90E94BB
:106E000052AD6B017C010F900F900F900F902DEC05
:106E10003CEC4CEC5DE30E94EBAF181654F02DEC0B
:106E20003CEC4CEC5DEBC701B6010E94B7AD87FFAF
:106E30001AC049895A896B897C8985E29AE00E9447
:106E4000367489899A89AB89BC898897A105B1056F
:106E500014F00C944B2982E30E940D18B301A20197
:106E600087E09AE01BC18DE793E00E94CCB59E8B32
:106E70008D8BD1018D919C91119792FF0BC05E96E5
:106E80008D919D910D90BC91A02D0297A105B1050A
:106E900009F453C40E947112162F072FF82EE92E01
:106EA0008CE393E00E944A129B01AC0188E393E0DB
:106EB00029AF3AAF4BAF5CAF0E944A12EF92FF92FC
:106EC0000F931F9300EFA02E03E2B02E04E7C02E15
:106ED00009E4D02E8601750129AD3AAD4BAD5CAD0C
:106EE0000E94655F20E041E060E081E00E942F6247
:106EF00069A37AA38BA39CA320E041E060E081E03A
:106F00000E942F6269AB7AAB8BAB9CAB9B01AC014F
:106F100069A17AA18BA19CA10E9452AD6B017C0159
:106F20000F900F900F900F902DEC3CEC4CEC5DE32C
:106F30000E94EBAF181654F02DEC3CEC4CEC5DEBE2
:106F4000C701B6010E94B7AD87FF21C049895A89A0
:106F50006B897C8982EB99E00E94367429893A8991
:106F60004B895C89283231054105510544F482E39F
:106F70000E940D18B301A20184E999E08FC081E855
:106F800099E00E94277389E699E00C9451298FE7D4
:106F900093E00E94CCB59E8F8D8FD1018D919C91F5
:106FA000119792FF0BC05E968D919D910D90BC91B3
:106FB000A02D0297A105B10509F4CCC30E9471125E
:106FC000162F072FF82EE92E84E493E00E944A1230
:106FD0009B01AC0180E493E029AF3AAF4BAF5CAFCB
:106FE0000E944A12EF92FF920F931F9310EFA12E6F
:106FF00013E2B12E14E7C12E19E4D12E86017501DA
:1070000029AD3AAD4BAD5CAD0E94655F20E041E03B
:1070100060E081E00E942F626B017C0120E041E092
:1070200060E081E00E942F626DAB7EAB8FAB98AFCA
:107030009B01AC01C701B6010E9452AD4B015C013E
:107040000F900F900F900F902DEC3CEC4CEC5DE30B
:107050000E94EBAF181654F02DEC3CEC4CEC5DEBC1
:10706000C501B4010E94B7AD87FF42C049895A8962
:107070006B897C898FE399E00E94367429893A896B
:107080004B895C8928323105410551054CF582E375
:107090000E940D18B301A20181E299E00E943674AA
:1070A000642D82E30E94EA17642D8AE30E94EA17A6
:1070B00082E30E940D18F2E04F0E511C611C711CFE
:1070C00029893A894B895C892E5F3F4F4F4F5F4F2B
:1070D000298B3A8B4B8B5C8B31E03DA30C941629AA
:1070E0008EE099E00E94277386EF98E00C94512976
:1070F00029A53AA54BA55CA56DA57EA58FA598A948
:107100000E9453AD20E030E040E05FE30E945FB0BA
:1071100020E030E040EA52E40E945FB020E030E03E
:1071200048EC54E40E9452AD0E9457AE4B015C0102
:107130008D899E89AA2797FDA095BA2F8D8B9E8B4E
:10714000AF8BB88F29A93AA94BA95CA969A17AA1EB
:107150008BA19CA10E9453AD20E030E040E05FE3B2
:107160000E945FB020E030E040EA52E40E945FB04D
:1071700020E030E048EC54E40E9452AD0E9457AE4B
:107180002B013C012D8D3E8D442737FD4095542F1A
:107190002D8F3E8F4F8F58A32DA93EA94FA958ADD3
:1071A000C701B6010E9453AD20E030E040E05FE34C
:1071B0000E945FB020E030E040EA52E40E945FB0FD
:1071C00020E030E048EC54E40E9452AD0E9457AEFB
:1071D0006B017C0181E893E00E94CCB59C014427BF
:1071E00037FD4095542F29A33AA34BA35CA380E01D
:1071F0000E94B75A0E94B34E89E49AE10E943E73FE
:1072000040918304509184046091850470918604B8
:1072100022E084EB99E10E941075898D9A8DAB8DE7
:10722000BC8D80937B0490937C04A0937D04B093E9
:107230007E0484149504A604B70414F58C149D04EC
:10724000AE04BF040CF042C0481859086A087B0815
:107250002D8D3E8D4F8D58A1420E531E641E751EFE
:10726000C818D908EA08FB0889A19AA1ABA1BCA15A
:10727000C80ED91EEA1EFB1E812C912C540152C04F
:10728000481459046A047B040CF54C145D046E0424
:107290007F04E4F484189508A608B7082D893E8970
:1072A0004F89588D820E931EA41EB51EC418D50892
:1072B000E608F70889A19AA1ABA1BCA1C80ED91E06
:1072C000EA1EFB1E412C512C320125C0C814D904E2
:1072D000EA04FB0404F5C414D504E604F704DCF462
:1072E0008C189D08AE08BF082D893E894F89588D9E
:1072F000820E931EA41EB51E4C185D086E087F08F2
:107300008D8D9E8DAF8DB8A1480E591E6A1E7B1EB5
:10731000C12CD12C760191E9891691E09906A1043E
:10732000B10474F4A1E94A16A1E05A06610471049B
:107330003CF4B1E9CB16B1E0DB06E104F104FCF06A
:1073400049895A896B897C8985EC98E00E9436745A
:107350008BEA98E00E94D86FB501A40187EA98E013
:107360000E943674B301A20183EA98E00E94367449
:10737000B701A6018FE998E00E943674BFCCC40122
:107380000E94B912C2010E94D912C6010E94F912CC
:1073900080E00E9499780C945B292DEC3CEC4CEC3D
:1073A0005DEBC301B2010E94B7AD87FF09C00C9429
:1073B000D12985E398E00E9427738DE198E0D0C041
:1073C0009FEF291A390AA5019401C701B6010E944D
:1073D00053AD20E030E040E05FE30E945FB02B015E
:1073E0003C01409183045091840460918504709124
:1073F000860422E08FE098E00E94107520917105CC
:10740000309172054091730550917405C301B2012A
:107410000E9452AD9B01AC01609183047091840481
:1074200080918504909186040E9453AD60938304FB
:107430007093840480938504909386040E94B34ED5
:107440004091830450918404609185047091860476
:1074500022E081E098E00E9410750E947112162FC0
:10746000072FF82EE92E84E493E00E944A129B0134
:10747000AC0180E493E029AF3AAF4BAF5CAF0E9420
:107480004A12EF92FF920F931F93A0EFAA2EA3E24E
:10749000BA2EA4E7CA2EA9E4DA2E8601750129AD19
:1074A0003AAD4BAD5CAD0E94655F20E041E060E02D
:1074B00081E00E942F626B017C0120E041E060E0EE
:1074C00081E00E942F626D8B7E8B8F8B988F9B014A
:1074D000AC01C701B6010E9452AD4B015C010F9097
:1074E0000F900F900F902DEC3CEC4CEC5DE30E9464
:1074F000EBAF181654F02DEC3CEC4CEC5DEBC501F9
:10750000B4010E94B7AD87FF33C04D855E856F859E
:10751000788982ED97E00E9436742D853E854F85EF
:1075200058892832310541055105A4F482E30E94AF
:107530000D188D859E85AF85B8890296A11DB11D58
:107540008D879E87AF87B88BAC01BD0184EB97E038
:107550000C94F62981EA97E00E94277389E897E066
:107560000E94D86F84EC99E10E9448730C94082A19
:107570002D893E894F89588DC701B6010E9453ADB0
:1075800020E030E040E05FE30E945FB09B01AC018F
:10759000C301B2010E9452AD20E030E040EA52E463
:1075A0000E945FB06B017C0120E030E0A9010E94E5
:1075B000B7AD87FF27C0C701B60190582091EF04EF
:1075C0003091F0044091F1045091F2040E94BEAD5C
:1075D0009B01AC010E9453AD6B017C0122E0AB0129
:1075E000BC0188E59AE10E941075A701960160919F
:1075F000EF047091F0048091F1049091F2040E94E4
:1076000052AD18C08090EF049090F004A090F10467
:10761000B090F204A5019401C701B6010E94BEAD6D
:107620009B01AC010E9453AD9B01AC01C501B401AB
:107630000E9453AD6093EF047093F0048093F104C3
:107640009093F204C090EF04D090F004E090F10425
:10765000F090F20420E030E042E852E4C701B601C5
:107660000E94BEAD4B015C012DEC3CEC4CE85FE3AD
:107670000E94EBAF181654F026E636E646E65FE3C6
:10768000C501B4010E94B7AD87FF13C022E0B70166
:10769000A6018EE697E00E94107580E090E0A2E8D7
:1076A000B2E48093EF049093F004A093F104B093BC
:1076B000F20422E049895A896B897C8986E597E042
:1076C0000E9410754091EF045091F0046091F10414
:1076D0007091F20422E08EE397E00E94107594E02E
:1076E0002916310414F00C94082A29893A894B8907
:1076F0005C896091EF047091F0048091F1049091A5
:10770000F2040E9452AD6B017C012DEC3CEC4CEC80
:107710005DE30E94EBAF181614F40C9474292DEC61
:107720003CEC4CEC5DEBC701B6010E94B7AD87FFA6
:1077300002C00C9474290C94082A41E061E081E0B5
:107740000E94A8618DE29AE10E94D86F80E00E94B9
:107750008E61A0CB41E061E081E00E94A8618DE2F2
:107760009AE10E94D86F80E00E948E6127CC80E071
:1077700090E4A7EEB4E48093A4029093A502A093B2
:10778000A602B093A7020E94B34ED1018D919C91A5
:107790009C01287133272831310509F4BEC020E04F
:1077A00041E060E081E00E942F62209171053091FC
:1077B000720540917305509174050E9452AD4B01C2
:1077C0005C0120E041E061E080E00E942F622091B6
:1077D00071053091720540917305509174050E94B6
:1077E00052AD2B013C019B01AC01C501B4010E94CB
:1077F00052AD6B017C012DEC3CEC4CEC5DE30E9446
:10780000EBAF181654F02DEC3CEC4CEC5DEBC701E3
:10781000B6010E94B7AD87FF22C022E0B701A601E2
:107820008DEF96E00E94107582E30E940D184BE1E7
:1078300050E060E070E08FED96E00E9436746BE1FE
:1078400082E30E94EA176BE18AE30E94EA1782E36F
:107850000E940D188BED96E00E94D86F13C0A30113
:107860009201C501B4010E9453AD20E030E040E038
:107870005FE30E945FB0AB01BC0122E08CEC96E0BC
:107880000E94107580E090E0A8ECB3E48093A4021D
:107890009093A502A093A602B093A7020E94B34EB4
:1078A0002DCA20E030E04FE253E42093830430936C
:1078B0008404409385045093860480E00E94997864
:1078C0000E94E67A0C946D2A209171053091720520
:1078D0004091730550917405C701B6010E9452ADE5
:1078E0009B01AC01609183047091840480918504B4
:1078F000909186040E9453AD609383047093840436
:1079000080938504909386040E94B34E0C94EB2AD6
:1079100080E00E9499780C940C2B90FF27C0D10135
:107920001E962D913D914D915C9151971A966D91B6
:107930007D918D919C911D975D96EC915D97EF9354
:107940005C96EC915C97EF935B96EC915B97EF9371
:107950005A96EC91EF93E0EFAE2EE3E2BE2EE4E711
:10796000CE2EE9E4DE2E860175011BC00E94711245
:10797000F101268537854089518942845384648486
:1079800075849F938F937F936F9360EFA62E63E22E
:10799000B62E64E7C62E69E4D62E86017501C301B2
:1079A000B2010E94655F0F900F900F900F90F7CE7D
:1079B00080E090E00E94B91280E090E00E94D9122D
:1079C00080E090E00E94F91280E00E9499780E9485
:1079D000E67A0C94B42F80E00E94B75A0E94B34E0E
:1079E00089E49AE10E943E7340918304509184049B
:1079F000609185047091860422E084EB99E10E94F5
:107A000010750C9483314C145D046E047F041CF5D6
:107A1000481459046A047B04F4F4C418D508E60831
:107A2000F70889899A89AB89BC89C80ED91EEA1ED4
:107A3000FB1E84189508A608B708800E911EA21E8A
:107A4000B31EC6010E94B912C4010E94F912412C52
:107A5000512C32012BC08C149D04AE04BF0434F5AC
:107A600084149504A604B7040CF5C818D908EA08CC
:107A7000FB0829893A894B895C89C20ED31EE41E12
:107A8000F51E481859086A087B088D899E89AF89B8
:107A9000B88D480E591E6A1E7B1EC6010E94B9127F
:107AA000C2010E94D912812C912C540191E9C9166E
:107AB00091E0D906E104F10414F40C9442324D85AE
:107AC0005E856F8578898EE295E00E943674B701F5
:107AD000A6018AE295E00E943674B301A20186E213
:107AE00095E00E943674B501A40182E295E00E94FF
:107AF00036740C94A22F83E994E00E9448730C948E
:107B00001835C6A4D7A4E0A8F1A820E030E0A90168
:107B1000C701B6010E94B7AD882361F120E030E0D3
:107B2000A901C701B6010E94EBAF18165CF420E072
:107B300030E040E251E4C701B6010E94B7AD18162B
:107B4000B4F00AC020E030E040E251ECC701B601D9
:107B50000E94EBAF87FD0BC085E793E00E944A12BD
:107B60009B01AC01C701B6010E9453AD4DC08AE62E
:107B700094E0C3CF20E030E0A901609169057091E5
:107B80006A0580916B0590916C050E94B7AD8111DB
:107B900061C020E030E0A90160916D0570916E0533
:107BA00080916F05909170050E94B7AD811152C010
:107BB0008091400587FF2CC0C090FB04D090FC044E
:107BC000E090FD04F090FE0460918D0570918E05AB
:107BD00080918F05909190050E9488AE9B01AC0129
:107BE0000E945FB09B01AC01C701B6010E9452AD7B
:107BF0000E94CCB02091C1053091C2054091C305CF
:107C00005091C4050E945FB00E9474120C94183504
:107C1000C090FB04D090FC04E090FD04F090FE04C2
:107C200060918D0570918E0580918F0590919005E2
:107C30009B01AC010E9426B1C61AD70AE80AF90ACC
:107C4000C701B6010E94B682BC0180E090E00E94AC
:107C500088AED0CF87E394E050CFC4010E94B91220
:107C6000C6010E94D912C2010E94F91236C8CF93F0
:107C7000DF93EC0140919B028881998144FF09C008
:107C800082FD2AC081FF05C02E813F812F3631053C
:107C900019F582FF05C0CE01DF91CF910C94D52656
:107CA00081FF05C0CE01DF91CF910C94E01891FFC8
:107CB00008C00E943213CC5ADF4F8881DF91CF91E8
:107CC000BAC242FF13C089E19EE10E940F73CE0148
:107CD000DF91CF910C941C710E9472AB6093F218EB
:107CE0007093F3188093F4189093F518DF91CF9167
:107CF000089580913E0580FD0BC00E94F9710E949D
:107D0000A16CEC01009721F0B2DFCE010E94E4717A
:107D10000E94A953EECF0E942D660C942818E9CF3B
:107D2000CF93DF93FC01E05CFF4F208121FD1FC05A
:107D3000DB014D915D916D917C91DC01AF5BBF4F9B
:107D40004D935D936D937C931397EC01CB5BDF4F69
:107D5000DC0117964D915D916D917C911A97488346
:107D600059836A837B83822F897F82608083DF913E
:107D7000CF9108959F92AF92BF92CF92DF92EF92F0
:107D8000FF920F931F93CF93DF93EC015B018C0164
:107D9000005C1F4FF801908092FC32C0CB84DC84E1
:107DA000ED84FE84A70196016F81788589859A8587
:107DB0000E9452AD9F7720E030E040E85FE30E94F0
:107DC00053AD20E030E040EA51E40E94EBAF1816DA
:107DD000BCF0F50180819181A281B381FE01EF5B4E
:107DE000FF4F80839183A283B383CB5BDF4FC88235
:107DF000D982EA82FB82892D897F8460F8018083A1
:107E0000DF91CF911F910F91FF90EF90DF90CF9076
:107E1000BF90AF909F9008958091400584608093BB
:107E20004005089508952F923F924F925F926F926E
:107E30007F928F929F92AF92BF92CF92DF92EF92FA
:107E4000FF920F931F93CF93DF93CDB7DEB7649765
:107E50000FB6F894DEBF0FBECDBF382E292E7A871D
:107E600069875A834983098B1A8B2B8B3C8B4AA4D5
:107E70005BA46CA47DA423E333E948E853E4C50183
:107E8000B4010E9453AD6D837E838F83988720E079
:107E900030E0A901C301B2010E94B7AD882359F1B6
:107EA0002EA53FA548A959A9C301B2010E9453AD0F
:107EB0004B015C0120E030E040EA50E4C301B20134
:107EC0000E945FB0A50194010E94BEAD6D877E87C0
:107ED0008F87988BA30192016EA57FA588A999A988
:107EE0000E945FB0A50194010E94BEAD6EA77FA75E
:107EF00088AB99AB08C080E090E0A0EAB0E48D8741
:107F00009E87AF87B88B2D813E814F8158856989C7
:107F10007A898B899C8990580E94BEAD0E942BAEB5
:107F20009B01AC01C701B6010E945FB06D837E83E7
:107F30008F83988769817A81A985BA856A1B7B0BB3
:107F4000882777FD8095982F0E948AAE20E030E048
:107F500040E05DE30E945FB069877A878B879C87EA
:107F6000032D122D212C312C89819A81AA2797FD6E
:107F7000A095BA2F89839A83AB83BC83A895698126
:107F80007A818B819C810E948AAE6B017C01B10158
:107F9000882777FD8095982F0E948AAE29853A859B
:107FA0004B855C850E945FB09B01AC01C701B601A7
:107FB0000E9452AD6B017C0123E333E548E853E4B2
:107FC0000E9453AD9B01AC0169897A898B899C8998
:107FD0000E94BEAD0E942BAE2D813E814F815885FF
:107FE0000E945FB04B015C0120E030EC4FE755E4AC
:107FF0000E945FB02D853E854F8558890E945FB0F5
:108000002B013C01A50194016EA57FA588A999A922
:108010000E9453AD20E030E040EA50E40E945FB09F
:108020009B01AC01C301B2010E94BEAD0E9457AEDC
:108030006D3F9FE0790714F06CEF7FE0D8016D93FE
:108040007C9320E030E040E051E4C701B6010E949B
:108050005FB00E9457AEF80173836283FFEF2F1A5F
:108060003F0A0C5F1F4F81E22816310409F086CFCA
:1080700064960FB6F894DEBF0FBECDBFDF91CF91EF
:108080001F910F91FF90EF90DF90CF90BF90AF9036
:108090009F908F907F906F905F904F903F902F9028
:1080A00008957F928F929F92AF92BF92CF92DF926C
:1080B000EF92FF920F931F93CF93DF938CE092E0A8
:1080C00090931D0380931C0385E4782E7F92D2E960
:1080D000DF93C0EECF931F921F921F921F921F92A9
:1080E000812C912C98ECA92E91E4B92EC12C20E57D
:1080F000D22E23ECE22E27E4F22E00E010E12BE852
:1081000035E44CE251E06EEC7FEF83EA93E08BDEE6
:108110007F92DF93CF931F921F921F921F921F9205
:1081200000E018E728E835E44CE251E06CEE7FEF20
:108130008FE193E078DE80910A01806480930A01E8
:108140003B9A809119022DB73EB7205F3F4F0FB683
:10815000F8943EBF0FBE2DBF87FD0CC061E00E94AA
:1081600085AC80911A02811105C061E080911902ED
:108170000E94BEAC0E9472AB6093460270934702AD
:1081800080934802909349029D9AA598DF91CF91E0
:108190001F910F91FF90EF90DF90CF90BF90AF9025
:1081A0009F908F907F900C94AA83CF92DF92EF9252
:1081B000FF92CF93DF93EC018B898130A9F5CE8CB0
:1081C000DF8CE8A0F9A020E030E0A901C701B601EA
:1081D0000E94B7AD882341F1688D70E080E090E0A7
:1081E0000E9488AE20E030E040E251E40E945FB09F
:1081F000A70196010E94BEAD6FA378A789A79AA791
:10820000698D70E080E090E00E9488AE20E030E070
:1082100040E251E40E945FB0A70196010E94BEAD0A
:108220006BA77CA78DA79EA7DF91CF91FF90EF90C2
:10823000DF90CF9008954F925F926F927F92AF92AE
:10824000BF92CF92DF92EF92FF920F931F93CF9343
:10825000DF93CDB7DEB72C970FB6F894DEBF0FBE15
:10826000CDBF8091810590918205A0918305B09149
:108270008405E0911C03F0911D03838F948FA58FDB
:10828000B68F2CE032E030931D0320931C038093C3
:10829000590590935A05A0935B05B0935C054090F7
:1082A00015025090160260901702709018024092CA
:1082B000E4025092E5026092E6027092E702A301A6
:1082C000920160E070E080E89FE30E94BEAD6093A1
:1082D000C5057093C6058093C7059093C805C090E7
:1082E0001B02D0901C02E0901D02F0901E02C09272
:1082F000D402D092D502E092D602F092D7026091D9
:108300001F027091200280912102909122026093BD
:10831000A8027093A9028093AA029093AB02609383
:10832000B8027093B9028093BA029093BB02A30182
:1083300092010E945FB00E945CAE6093B50570939D
:10834000B6058093B7059093B8056093A505709323
:10835000A6058093A7059093A8052091230230914C
:1083600024024091250250912602C301B2010E94CD
:108370005FB09B01AC0160E074E284E798E40E9486
:10838000BEAD0E94C5AE0E945CAE162F6093CD05B7
:10839000A3019201C701B6010E945FB09B01AC012D
:1083A00060E074E284E798E40E94BEAD0E94C5AE2E
:1083B0000E945CAE603118F46093CC0503C08FE07E
:1083C0008093CC058091CC05811710F01093CC05DB
:1083D0006091CC0570E080E090E00E9488AEA3013F
:1083E00092010E945FB09B01AC0160E074E284E7FF
:1083F00098E40E94BEAD2B013C01A70196010E94AA
:10840000B7AD87FF08C04092D4025092D502609267
:10841000D6027092D70287E392E0C7DE2091690509
:1084200030916A0540916B0550916C052D833E8318
:108430004F83588740906D0550906E0560906F0592
:10844000709070058091710590917205A0917305EF
:10845000B091740589879A87AB87BC8720917B048C
:1084600030917C0440917D0450917E0429833A83AD
:108470004B835C83E0901C03F0901D03F701818126
:108480009281A381B4819C01AD0166277727CB013E
:10849000621B730B840B950B0E948AAE2091B90569
:1084A0003091BA054091BB055091BC050E945FB068
:1084B00060936F04709370048093710490937204BE
:1084C000F70185819681A781B0859C01AD01662762
:1084D0007727CB01621B730B840B950B0E948AAE2E
:1084E0002091BD053091BE054091BF055091C0055A
:1084F0000E945FB060936B0470936C0480936D0472
:1085000090936E0480917704909178040E9488146F
:1085100080913F0580FF24C08091BF028F9380919E
:10852000BE028F938091BD028F938091BC028F9386
:1085300030EFA32E33E2B32E34E7C32E39E4D32E2B
:10854000E984FA840B851C85A30192016D817E81EB
:108550008F8198850E94FA570F900F900F900F907F
:1085600089819A81AB81BC8180937B0490937C0448
:10857000A0937D04B0937E0480E00E94B75A2C96AD
:108580000FB6F894DEBF0FBECDBFDF91CF911F9124
:108590000F91FF90EF90DF90CF90BF90AF907F90C2
:1085A0006F905F904F900C9487850895E0911C0325
:1085B000F0911D03858587FD06C061E096859111C8
:1085C00060E00C94BEAC08958091190287FD07C04D
:1085D00061E090911A02911160E00C94BEAC089594
:1085E0002F923F924F925F926F927F928F929F92C3
:1085F000AF92BF92CF92DF92EF92FF920F931F93B1
:10860000CF93DF9300D01F92CDB7DEB79C838B83CF
:10861000DC011196EC91E53338F4E23348F5EE23B2
:1086200069F0ED3090F50DC0E43628F4E13648F4F9
:10863000EC33F1F02AC0E436D9F027C049E150E02C
:1086400026C0AB81BC8112968C91A82FB0E0AA0FF6
:10865000BB1FA95DBB4F4D915C918CEF9FE0841BCC
:10866000950BAB81BC8114969C938E93139715C088
:10867000AB81BC8112968C91A82FB0E0AA0FBB1FD2
:10868000A95DBB4F4D915C9102C04FEF5FE0AB81A4
:10869000BC8114965C934E931397AB81BC81139667
:1086A0000D911C911497E53338F5E23308F0A0C022
:1086B000EE2309F450C0ED3008F081C1E1508E2F57
:1086C00090E0FC01E154F34F4491440FFC01EE0FA4
:1086D000FF1FE553F34F85919491FC018590949091
:1086E000FC013296A590B4907CEF672E7FE0772E48
:1086F000601A710A52E03CC0E436C0F4E13608F07A
:10870000DBC0EC3309F05BC1B801882777FD8095A9
:10871000982F0E948AAE20E030E04AE754E40E949D
:108720005FB020E030E040E859E325C1E43609F0CD
:1087300046C1B801882777FD8095982F0E948AAEA0
:1087400020E030E04AEF53E40E945FB020E030E0E8
:1087500040E859E32CC180E090E0A8ECB1E4EB8163
:10876000FC8187839087A187B28729C15101480185
:10877000541708F011C1FC01E50FF11DE50FF11DC3
:1087800005911491FC0161E0650FE60FF11D5E5F3C
:10879000E60FF11D25903490601671063CF7B50187
:1087A000882777FD8095982F0E948AAE6B017C0107
:1087B000B30168197909882777FD8095982F0E9461
:1087C0008AAE2B013C01B1016A197B09882777FD2C
:1087D0008095982F0E948AAE9B01AC01C301B20123
:1087E0000E945FB02B013C01B80168197909ADC046
:1087F000EE528E2F90E0FC01E154F34F6491660F2E
:10880000FC01EE0FFF1FE553F34F85919491FC019E
:1088100025903490FC0132968590949072E0761702
:1088200008F044C0FC01E70FF11DE70FF11DA59012
:10883000B490FC0121E0270FE20FF11D7E5FE20FF3
:10884000F11D259134910A151B056CF5B40188279B
:1088500077FD8095982F29833A830E948AAE6B0119
:108860007C01B80162197309882777FD8095982FDC
:108870000E948AAE2B013C0129813A81B901681915
:108880007909882777FD8095982F0E948AAE9B01F1
:10889000AC01C301B2010E945FB02B013C01B501E4
:1088A0006219730952C049011501B9CFB90188276E
:1088B00077FD8095982F75C0E23639F0A090A3031C
:1088C000B090A403E3EAF3E006C0A0901F03B090C9
:1088D0002003EFE1F3E0828093804CEF642E4FE0C1
:1088E000742E601A710A82E0048115818E5F2680E1
:1088F0003780601671060CF049C0B401882777FDF7
:108900008095982F0E948AAE6B017C01B3016A1991
:108910007B09882777FD8095982F0E948AAE2B01CE
:108920003C01B10168197909882777FD8095982F56
:108930000E948AAE9B01AC01C301B2010E945FB0EC
:108940002B013C01B8016A197B09882777FD8095C6
:10895000982F0E948AAE9B01AC01C301B2010E9414
:10896000BEAD9B01AC01C701B6010E9453AD20E032
:1089700030E040E05EE30E945FB0AB81BC811796BF
:108980006D937D938D939C931A9719C0349682347E
:1089900019F041015801A8CFB101882777FD8095D2
:1089A000982F0E948AAE20E030E040E05EE30E9413
:1089B0005FB0EB81FC8167837087818792870F901E
:1089C0000F900F900F90DF91CF911F910F91FF901B
:1089D000EF90DF90CF90BF90AF909F908F907F905F
:1089E0006F905F904F903F902F9008958F929F923D
:1089F000AF92BF92CF92DF92EF92FF920F931F93AD
:108A0000CF93DF93EC01CB01BA016B877C878D8715
:108A10009E87FE01E05CFF4F2081297F208320E0BC
:108A200030E040E051E40E945FB00E9457AE4B013D
:108A30002981253318F5223308F08AC0222309F44E
:108A400048C02D3008F019C1215030E0F901E1543F
:108A5000F34FB490BB0CF901EE0FFF1FE553F34F3A
:108A600025913491F901E590F490F9013296459100
:108A70005491C12CD12CB2E0AB2E30C02436B0F4CE
:108A8000213608F0B4C02C3309F0F7C0882777FDF1
:108A90008095982F2CE0660F771F881F991F2A95C5
:108AA000D1F728EE33E040E050E09CC0243609F0D6
:108AB000E4C0882777FD8095982F0CE0660F771F1C
:108AC000881F991F0A95D1F724EF31E040E050E06C
:108AD00089C01E821D82D1C0A8017D01AB1498F50A
:108AE000F901EA0DF11DEA0DF11DA591B4916D0199
:108AF000F90111E01A0DE10FF11DA394A394E10F08
:108B0000F11D059114910815190534F79A01261BDA
:108B1000370BC7018A1B9B0BDC016CEFC62E6FE085
:108B2000D62ECE18DF080E94A0B19A01201B310B6F
:108B3000442737FD4095542F0E947EB1C20ED31EAC
:108B4000DE82CD829AC08CEF9FE08C199D0993C084
:108B50002E5230E0F901E154F34FA491AA0FF9012C
:108B6000EE0FFF1FE553F34F25913491F901059165
:108B70001491F901329645915491C12CD12CB2E057
:108B8000BA1768F5F901EB0FF11DEB0FF11DA59078
:108B9000B4906501F901FF24F394FB0EEF0DF11D74
:108BA000BE5FEF0DF11DE590F4908E149F04A4F4C8
:108BB0009A01261B370BD801AA19BB090E94A0B144
:108BC0009A012E193F09442737FD4095542F0E94E2
:108BD0007EB1200F311F08C0A7018501D1CFCD8202
:108BE000DE824BC00E947EB13E832D8346C022367A
:108BF00039F0E090A303F090A403A3EAB3E006C029
:108C0000E0901F03F0902003AFE1B3E012964D9186
:108C10005C91139722E014960D911C9115972E5F8D
:108C20001696ED91FC911797E815F905D4F49A0181
:108C3000261B370BD701A01BB10B0CEF1FE00E1941
:108C40001F090E94A0B19A012E1B3F0B442737FD3C
:108C50004095542F0E947EB1020F131F1E830D8377
:108C60000CC01496223419F0AF017801D4CF8CEFE8
:108C70009FE0801B910B9E838D83DF91CF911F918D
:108C80000F91FF90EF90DF90CF90BF90AF909F90AB
:108C90008F9008959F92AF92BF92CF92DF92EF9202
:108CA000FF920F931F93CF93DF936B017C01042FEF
:108CB000922EE0910A02F0910B02C1E020E030E038
:108CC00040E751E463857485858596850E94EBAF06
:108CD00018160CF0C0E011E01C2720E030E040E75F
:108CE00053E4C701B6010E94EBAF18166CF020E008
:108CF00030E0A901C701B6010E94B7AD87FF0AC0E5
:108D0000C12CD12C760106C0C12CD12C90E7E92EC4
:108D100093E4F92EC02FD0E0FE01EE0FFF1FE65FB7
:108D2000FD4FA080B180F5018181811103C0C12C6C
:108D3000D12C7601B701A601C50158DE992081F03A
:108D400020E030E040EF51E4C701B6010E94EBAFF4
:108D5000181634F4F501E05CFF4F80818160808358
:108D600020E030E040E252E4C701B6010E94EBAFE0
:108D700087FD0EC023E82C9FC0012D9F900D11246C
:108D8000845F9D4FFC01E458FF4F20813196208382
:108D9000602F70E080E090E00E9488AEAB01BC01E3
:108DA00020E08CEF9BE10E944D7520E0B701A60109
:108DB00083EF9DE10E941075E0910A02F0910B0291
:108DC00020E030E040E751E4638574858585968531
:108DD0000E94EBAF18167CF0111119C0DF91CF91F2
:108DE0001F910F91FF90EF90DF90CF90BF90AF90C9
:108DF0009F900C94677F112351F00E9472AB609397
:108E00006504709366048093670490936804DF910F
:108E1000CF911F910F91FF90EF90DF90CF90BF9077
:108E2000AF909F900895E0910A02F0910B02168294
:108E300015821386148615861686E081F0E0E851C7
:108E4000F74E10828FEF80938F0208952F923F92FA
:108E50004F925F926F927F928F929F92AF92BF924A
:108E6000CF92DF92EF92FF920F931F93CF93DF93F6
:108E7000CDB7DEB7E5970FB6F894DEBF0FBECDBF16
:108E80009DAB8CAB4E8B5F8B688F798F2E8F0BAB2E
:108E90000E9472AB6A8F7B8F8C8F9D8FACA9BDA90E
:108EA00096968C9190E0959587952C01662457FCB9
:108EB0006094762C89EE9BE10E943E73B4DFBE8DF8
:108EC000B0938F02ACA9BDA9EC91F0E0E851F74E48
:108ED00096968C918083BE8DB11104C080918802DA
:108EE00080938902530142012A8D3B8D4C8D5D8D0B
:108EF0002BA33CA34DA35EA32F8F38A349A35AA352
:108F000019821F8630EA388B41E4498B1A8A1B8A02
:108F100050EA5C8B81E48D8B1BA61CA61DA61EA6A9
:108F20001FA218A619A61AA6C12CD12C76011FA61D
:108F300018AA19AA1AAA91E099871E861D86A895D3
:108F40008CA99DA94DDBACA9BDA917963C9017979C
:108F500018960C91189719961C9119971A962C909F
:108F60000E9472AB6D837E838F839887232D302F71
:108F7000412F522D6A897B898C899D890E94B7ADCA
:108F800087FF04C03A8A0B8B1C8B2D8A232D302F30
:108F9000412F522D69817F85888999890E94B7ADBB
:108FA00087FD04C039820F87188B298AB985BB23B6
:108FB00009F449C02E893F89488D598D632D702F42
:108FC000812F922D0E94EBAF18160CF086C08D8178
:108FD0009E81AF81B8852BA13CA14DA15EA1821BD2
:108FE000930BA40BB50B3E8D311105C044EC59E039
:108FF00060E070E004C04CED55E060E070E04817C0
:1090000059076A077B0708F068C0ECA9FDA9208111
:10901000E22FF0E0E851F74E242D281920838FA786
:1090200098ABA9ABBAABFE89FA8B2F892B8B388D05
:109030003C8B498D4D8B8D819E81AF81B8858F8F03
:1090400098A3A9A3BAA32E893F89488D598D632D72
:10905000702F812F922D0E94B7AD87FF07C28D819F
:109060009E81AF81B8852F8D38A149A15AA1821B5D
:10907000930BA40BB50B3E8D3111E5C048E853E1CD
:1090800060E070E0481759076A077B0708F0EEC1F7
:109090004D855E85452B09F0DBC0ACA9BDA9EC91DF
:1090A000F0E0E851F74E882D840D8083ED85FE8534
:1090B0003196FE87ED87FE89F9832F892F87388DBA
:1090C000388B498D498B8D819E81AF81B8858BA36B
:1090D0009CA3ADA3BEA391E0998720E030E040E2DD
:1090E00052E46E897F89888D998D0E9453AD9B01D2
:1090F000AC01632D702F812F922D0E94EBAF1816BB
:109100001CF48AE79BE13BC08D819E81AF81B885CD
:109110002A8D3B8D4C8D5D8D821B930BA40BB50B63
:10912000893E9340A105B10558F080E00E94B31834
:109130008D819E81AF81B8858A8F9B8FAC8FBD8FCB
:109140008D819E81AF81B885880F991FAA1FBB1F93
:109150002BA13CA14DA15EA1821B930BA40BB50BCF
:109160002F8D38A149A15AA1821B930BA40BB50BDB
:1091700081389F44A241B105E8F08DE59BE10E9452
:109180004873E5960FB6F894DEBF0FBECDBFDF91F2
:10919000CF911F910F91FF90EF90DF90CF90BF90F4
:1091A000AF909F908F907F906F905F904F903F9087
:1091B0002F9039CE4D855E85463051050CF4BFCEDB
:1091C00082E09BE10E943E732EDE5BA9552309F4E9
:1091D0004FC1ACA9BDA95A96CD92DD92ED92FC92F9
:1091E0005D972FA138A549A55AA55E962D933D936D
:1091F0004D935C9391972BA53CA54DA55EA59296AA
:109200002D933D934D935C93959781E053968C936A
:1092100080E0E5960FB6F894DEBF0FBECDBFDF91BC
:10922000CF911F910F91FF90EF90DF90CF90BF9063
:10923000AF909F908F907F906F905F904F903F90F6
:109240002F900C94997848EB5BE060E070E01ACFC7
:109250002FA538A949A95AA9280F391F4A1F5B1FF2
:1092600029873A874B875C872FA538A949A95AA92E
:10927000281B390B4A0B5B0BCA01B901A5019401EC
:109280000E9426B129853A854B855C850E947EB176
:10929000240D351D461D571D24313105410551054D
:1092A000A4F0ACA9BDA996968C9190E04497AA270A
:1092B00097FDA095BA2F29013A0182179307A407B9
:1092C000B50744F42C013D0105C034E1432E512C77
:1092D000612C712CECA9FDA926A1822F869590E026
:1092E000A0E0B0E084159505A605B7056CF4822FC3
:1092F00090E001974C01AA2497FCA094BA2C841802
:109300009508A608B70802C053014201B301A201A3
:1093100081EE9BE10E941E74B501A4018CED9BE1DE
:109320000E941E7422E049815F856889798985EDF4
:109330009BE10E944D7522E04A895B896C897D8999
:109340008EEC9BE10E9410752D853E852330310502
:109350000CF4A3CEC501B4010E948AAE20E030E037
:1093600040E850E40E945FB06B017C0129813F8599
:10937000488959896A897B898C899D890E9452AD67
:1093800020ED3FE049E450E40E945FB09B01AC0156
:10939000C701B6010E94BEAD6B017C0169857A856B
:1093A0008B859C850E948AAE20E030E04AE754E439
:1093B0000E94BEAD69837A838B839C8322E0B701D0
:1093C000A60188EC9BE10E944D7522E049815A81FB
:1093D0006B817C8182EC9BE10E9410752AE939E95E
:1093E00049E15FE3C701B6010E945FB06B017C01F8
:1093F0009B01AC010E9453AD29813A814B815C8174
:109400000E94BEAD6FA378A789A79AA729813A8148
:109410004B815C81C701B6010E945FB020E030E063
:1094200040E05EE30E945FB06BA77CA78DA79EA77C
:1094300085EB9BE10E94277322E0B701A6018FEA2A
:109440009BE10E94107522E04FA158A569A57AA55D
:1094500089EA9BE10E94107522E04BA55CA56DA5F1
:109460007EA583EA9BE10E94107517CE198635CE42
:10947000E5960FB6F894DEBF0FBECDBFDF91CF915A
:109480001F910F91FF90EF90DF90CF90BF90AF9022
:109490009F908F907F906F905F904F903F902F9014
:1094A0000895CF93DF930E9472ABAB01BC018BEFA9
:1094B0009AE10E941E74E0919102F0E0EE0FFF1F0E
:1094C000E65FFD4FC081D1814F81588569857A85DE
:1094D00022E08DE89DE10E944D754B855C856D8590
:1094E0007E8520E08DE89DE10E944D75E881F0E0E9
:1094F000E851F74E608170E08DE89DE1DF91CF91FA
:109500000C94F8738091400582FF22C060E070E007
:1095100081EF9AE10E94EC73E0910A02F0910B0254
:1095200067817085818592850E9457AE605171096F
:109530006D31714018F08CED9AE102C082ED9AE134
:109540000E94277385EA9AE10E94487381E008959A
:1095500080E008952F923F924F925F926F927F9298
:109560008F929F92AF92BF92CF92DF92EF92FF9233
:109570000F931F93CF93DF9300D01F921F92CDB70D
:10958000DEB7A8950E9472AB69837A838B839C8334
:1095900000910A0210910B0220E030E040E252E418
:1095A000D80117966D917D918D919C911A970E948B
:1095B000B7AD87FF10C020E030E040E252E4F80190
:1095C00063857485858596850E94B7AD87FF03C046
:1095D0001092890204C08091880280938902809150
:1095E0008F02811109C080911E03882309F46FC284
:1095F000815080931E036BC2C8010E94F04280918B
:10960000400582FD1CC0D8011796CD90DD90ED90ED
:10961000FC901A9720E030E040E851E4C701B60121
:109620000E94B7AD87FD66C220E030E046E953E412
:10963000C701B6010E94EBAF18160CF45BC2812C77
:109640008091400582FD40C2FF24F394F8012385F8
:1096500034854585568567817085818592850E9410
:10966000EBAF87FDF12C992493949F2441F478016A
:10967000F0E4EF0EF11CD7018C9180FD48C2C98047
:10968000DA80EB80FC80F801E75BFF4F408051807F
:10969000628073805801B1E4AB0EB11CF50180818A
:1096A0009181A281B381A7019601281B390B4A0B36
:1096B0005B0B421653066406750698F5180130E4F4
:1096C000230E311CD101BC91BD838B2F867049F1D3
:1096D00080913F0586FF25C0FD81F1FF56C27801CC
:1096E000E5E4EE0EF11CD7012D913D914D915C9179
:1096F000F80167817085818592850E9452AD20E0D6
:1097000030E040E85FE30E94B7AD87FD09C28D817C
:10971000897FD1018C93BE016F5F7F4FC8010E948A
:10972000903ED8019F968C919F971796CD90DD9093
:10973000ED90FC901A97F801B4E08B9FE00DF11DBD
:109740001124C0AAD1AAE2AAF3AA8F5F8370F801FC
:1097500087A78389813009F0BCC043845484658421
:10976000768420E030E040EA51E4C301B2010E9477
:10977000B7AD87FDC0C0A7019601C301B2010E9429
:1097800052AD6B017C0120E030E040EA51E40E94E0
:10979000EBAF18160CF4C6C020E030E040EA51EC04
:1097A000C701B6010E94B7AD87FDD0C0BE016F5F93
:1097B0007F4FC8010E94BA3EF801228D338D448D3F
:1097C000558DC701B6010E945FB02B013C01D80145
:1097D00054962D913D914D915C915797C701B601DB
:1097E0000E9453AD6B017C01F80123A434A4A5A40D
:1097F000B6A49101A5010E94B7AD87FD16C0D8019E
:1098000097962C90979798963C9098979996AC90AD
:1098100099979A96BC909101A501B601C7010E9443
:10982000EBAF181614F016015701C101D501F8016C
:10983000848B958BA68BB78B268D378D40A151A13C
:10984000B101C5010E945FB02DEC3CEC4CEC5DE336
:109850000E945FB09B01AC01C301B2010E9453ADF5
:109860006B017C01D8019F968C91F801B4E08B9F2D
:10987000E00DF11D1124D80117962D913D914D91C8
:109880005C911A9760A971A982A993A90E9452AD0F
:10989000F80122A133A144A155A10E945FB02FED90
:1098A0003FE445E550E40E945FB09B01AC01C70175
:1098B000B6010E9453AD0E9457AE77FD47C0D80154
:1098C00096962C9130E0261737070CF4B901F62E46
:1098D00098C0833009F09CC0F801438454846584A7
:1098E000768420E030E040EA51E4C301B2010E94F6
:1098F000B7AD87FF07C0F801E05CFF4F8081897F2B
:10990000808324C0A7019601C301B2010E9452AD19
:109910006B017C0120E030E040EA51E40E94EBAFB3
:10992000181654F4D8019696FC90BE016F5F7F4FD5
:10993000C8010E94903E65C020E030E040EA51EC52
:10994000C701B6010E94B7AD87FF02C0F12C59C014
:10995000BE016F5F7F4FC8010E94BA3EF801C78009
:10996000D084E184F28420E030E040E450E4648973
:109970007589868997890E945FB02B013C01D801C7
:109980009F968C91F801B4E08B9FE00DF11D11249E
:1099900020A931A942A953A9C701B6010E9452AD1D
:1099A0002FED3FE445E550E40E945FB09B01AC0120
:1099B000C301B2010E9453AD20E030E040E85EE315
:1099C0000E945FB0F801648B758B868B978B228D1C
:1099D000338D448D558D0E945FB09B01AC01C70152
:1099E000B6010E9453ADD8011B962D913D914D912A
:1099F0005C911E970E94EBAF18160CF4A7CFF801EC
:109A0000F08CD801EC91F0E0E851F74EF0823CC0C8
:109A1000823021F589819A81AB81BC81F80147852B
:109A20005089618972896C017D01C41AD50AE60AE0
:109A3000F70A29E8C21623E1D206E104F10420F175
:109A40002081E22FF0E0E851F74E292D2195208367
:109A5000F8018787908BA18BB28B07C0E081F0E083
:109A6000E851F74E892D81958083992039F0BE0108
:109A70006F5F7F4FC8010E94903E06C0F801E05C16
:109A8000FF4F8081897F808320E030E040E753E40E
:109A9000F80167817085818592850E94EBAF181669
:109AA00034F4D801EC91F0E0E851F74E1082809147
:109AB0001C0390911D038B960817190729F4992010
:109AC00011F02F9A01C02F98882009F48CCD809135
:109AD000400582FFAAC0E0910A02F0910B02E081EA
:109AE000F0E0E851F74E108280919B0288608093ED
:109AF0009B029BC080911E038F5F80931E038B305F
:109B000018F00E940C3FFEDC8824839499CD63E01A
:109B100082E30E949475F70180818E7F8083AFCDB0
:109B200080911E038F5F80931E038B3008F46AC000
:109B30000E940C3F80EE93E10E944873D7012D9163
:109B40003D914D915C91F801678170858185928589
:109B50000E9452ADAB01BC0122E08FE49CE00E9468
:109B60004D7549815A816B817C81F501808191819C
:109B7000A281B381481B590B6A0B7B0B87E49CE0E5
:109B80000E941E7483E49CE03BC0F8012385348569
:109B90004585568567817085818592850E9452AD85
:109BA0009F7720E030E040EA51E40E94EBAF1816C6
:109BB00064F580911E038F5F80931E038B3010F13C
:109BC0000E940C3F80EE93E10E944873F801EB5B2A
:109BD000FF4F408151816281738122E081E29CE0EC
:109BE0000E944D75D80117964D915D916D917C91B4
:109BF0001A9722E086E19CE00E944D758EE09CE081
:109C00000E942773882483948CCDB8EECB0EB3E0EA
:109C1000DB1EE11CF11CC418D508E608F708F501A5
:109C2000C082D182E282F3827CCD0F900F900F90A0
:109C30000F900F90DF91CF911F910F91FF90EF90B8
:109C4000DF90CF90BF90AF909F908F907F906F905C
:109C50005F904F903F902F900895882321F080913E
:109C60000B01826003C080910B018D7F80930B01FB
:109C70000895882321F080910B01816003C08091B9
:109C80000B018E7F80930B010895882321F0809132
:109C90000B01846003C080910B018B7F80930B01CB
:109CA0000895FB01DC018091C905882349F023E375
:109CB00033E34BEC51E4CD010E945FB0FB01DC01CA
:109CC000BF01CD010895CF93DF931F92CDB7DEB7CB
:109CD0009091400590FF02C0811127C020913F055F
:109CE00023FD23C0916090934005179A169A159A08
:109CF00089830E94E4421092EA188981811115C07B
:109D000020E040E060E070E0CB010E944A4640E085
:109D100060E070E0CB010E94D5429B9AA39A8091AB
:109D20003F058F7B886080933F050F90DF91CF9137
:109D30000895CF93C0914005CD7FC093400520E0AA
:109D400030E0A901609131027091320280913302BA
:109D5000909134020E94B7AD882319F0C260C0937D
:109D60004005CF9108952F923F924F925F926F924C
:109D70007F928F929F92AF92BF92CF92DF92EF929B
:109D8000FF920F931F93CF93DF93CDB7DEB76D97FD
:109D90000FB6F894DEBF0FBECDBF8BE793E00E94F5
:109DA000CCB59093C6048093C50489E793E00E94E4
:109DB000CCB59093C4048093C304C090E002D090CB
:109DC000E102E090E202F090E302C092DC02D09265
:109DD000DD02E092DE02F092DF02C092D802D09261
:109DE000D902E092DA02F092DB028091B402909103
:109DF000B502A091B602B091B7028093B0029093E1
:109E0000B102A093B202B093B3028093AC029093DC
:109E1000AD02A093AE02B093AF028091C4029091C4
:109E2000C502A091C602B091C7028093C002909370
:109E3000C102A093C202B093C3028093BC0290936C
:109E4000BD02A093BE02B093BF028091D002909158
:109E5000D102A091D202B091D3028093CC02909310
:109E6000CD02A093CE02B093CF028093C80290930C
:109E7000C902A093CA02B093CB028091A402909130
:109E8000A502A091A602B091A7028093A002909390
:109E9000A102A093A202B093A30280939C0290938C
:109EA0009D02A0939E02B0939F0220918304309163
:109EB00084044091850450918604C701B6010E9434
:109EC0005FB00E9457AE6093A3047093A404809384
:109ED000A5049093A60420918F04309190044091A2
:109EE000910450919204C701B6010E945FB00E9494
:109EF00057AE60939F047093A0048093A104909345
:109F0000A2042091870430918804409189045091E3
:109F10008A04C701B6010E945FB00E9457AE6093E9
:109F20009B0470939C0480939D0490939E042091C5
:109F30007F04309180044091810450918204C701D4
:109F4000B6010E945FB00E9457AE60939704709371
:109F500098048093990490939A04C090EF04D09051
:109F6000F004E090F104F090F20481E993E00E94A3
:109F70004A129B01AC01C701B6010E9453AD2B01EF
:109F80003C01C090EF04D090F004E090F104F09018
:109F9000F20485E993E00E944A129B01AC01C701DB
:109FA000B6010E9453AD4B015C01C090EF04D0900C
:109FB000F004E090F104F090F20489E993E00E944B
:109FC0004A129B01AC01C701B6010E9453AD6B015F
:109FD0007C0185E893E00E944A122BED3FE049E4C2
:109FE00050E40E945FB020E030E044E353E40E947C
:109FF000BEAD0E94BBAD9B01AC01C301B2010E948A
:10A000005FB02091E0023091E1024091E202509174
:10A01000E3020E945FB020E030E040E05FE30E9496
:10A0200053AD0E94C5AE0E9457AE6093E704709393
:10A03000E8048093E9049093EA0485E893E00E94A1
:10A040004A122BED3FE049E450E40E945FB020E06B
:10A0500030E044E353E40E94BEAD0E94C2B09B01D5
:10A06000AC01C301B2010E945FB02091E0023091C7
:10A07000E1024091E2025091E3020E945FB020E0D1
:10A0800030E040E05FE30E9453AD0E94C5AE0E9405
:10A0900057AE6093E3047093E4048093E5049093D7
:10A0A000E60489E893E00E944A122BED3FE049E480
:10A0B00050E40E945FB020E030E044E353E40E94AB
:10A0C000BEAD0E94BBAD9B01AC01C501B4010E94B5
:10A0D0005FB02091E0023091E1024091E2025091A4
:10A0E000E3020E945FB020E030E040E05FE30E94C6
:10A0F00053AD0E94C5AE0E9457AE6093DF047093CB
:10A10000E0048093E1049093E20489E893E00E94E4
:10A110004A122BED3FE049E450E40E945FB020E09A
:10A1200030E044E353E40E94BEAD0E94C2B09B0104
:10A13000AC01C501B4010E945FB02091E0023091F2
:10A14000E1024091E2025091E3020E945FB020E000
:10A1500030E040E05FE30E9453AD0E94C5AE0E9434
:10A1600057AE6093DB047093DC048093DD0490931E
:10A17000DE048DE893E00E944A122BED3FE049E4B3
:10A1800050E40E945FB020E030E044E353E40E94DA
:10A19000BEAD0E94BBAD9B01AC01C701B6010E94E0
:10A1A0005FB02091E0023091E1024091E2025091D3
:10A1B000E3020E945FB020E030E040E05FE30E94F5
:10A1C00053AD0E94C5AE0E9457AE6093D704709302
:10A1D000D8048093D9049093DA048DE893E00E9428
:10A1E0004A122BED3FE049E450E40E945FB020E0CA
:10A1F00030E044E353E40E94BEAD0E94C2B09B0134
:10A20000AC01C701B6010E945FB02091E00230911D
:10A21000E1024091E2025091E3020E945FB020E02F
:10A2200030E040E05FE30E9453AD0E94C5AE0E9463
:10A2300057AE6093D3047093D4048093D504909365
:10A24000D60485EA93E00E944A126B017C0181E703
:10A2500093E00E944A129B01AC01C701B6010E9423
:10A2600053AD2091E0023091E1024091E202509121
:10A27000E3020E945FB00E945CAE6093FF047093A3
:10A280000005809301059093020589EA93E00E94FE
:10A290004A126B017C0181E793E00E944A129B0104
:10A2A000AC01C701B6010E9453AD2091E00230918C
:10A2B000E1024091E2025091E3020E945FB00E94ED
:10A2C0005CAE6093FB047093FC048093FD04909358
:10A2D000FE048DEA93E00E944A126B017C0181E743
:10A2E00093E00E944A129B01AC014090E002509022
:10A2F000E1026090E2027090E302C701B6010E94A1
:10A3000053ADA30192010E945FB00E945CAE4B016D
:10A310005C01C090FF04D0900005E0900105F09032
:10A320000205109140058FEFC816D806E104F1042C
:10A33000C0F46091EF047091F0048091F104909169
:10A34000F2049B01AC010E9453ADA30192010E9453
:10A350005FB020E03EEF4FE757E40E94EBAF1816E6
:10A36000D4F5106810934005C701B6010E9488AE6D
:10A370009B01AC010E945FB06093FF0470930005E5
:10A3800080930105909302056091FB047091FC0499
:10A390008091FD049091FE040E9488AE9B01AC0167
:10A3A0000E945FB06093FB047093FC048093FD04F3
:10A3B0009093FE04C501B4010E9488AE9B01AC01DC
:10A3C0000E945FB06093F7047093F8048093F904DF
:10A3D0009093FA0433C01F7710934005A7019601AC
:10A3E000C701B6010E9426B16093FF047093000577
:10A3F00080930105909302056091FB047091FC0429
:10A400008091FD049091FE049B01AC010E9426B155
:10A410006093FB047093FC048093FD049093FE040E
:10A42000A5019401C501B4010E9426B16093F7040F
:10A430007093F8048093F9049093FA048DE993E003
:10A440000E944A129B01AC010E945FB06093F3042A
:10A450007093F4048093F5049093F604198A1A8A91
:10A460001B8A1C8A1D861E861F86188A8091A3045B
:10A470009091A404A091A504B091A6048D8B9E8B0D
:10A48000AF8BB88FBE016F5F7F4FCE010D960E94DC
:10A49000949489819A81AB81BC81809303059093C8
:10A4A0000405A0930505B09306058091A30490913F
:10A4B000A404A091A504B091A6048093A70490934E
:10A4C000A804A093A904B093AA048093AB0490932A
:10A4D000AC04A093AD04B093AE0410929704109214
:10A4E00098041092990410929A0410929B0410926E
:10A4F0009C0410929D0410929E0410929F0410924E
:10A50000A0041092A1041092A2044090E002509086
:10A51000E1026090E2027090E30220E030E040E768
:10A5200051E4C301B2010E945FB00E9457AE609334
:10A53000EB047093EC048093ED049093EE0488EDAB
:10A54000882E82E0982E99EBA92E95E0B92E0CEA80
:10A5500012E029EA222E25E0322EECE9F2E0FD8F0E
:10A56000EC8F89E995E09B8F8A8F198EF401C19059
:10A57000D190E190F1904F01A701960160E070E069
:10A5800080E89FE30E94BEADF501619371938193D2
:10A5900091935F01F80161917191819191918F0186
:10A5A000A70196010E945FB00E945CAEF101619329
:10A5B0007193819391931F01EC8DFD8D6191719148
:10A5C00081919191FD8FEC8FA70196010E945FB060
:10A5D0000E945CAEEA8DFB8D6193719381939193A0
:10A5E000FB8FEA8FF98DFF5FF98FF43009F0BECF52
:10A5F000A0909C02B0909D02C0909E02D0909F02BD
:10A60000E090AC02F090AD020091AE021091AF026A
:10A610009501A601B701C8010E94B7AD87FF02C02E
:10A62000750186012091D8023091D9024091DA0259
:10A630005091DB02B701C8010E945FB09B01AC01E1
:10A6400060E070E080E090E40E94BEAD0E94CCB07B
:10A650009B01AC01B701C8010E945FB06093B304D5
:10A660007093B4048093B5049093B604A090A402B0
:10A67000B090A502C090A602D090A702E090B402CC
:10A68000F090B5020091B6021091B7029501A601B3
:10A69000B701C8010E94B7AD87FF02C075018601EE
:10A6A0009701A801C301B2010E945FB09B01AC01F8
:10A6B00060E070E080E090E40E94BEAD0E94CCB00B
:10A6C0009B01AC01B701C8010E945FB06093AF0469
:10A6D0007093B0048093B1049093B2042ADB6D961A
:10A6E0000FB6F894DEBF0FBECDBFDF91CF911F91A3
:10A6F0000F91FF90EF90DF90CF90BF90AF909F9021
:10A700008F907F906F905F904F903F902F90089523
:10A71000EF92FF920F931F93609341057093420550
:10A720008093430590934405209345053093460557
:10A730004093470550934805E0924905F0924A0539
:10A7400000934B0510934C051F910F91FF90EF90D4
:10A750000895CF92DF92EF92FF9281E00E94191349
:10A760000E9472AB20919207211144C020913D05B7
:10A7700022FD40C0C090F218D090F318E090F41879
:10A78000F090F5189B01AC012C193D094E095F09A9
:10A7900069017A018091F3029091F402A091F5028F
:10A7A000B091F6020097A105B10541F08C159D0509
:10A7B000AE05BF0518F480E086DA05C080913F053C
:10A7C000877F80933F058091EF029091F002A091E6
:10A7D000F102B091F2020097A105B10599F08C1534
:10A7E0009D05AE05BF0570F481E0FF90EF90DF900E
:10A7F000CF9069CA6093F2187093F3188093F4189D
:10A800009093F518FF90EF90DF90CF900895AF925E
:10A81000BF92CF92DF92EF92FF920F931F93CF934D
:10A82000DF93EB01D82EC92E109275051092760594
:10A8300010927705109278051092790510927A059A
:10A8400010927B0510927C0510927D0510927E057A
:10A8500010927F051092800569E875E085E795E024
:10A860000E9494946091A3047091A4048091A50423
:10A870009091A6040E948AAE20E030E040EC5FE3B5
:10A880000E945FB00E9457AE7B018C0121E02F93A4
:10A890002F93CF92DF92DF93CF93A12CB12C650140
:10A8A00020E030E0A90160E070E0CB010E94AE9FA3
:10A8B00010926F041092700410927104109272043E
:10A8C00010926B0410926C0410926D0410926E043E
:10A8D0000F900F900F900F900F900F90DF91CF91EE
:10A8E0001F910F91FF90EF90DF90CF90BF90AF90AE
:10A8F00008954F925F926F927F928F929F92AF9244
:10A90000BF92CF92DF92EF92FF920F931F93CF935C
:10A91000DF9300D01F92CDB7DEB76091C402709173
:10A92000C5028091C6029091C70271DF6091E0027A
:10A930007091E1028091E2029091E3029B01AC01EF
:10A940000E9453AD20E030E040EA50EC0E945FB03E
:10A950000E9457AE2B013C011F92992493949F9221
:10A9600020E030E040E05FE36091C4027091C502F6
:10A970008091C6029091C7020E945FB09F938F930F
:10A980007F936F93A12CB12C65018301720120E0AC
:10A9900030E0A90160E070E0CB010E94AE9F20E0B2
:10A9A00030E040E05FE36091C4027091C5028091A5
:10A9B000C6029091C7020E945FB029DF20E030E01C
:10A9C00040EA50EC6091E0027091E1028091E20275
:10A9D0009091E3020E945FB00E9457AE1F929F9237
:10A9E0002091C7022F932091C6022F932091C50278
:10A9F0002F932091C4022F937B018C0120E030E043
:10AA0000A90160E070E0CB010E94AE9F8DE793E06A
:10AA10000E94CCB580909F049090A004A090A104C7
:10AA2000B090A204B094A09490948094811C911C46
:10AA3000A11CB11CAA2797FDA095BA2F881A990AC4
:10AA4000AA0ABB0A8FE793E00E94CCB5C0909B0492
:10AA5000D0909C04E0909D04F0909E04F094E094CB
:10AA6000D094C094C11CD11CE11CF11CAA2797FDF5
:10AA7000A095BA2FC81AD90AEA0AFB0A81E893E01E
:10AA80000E94CCB54091970450919804609199042C
:10AA900070919A0470956095509541955F4F6F4FF6
:10AAA0007F4FAA2797FDA095BA2F481B590B6A0B19
:10AAB0007B0B0FB6F894DEBF0FBECDBF2A013B0162
:10AAC0008C149D04AE04BF0444F484169506A606B7
:10AAD000B70654F42401350107C0C416D506E606AE
:10AAE000F70614F42601370184189508A608B7085C
:10AAF000C418D508E608F708DB01CA0184199509CE
:10AB0000A609B70989839A83AB83BC831092750524
:10AB100010927605109277051092780510927905BB
:10AB200010927A0510927B0510927C058091A30407
:10AB30009091A404A091A504B091A60480937D05F2
:10AB400090937E05A0937F05B093800569E875E03A
:10AB500085E795E00E9494948091890590918A05FB
:10AB6000A0918B05B0918C0588199909AA09BB0998
:10AB70008093890590938A05A0938B05B0938C05EB
:10AB800080918D0590918E05A0918F05B0919005D3
:10AB90008C199D09AE09BF0980938D0590938E0590
:10ABA000A0938F05B09390058091910590919205A7
:10ABB000A0919305B091940529813A814B815C81E4
:10ABC000821B930BA40BB50B809391059093920578
:10ABD000A0939305B09394051F9281E08F93809189
:10ABE000C7028F938091C6028F938091C5028F9385
:10ABF0008091C4028F93A12CB12C65018301720155
:10AC000020E030E0A90160E070E0CB010E94AE9F3F
:10AC100010927505109276051092770510927805BE
:10AC20001092790510927A0510927B0510927C059E
:10AC30008091A3049091A404A091A504B091A604CE
:10AC400080937D0590937E05A0937F05B09380054A
:10AC5000109241051092420510924305109244054E
:10AC6000109245051092460510924705109248052E
:10AC70001092490510924A0510924B0510924C050E
:10AC800069E875E085E795E00E94949480918905D4
:10AC900090918A05A0918B05B0918C058093C70493
:10ACA0009093C804A093C904B093CA0480918D0501
:10ACB00090918E05A0918F05B09190058093CB0463
:10ACC0009093CC04A093CD04B093CE0480919105D1
:10ACD00090919205A0919305B09194058093CF0433
:10ACE0009093D004A093D104B093D2046091030553
:10ACF0007091040580910505909106050E948AAE29
:10AD00006B017C0120E030E040EA50E46091E00219
:10AD10007091E1028091E2029091E3020E945FB0A3
:10AD20009B01AC01C701B6010E9453AD0E9457AE12
:10AD300060930305709304058093050590930605C1
:10AD40000F900F900F900F900F900F90E0911C03B9
:10AD5000F0911D0380810F900F900F900F90DF9165
:10AD6000CF911F910F91FF90EF90DF90CF90BF9008
:10AD7000AF909F908F907F906F905F904F900C94CA
:10AD80001B410F931F93CF93DF9380918705C1E001
:10AD900018161CF0C0E08F5F01C0815080938705BA
:10ADA000179816981598809140058E7F80934005DE
:10ADB0008FEF8093EA180091090110910901D09159
:10ADC00009018C2F0E942D4E8C2F0E94394E8C2F02
:10ADD0000E94454E81E090E00E94C6AB409A419AA5
:10ADE000429A82E090E00E94C6AB40984198429817
:10ADF00001FB882780F90E942D4E812F81700E94CF
:10AE0000394ED2FB882780F9DF91CF911F910F91A6
:10AE10000C94454E4F925F926F927F928F929F92C9
:10AE2000AF92BF92CF92DF92EF92FF920F931F9358
:10AE3000CF93DF93CDB7DEB728970FB6F894DEBF78
:10AE40000FBECDBF2B013C0129833A834B835C832A
:10AE5000ED82FE820F83188785017401209115050C
:10AE60003091160540911705509118050E945FB06A
:10AE70004B015C0120912105309122054091230571
:10AE80005091240569817A818B819C810E945FB0F9
:10AE90009B01AC01C501B4010E9453AD4B015C01A3
:10AEA00020912D0530912E0540912F0550913005B0
:10AEB0006D817E818F8198850E945FB09B01AC017E
:10AEC000C501B4010E9453ADF60160837183828392
:10AED00093832091190530911A0540911B055091DB
:10AEE0001C05C301B2010E945FB04B015C012091BF
:10AEF0002505309126054091270550912805698147
:10AF00007A818B819C810E945FB09B01AC01C5015D
:10AF1000B4010E9453AD4B015C0120913105309189
:10AF2000320540913305509134056D817E818F81CA
:10AF300098850E945FB09B01AC01C501B4010E94DD
:10AF400053ADF801608371838283938320911D0543
:10AF500030911E0540911F0550912005C301B2019B
:10AF60000E945FB04B015C012091290530912A05B8
:10AF700040912B0550912C0569817A818B819C81B0
:10AF80000E945FB09B01AC01C501B4010E9453ADAA
:10AF90004B015C0120913505309136054091370514
:10AFA000509138056D817E818F8198850E945FB0B8
:10AFB0009B01AC01C501B4010E9453ADF701608350
:10AFC00071838283938328960FB6F894DEBF0FBEF9
:10AFD000CDBFDF91CF911F910F91FF90EF90DF9048
:10AFE000CF90BF90AF909F908F907F906F905F9029
:10AFF0004F9008954F925F926F927F928F929F929F
:10B00000AF92BF92CF92DF92EF92FF920F931F9376
:10B01000CF93DF93CDB7DEB764970FB6F894DEBF5A
:10B020000FBECDBF69837A838B839C832D833E8340
:10B030004F835887E986FA860B871C8725013601DE
:10B04000E62EF72E082F192F20EF33E244E759E4BC
:10B05000B701C8010E94B7AD81110DC0809169058B
:10B0600090916A05A0916B05B0916C0589839A83D4
:10B07000AB83BC830AC0C701D80180936905909354
:10B080006A05A0936B05B0936C05CD80DE80EF80E0
:10B09000F88420EF33E244E759E4C701B6010E9487
:10B0A000B7AD81110DC080916D0590916E05A09195
:10B0B0006F05B09170058D839E83AF83B88708C0FC
:10B0C000C0926D05D0926E05E0926F05F09270050A
:10B0D000C984DA84EB84FC8420EF33E244E759E44A
:10B0E000C701B6010E94B7AD81110DC080917105F5
:10B0F00090917205A0917305B091740589879A8724
:10B10000AB87BC8708C0C0927105D0927205E092EF
:10B110007305F09274058091400585FF3DC0298537
:10B120003A854B855C852D873E874F87588B2091CC
:10B130006B0430916C0440916D0450916E046D81EC
:10B140007E818F8198850E9453AD698B7A8B8B8B22
:10B150009C8B20916F043091700440917104509148
:10B16000720469817A818B819C810E9453ADAE010A
:10B17000475F5F4F4A01DE0115965D019E012F5F1B
:10B180003F4F6901ED84FE840F85188929893A892A
:10B190004B895C893FDE24C020916F04309170049C
:10B1A000409171045091720469817A818B819C81F4
:10B1B0000E9453AD69837A838B839C8320916B04B7
:10B1C00030916C0440916D0450916E046D817E81CC
:10B1D0008F8198850E9453AD6D837E838F8398877E
:10B1E0002091D8023091D9024091DA025091DB02CD
:10B1F00069817A818B819C810E945FB020E030E080
:10B2000040E05FE30E9453AD0E94C5AE0E9457AE7E
:10B2100060934D0570934E0580934F0590935005B4
:10B220002091DC023091DD024091DE025091DF027C
:10B230006D817E818F8198850E945FB020E030E033
:10B2400040E05FE30E9453AD0E94C5AE0E9457AE3E
:10B250006093510570935205809353059093540564
:10B260002091E0023091E1024091E2025091E3022C
:10B2700069857A858B859C850E945FB020E030E0EF
:10B2800040E05FE30E9453AD0E94C5AE0E9457AEFE
:10B290006093550570935605809357059093580514
:10B2A00020EF33E244E759E4C301B2010E94B7AD95
:10B2B0008823C1F080919B0283FD14C0E0911C03A0
:10B2C000F0911D0320E030E046E153E462A973A948
:10B2D00084A995A90E94EBAF18165CF180913F05F7
:10B2E00087FD27C020EF33E244E759E468A579A53C
:10B2F0008AA59BA50E94B7AD882361F088A599A572
:10B30000AAA5BBA580937B0490937C04A0937D04A5
:10B31000B0937E0441E061E081E00E947B9A81115C
:10B3200006C08FE693E10E94347380E019C081E08B
:10B3300017C02091E4023091E5024091E60250915D
:10B34000E702C301B2010E945FB00E9457AE609352
:10B35000590570935A0580935B0590935C05C2CFA5
:10B3600064960FB6F894DEBF0FBECDBFDF91CF91CC
:10B370001F910F91FF90EF90DF90CF90BF90AF9013
:10B380009F908F907F906F905F904F9008954F9215
:10B390005F926F927F928F929F92AF92BF92CF9265
:10B3A000DF92EF92FF920F931F93CF93DF93CDB76E
:10B3B000DEB728970FB6F894DEBF0FBECDBF2B01C6
:10B3C0003C0129833A834B835C83ED82FE820F83A9
:10B3D000188785017401209115053091160540915B
:10B3E0001705509118050E945FB04B015C01209138
:10B3F000190530911A0540911B0550911C05698172
:10B400007A818B819C810E945FB09B01AC01C50158
:10B41000B4010E9453AD4B015C0120911D05309198
:10B420001E0540911F05509120056D817E818F8101
:10B4300098850E945FB09B01AC01C501B4010E94D8
:10B4400053ADF6016083718382839383209121053C
:10B45000309122054091230550912405C301B2018A
:10B460000E945FB04B015C012091250530912605BB
:10B47000409127055091280569817A818B819C81B3
:10B480000E945FB09B01AC01C501B4010E9453ADA5
:10B490004B015C012091290530912A0540912B0533
:10B4A00050912C056D817E818F8198850E945FB0BF
:10B4B0009B01AC01C501B4010E9453ADF80160834A
:10B4C00071838283938320912D0530912E054091C5
:10B4D0002F0550913005C301B2010E945FB04B01AE
:10B4E0005C01209131053091320540913305509136
:10B4F000340569817A818B819C810E945FB09B01B8
:10B50000AC01C501B4010E9453AD4B015C01209117
:10B5100035053091360540913705509138056D81DC
:10B520007E818F8198850E945FB09B01AC01C5012F
:10B53000B4010E9453ADF7016083718382839383CA
:10B5400028960FB6F894DEBF0FBECDBFDF91CF9126
:10B550001F910F91FF90EF90DF90CF90BF90AF9031
:10B560009F908F907F906F905F904F9008953F9243
:10B570004F925F926F927F928F929F92AF92BF9203
:10B58000CF92DF92EF92FF920F931F93CF93DF93AF
:10B5900000D01F92CDB7DEB7382E6091750570913F
:10B5A000760580917705909178050E948AAE20916A
:10B5B000B9053091BA054091BB055091BC050E9478
:10B5C0005FB02B013C016093690570936A0580931D
:10B5D0006B0590936C056091790570917A05809167
:10B5E0007B0590917C050E948AAE2091BD0530912B
:10B5F000BE054091BF055091C0050E945FB06983B0
:10B600007A838B839C8360936D0570936E05809322
:10B610006F059093700560917D0570917E05809116
:10B620007F05909180050E948AAE2091C1053091DE
:10B63000C2054091C3055091C4050E945FB060935C
:10B640007105709372058093730590937405209132
:10B65000400525FF15C041E7842E45E0942E5DE6A8
:10B66000A52E55E0B52EE9E6CE2EE5E0DE2E7B01D7
:10B670008C0129813A814B815C81C301B20187DE53
:10B6800020916F04309170044091710450917204C4
:10B690006091690570916A0580916B0590916C05C8
:10B6A0000E9452AD2B013C016093690570936A05BD
:10B6B00080936B0590936C0520916B0430916C0422
:10B6C00040916D0450916E0460916D0570916E050E
:10B6D00080916F05909170050E9452AD60936D0549
:10B6E00070936E0580936F0590937005332001F180
:10B6F00040925D0550925E0560925F057092600514
:10B70000609361057093620580936305909364056F
:10B710008091710590917205A0917305B0917405A7
:10B720008093650590936605A0936705B0936805BF
:10B730000F900F900F900F90DF91CF911F910F916D
:10B74000FF90EF90DF90CF90BF90AF909F908F9041
:10B750007F906F905F904F903F9008954F925F92CF
:10B760006F927F928F929F92AF92BF92CF92DF9211
:10B77000EF92FF920F931F93CF93DF932B013C0126
:10B7800049015A016701780180913F0585FD53C049
:10B7900020E030E048EC52ECC701B6010E94EBAF6C
:10B7A00087FD1DC02DEC3CEC4CE45DE3609183040F
:10B7B0007091840480918504909186040E9453AD19
:10B7C00020E030E040EA50E40E9453AD9B01AC0120
:10B7D000C1E0C701B6010E94B7AD18160CF4C0E075
:10B7E000A3019201C301B2010E945FB06B017C0111
:10B7F000A5019401C501B4010E945FB09B01AC0199
:10B80000C701B6010E9453ADD1E02091F3043091FD
:10B81000F4044091F5045091F6040E94B7AD181657
:10B820000CF4D0E0CD2341F481E0A1DE8FEB93E175
:10B830000E943C1301C0C1E08C2FDF91CF911F917A
:10B840000F91FF90EF90DF90CF90BF90AF909F90BF
:10B850008F907F906F905F904F9008952F923F92BE
:10B860004F925F926F927F928F929F92AF92BF9210
:10B87000CF92DF92EF92FF920F931F93CF93DF93BC
:10B88000CDB7DEB760970FB6F894DEBF0FBECDBF61
:10B890001C0180918605F1011081811169C013FF9F
:10B8A00020C062857385848595850E94514E2091C4
:10B8B00041053091420540914305509144050E9455
:10B8C00052AD6093690570936A0580936B05909300
:10B8D0006C0560935D0570935E0580935F059093A2
:10B8E000600514FF21C0F101668577858089918903
:10B8F0000E94514E209145053091460540914705E3
:10B90000509148050E9452AD60936D0570936E058D
:10B9100080936F0590937005609361057093620545
:10B92000809363059093640515FF8BC0F1016289D4
:10B930007389848995890E94514E209149053091DF
:10B940004A0540914B0550914C050E9452AD6093C1
:10B9500071057093720580937305909374056093DD
:10B96000650570936605809367059093680569C0C7
:10B9700013FF21C0F10162857385848595850E943E
:10B98000514E20915D0530915E0540915F055091CB
:10B9900060050E9453AD60935D0570935E058093D2
:10B9A0005F05909360056093690570936A058093C5
:10B9B0006B0590936C0514FF21C0F10166857785B6
:10B9C000808991890E94514E2091610530916205D4
:10B9D00040916305509164050E9453AD60936105E9
:10B9E00070936205809363059093640560936D0581
:10B9F00070936E0580936F059093700515FF21C0BD
:10BA0000F10162897389848995890E94514E209140
:10BA100065053091660540916705509168050E9463
:10BA200053AD6093650570936605809367059093A9
:10BA30006805609371057093720580937305909308
:10BA400074058091400540906505509066056090B2
:10BA500067057090680585FF3BC020916B043091AD
:10BA60006C0440916D0450916E0460916105709179
:10BA7000620580916305909164050E9453AD6D87C6
:10BA80007E878F87988B20916F043091700440914E
:10BA900071045091720460915D0570915E05809112
:10BAA0005F05909160050E9453AD9E012F5F3F4F4F
:10BAB0004901AE014B5F5F4F5A01FE0139966F019C
:10BAC000830172012D853E854F855889A3D930C0E9
:10BAD00020916F0430917004409171045091720470
:10BAE00060915D0570915E0580915F0590916005A4
:10BAF0000E9453AD69877A878B879C8720916B045E
:10BB000030916C0440916D0450916E046091610518
:10BB10007091620580916305909164050E9453AD18
:10BB20006D837E838F83988749825A826B827C8261
:10BB30002091D8023091D9024091DA025091DB0273
:10BB400069857A858B859C850E945FB020E030E016
:10BB500040E05FE30E9453AD0E94C5AE0E9457AE25
:10BB600060934D0570934E0580934F05909350055B
:10BB70002091DC023091DD024091DE025091DF0223
:10BB80006D817E818F8198850E945FB020E030E0DA
:10BB900040E05FE30E9453AD0E94C5AE0E9457AEE5
:10BBA000609351057093520580935305909354050B
:10BBB0002091E0023091E1024091E2025091E302D3
:10BBC00069817A818B819C810E945FB020E030E0A6
:10BBD00040E05FE30E9453AD0E94C5AE0E9457AEA5
:10BBE00060935505709356058093570590935805BB
:10BBF000F1010081118106FF35C180919B0283FD17
:10BC000031C1F101C688D788E08CF18C8090E402C4
:10BC10009090E502A090E602B090E702A5019401A1
:10BC2000C701B6010E945FB00E94514E0E9457AEFC
:10BC30002B013C0180918605E0911C03F0911D03CE
:10BC4000811104C0809185058823B1F120E030E0A6
:10BC500046E153E462A973A984A995A90E94B7ADEE
:10BC600087FF08C080913F0587FD04C0412C512CFF
:10BC7000320115C0C701B6019F772091960230911D
:10BC8000970240919802509199020E945FB020E083
:10BC900030E04AE754E40E94EBAF18163CF3809181
:10BCA000810590918205A0918305B0918405840D52
:10BCB000951DA61DB71DDEC020E030E046E153E42F
:10BCC00062A973A984A995A90E94B7AD87FF04C092
:10BCD00080913F0587FFD7C08091810590918205B3
:10BCE000A0918305B0918405A3019201281B390B13
:10BCF0004A0B5B0BCA01B9010E948AAE9F77209163
:10BD000096023091970240919802509199020E94B8
:10BD10005FB06B017C0120E030E04AE754E4C501EC
:10BD2000B4010E945FB09B01AC01C701B6010E9443
:10BD3000EBAF18160CF4A7C04092590550925A0563
:10BD400060925B0570925C0510FF3DC08091C90553
:10BD50000091790410917A048823C9F02FE737EB1A
:10BD60004AE85BE3F101628D738D848D958D0E94AD
:10BD70005FB06B017C01B801882777FD8095982F13
:10BD80000E948AAE9B01AC01C701B60112C0B80186
:10BD9000882777FD8095982F0E948AAEF101228D29
:10BDA000338D448D558D0E945FB02EE333EC4EE20F
:10BDB00059E30E945FB060937B0470937C0480938E
:10BDC0007D0490937E04E0906505F09066050091F7
:10BDD00067051091680520916105309162054091D9
:10BDE00063055091640560915D0570915E058091D9
:10BDF0005F0590916005B2DC811111C080915905F9
:10BE000090915A05A0915B05B0915C0580938105E6
:10BE100090938205A0938305B09384050AC0F10135
:10BE2000808191819C0128733327232BC9F486FDDF
:10BE300002C080E031C04091590550915A0560918F
:10BE40005B0570915C058091810590918205A091C0
:10BE50008305B0918405481759076A077B0749F3A2
:10BE600081E01AC08091810590918205A09183059F
:10BE7000B09184058093590590935A05A0935B0572
:10BE8000B0935C0561CF409281055092820560922B
:10BE900083057092840550CF60960FB6F894DEBF8C
:10BEA0000FBECDBFDF91CF911F910F91FF90EF900B
:10BEB000DF90CF90BF90AF909F908F907F906F90CA
:10BEC0005F904F903F902F9008954F925F926F92A6
:10BED0007F92AF92BF92CF92DF92EF92FF920F9339
:10BEE0001F93CF93DF93CDB7DEB728970FB6F894A3
:10BEF000DEBF0FBECDBF69837A838B839C8329010C
:10BF00003A01ED82FE820F83188720EF33E244E787
:10BF100059E40E94B7AD882311F120916F0430914C
:10BF20007004409171045091720469817A818B810F
:10BF30009C810E9453AD2091D8023091D90240914A
:10BF4000DA025091DB020E945FB00E9457AE60930C
:10BF50004D0570934E0580934F059093500520EF4B
:10BF600033E244E759E4C301B2010E94B7AD88232C
:10BF700001F120916B0430916C0440916D0450915B
:10BF80006E04C301B2010E9453AD2091DC023091D6
:10BF9000DD024091DE025091DF020E945FB00E94FC
:10BFA00057AE60935105709352058093530590935B
:10BFB000540520EF33E244E759E46D817E818F819F
:10BFC00098850E94B7AD8823C1F02091E00230919E
:10BFD000E1024091E2025091E3026D817E818F8106
:10BFE00098850E945FB00E9457AE6093550570938C
:10BFF0005605809357059093580520EF33E244E7A8
:10C0000059E4C601B5010E94B7AD8823B1F0209173
:10C01000E4023091E5024091E6025091E702C60148
:10C02000B5010E945FB00E9457AE609359057093AE
:10C030005A0580935B0590935C0520EF33E244E75B
:10C0400059E46A8D7B8D8C8D9D8D0E94B7AD8823C0
:10C0500061F08A8D9B8DAC8DBD8D80937B04909318
:10C060007C04A0937D04B0937E0440E061E081E015
:10C070000E947B9A811106C089E993E10E94347382
:10C0800080E003C080E073DA81E028960FB6F89470
:10C09000DEBF0FBECDBFDF91CF911F910F91FF90FB
:10C0A000EF90DF90CF90BF90AF907F906F905F90B8
:10C0B0004F9008950E94321380E059DA809169050B
:10C0C00090916A05A0916B05B0916C0580935C041A
:10C0D00090935D04A0935E04B0935F0480916D051E
:10C0E00090916E05A0916F05B091700580935804F2
:10C0F00090935904A0935A04B0935B048091710506
:10C1000090917205A0917305B091740580935404C9
:10C1100090935504A0935604B09357046091810501
:10C120007091820580918305909184050E948AAE6A
:10C130002091C5053091C6054091C7055091C805AD
:10C140000E945FB060935004709351048093520436
:10C150009093530480917B0490917C04A0917D0482
:10C16000B0917E048093920290939302A0939402E4
:10C17000B093950208958F929F92AF92BF92CF9203
:10C18000DF92EF92FF920F931F93CF93DF93982E3E
:10C19000C62FD42FC22E20E030E0A9016091920278
:10C1A0007091930280919402909195020E94B7AD94
:10C1B00087FDA7C0911005C0C11103C0E1E0ED27C4
:10C1C00001C0E0E0CC2049F0A0905004B0905104B0
:10C1D000C0905204D090530408C0F0EFAF2EF3E2A9
:10C1E000BF2EF4E7CF2EF9E4DF2EE11102C0DD23EC
:10C1F000B9F0509154044091550430915604209167
:10C200005704852F942FA32FB22F80936505909309
:10C210006605A0936705B0936805E11107C004C0E7
:10C2200050EF43E234E729E4CC23B9F0D09158042D
:10C23000C091590470915A0460915B048D2F9C2F1A
:10C24000A72FB62F8093610590936205A093630595
:10C25000B0936405E11107C004C0D0EFC3E274E7F6
:10C2600069E49920B1F080905C0490905D04F091B5
:10C270005E04E0915F04C401AF2FBE2F80935D0583
:10C2800090935E05A0935F05B0936005B82DA92D2E
:10C2900004C0B0EFA3E2F4E7E9E41F930F93FF9229
:10C2A000EF92E52EF42E032F122F2D2F3C2F472F28
:10C2B000562F6B2F7A2F8F2F9E2F0E94FA57809127
:10C2C000920290919302A0919402B0919502809372
:10C2D0007B0490937C04A0937D04B0937E040F9024
:10C2E0000F900F900F9080E0DF91CF911F910F91F1
:10C2F000FF90EF90DF90CF90BF90AF909F908F9086
:10C3000036C9DF91CF911F910F91FF90EF90DF9091
:10C31000CF90BF90AF909F908F90089590914005DF
:10C3200095FB222720F9821791F0882311F0906263
:10C3300001C09F7D90934005882319F080E09AE129
:10C3400002C08AEE99E10E943E7380E010C9089510
:10C350009F92AF92BF92CF92DF92EF92FF920F9394
:10C360001F93CF93DF931F921F92CDB7DEB7182F85
:10C370009090400595FA992490F880E04A8369836B
:10C38000CDDF90913F05916090933F054A8169818F
:10C39000112319F0411103C005C061115CC00E9456
:10C3A00079541DC010924D0510924E0510924F0504
:10C3B00010925005662341F01092510510925205DB
:10C3C000109253051092540540E060E081E00E9415
:10C3D0007B9A811104C087E393E10E943473E0905B
:10C3E0008304F09084040091850410918604809168
:10C3F000C7028F938091C6028F938091C5028F935D
:10C400008091C4028F93A0EFAA2EA3E2BA2EA4E7D4
:10C41000CA2EA9E4DA2E20E030E0A901CA01B90150
:10C420000E94FA5781E0A3D88DE293E10E943C1369
:10C43000892D0F900F900F900F900F900F90DF911C
:10C44000CF911F910F91FF90EF90DF90CF90BF9011
:10C45000AF909F9063CF442309F4AECFA0CF2F922B
:10C460003F924F925F926F927F928F929F92AF9284
:10C47000BF92CF92DF92EF92FF920F931F93CF93D1
:10C48000DF93CDB7DEB72B970FB6F894DEBF0FBEA4
:10C49000CDBF6A874D8340916F04509170046091C5
:10C4A00071047091720449835A836B837C8340903A
:10C4B0006B0450906C0460906D0470906E0488233F
:10C4C00009F4AEC0222321F08DE29AE10E94D86FD8
:10C4D000C0907105D0907205E0907305F0907405DE
:10C4E00081EA93E00E944A129B01AC01C701B601A8
:10C4F0000E94EBAF18161CF5E090C4021091C50223
:10C500000091C602F090C70281EA93E00E944A12AD
:10C51000FF920F931F93EF9210EFA12E13E2B12E13
:10C5200014E7C12E19E4D12E7B018C01A6019501DF
:10C53000C601B501CADC0F900F900F900F9080E2FA
:10C5400093E00E944A12DC01CB01B05880936F0443
:10C5500090937004A0937104B093720484E293E00A
:10C560000E944A12DC01CB01B05880936B04909377
:10C570006C04A0936D04B0936E0488E493E00E9471
:10C580004A12E62E172F082FF92EA301920160916F
:10C590006B0470916C0480916D0490916E040E9404
:10C5A00052AD2091DC023091DD024091DE025091CB
:10C5B000DF020E945FB00E9457AE2B013C0129812F
:10C5C0003A814B815C8160916F047091700480911D
:10C5D0007104909172040E9452AD2091D802309162
:10C5E000D9024091DA025091DB020E945FB00E94B2
:10C5F00057AE21E02F932F93FF920F931F93EF924B
:10C60000A12CB12C6501E12CF12C8701A301920131
:10C610000E94AE9F0F900F900F900F900F900F9071
:10C620000E94321320E030E040E251E46091E002E9
:10C630007091E1028091E2029091E3020E945FB06A
:10C640000E9457AE6E837F838887998760917D05AE
:10C6500070917E0580917F059091800569837A8332
:10C660008B839C838091910590919205A091930575
:10C67000B09194058093CF049093D004A093D104FB
:10C68000B093D2041B86412C512C32017D81272E80
:10C69000312C7B85872E992487FC909482149304F7
:10C6A0000CF01FC1C090A304D090A404E090A50496
:10C6B000F090A6048091970490919804A091990419
:10C6C000B0919A04C81AD90AEA0AFB0ACC0CDD1CFC
:10C6D000EE1CFF1C8FEF9FEFDC018093BF04909353
:10C6E000C004A093C104B093C20480E293E00E940E
:10C6F0004A1284E293E00E944A12809140058064CD
:10C70000809340050E9493180E9493180AE010E05D
:10C710008091000181FF38C08CE293E00E944A12B0
:10C72000A7019601EE24FF248701E21AF30A040B05
:10C73000150B31E03F933F939F938F937F936F93BC
:10C74000A12CB12C650120E030E0A90160E070E08F
:10C75000CB010E94AE9F0F900F900F900F900F9003
:10C760000F908091BF049091C004A091C104B0913A
:10C77000C204B7FF18C084EC99E10E944873812C71
:10C78000912C30E82FEBFAC180E293E10E942773ED
:10C7900064E670E080E090E00E94A1AB01501109D6
:10C7A00009F0B6CFB9CF809140058F7B80934005CB
:10C7B0000091CF041091D0042091D1043091D20483
:10C7C0008091910590919205A0919305B091940567
:10C7D000B901A801481B590B6A0B7B0BDB01CA018D
:10C7E0004093BF045093C0046093C1047093C2048B
:10C7F0004091890550918A0560918B0570918C0557
:10C80000480F591F6A1F7B1F4093890550938A0563
:10C8100060938B0570938C0540918D0550918E052A
:10C8200060918F0570919005480F591F6A1F7B1FFB
:10C8300040938D0550938E0560938F0570939005FE
:10C8400000939105109392052093930530939405DE
:10C8500040917D0550917E0560917F057091800526
:10C86000480F591F6A1F7B1F40937D0550937E051B
:10C8700060937F057093800589819A81AB81BC812B
:10C88000841B950BA60BB70B480E591E6A1E7B1E08
:10C89000C40101968215930504F58CE293E00E9491
:10C8A0004A121F9251E05F939F938F937F936F93F0
:10C8B000A12CB12C6501EE80FF800885198520E050
:10C8C00030E0A90160E070E0CB010E94AE9F0F90C4
:10C8D0000F900F900F900F900F906B856F5F6B878D
:10C8E000D8CEC301B2010E948AAE2091C105309119
:10C8F000C2054091C3055091C4050E945FB06B0111
:10C900007C01AD816A2F70E080E090E00E9488AEEB
:10C910009B01AC01C701B6010E94BEAD6B017C0159
:10C9200088E293E00E944A129B01AC01C701B60164
:10C930000E9453AD4B018E839D8322E0AB01BC016D
:10C940008CE99AE10E944D7520E030E040EA52E423
:10C95000B4018E819D810E945FB020E030E048EC00
:10C9600054E40E9452ADAB01BC0122E080E79AE1A1
:10C970000E944D754091690550916A0560916B0563
:10C9800070916C0522E088E09EE10E944D75409117
:10C990006D0550916E0560916F057091700522E0F4
:10C9A00084E09EE10E94107580E00E94B75A8AE1FF
:10C9B00093E10E943C138CE293E00E944A129B0197
:10C9C00040917D0550917E0560917F0570918005B5
:10C9D000E980FA800B811C81E41AF50A060B170B1B
:10C9E0001F9241E04F939F938F933F932F93A12CDE
:10C9F000B12C650120E030E0A90160E070E0CB01DE
:10CA00000E94AE9F0F900F900F900F900F900F907D
:10CA1000BA85BB2309F4B0C0C0906F04D0907004F5
:10CA2000E0907104F090720420906B0430906C04DC
:10CA300040906D0450906E048CE29AE10E94D86F91
:10CA400060901C0370901D036114710409F444C0CC
:10CA5000F30181819281A381B4819C01AD0166279C
:10CA60007727CB01621B730B840B950B0E948AAE58
:10CA70002091B9053091BA054091BB055091BC0594
:10CA80000E945FB060936F04709370048093710490
:10CA900090937204F30185819681A781B0859C01F2
:10CAA000AD0166277727CB01621B730B840B950BB7
:10CAB0000E948AAE2091BD053091BE054091BF0510
:10CAC0005091C0050E945FB060936B0470936C043A
:10CAD00080936D0490936E0488E493E00E944A1260
:10CAE0005B01182F092FA201910160916B047091D5
:10CAF0006C0480916D0490916E040E9452AD20915F
:10CB0000DC023091DD024091DE025091DF020E9492
:10CB10005FB00E9457AE2B013C01A70196016091C6
:10CB20006F047091700480917104909172040E945E
:10CB300052AD2091D8023091D9024091DA02509141
:10CB4000DB020E945FB00E9457AE21E02F932F932B
:10CB50000F931F93BF92AF92A12CB12C6501E12CD2
:10CB6000F12C8701A30192010E94AE9F0F900F90BC
:10CB70000F900F900F900F903E812D81B401832F65
:10CB8000922F2B960FB6F894DEBF0FBECDBFDF916C
:10CB9000CF911F910F91FF90EF90DF90CF90BF90BA
:10CBA000AF909F908F907F906F905F904F903F904D
:10CBB0002F90089540E050E060E87FE34093350512
:10CBC00050933605609337057093380540932505DB
:10CBD000509326056093270570932805409315050B
:10CBE0005093160560931705709318051092310540
:10CBF00010923205109233051092340510922D05D3
:10CC000010922E0510922F051092300510922905D2
:10CC100010922A0510922B0510922C0510922105D6
:10CC200010922205109223051092240510921D05E2
:10CC300010921E0510921F051092200510921905E2
:10CC400010921A0510921B0510921C05811104C048
:10CC500085E19AE10C943E73089588E10FB6F8944B
:10CC600080936000109260000FBE9B9AA398809101
:10CC70003F05806480933F05389A399A3A9A8091AB
:10CC80000A01826080930A0180910A018160809389
:10CC90000A0180910A01846080930A010F9A179A11
:10CCA0000E9A169A0D9A159A3F98479A0A98129AD0
:10CCB0000998119A809101018D7F809301018091E3
:10CCC0000201826080930201809101018062809361
:10CCD0000101809102018F7D809302018091010109
:10CCE00088608093010180910201877F8093020117
:10CCF0006D9A75980E944E160E946F1781E05ADF58
:10CD000080E090E0A8E4B2E480937B0490937C04FC
:10CD1000A0937D04B0937E0484E690E090937A041F
:10CD2000809379049093780480937704109265053A
:10CD300010926605109267051092680510926105C1
:10CD400010926205109263051092640510925D05C1
:10CD500010925E0510925F05109260051092080512
:10CD6000109207051092E8181092E9181092EA182C
:10CD70001092EB1880E090E0A0E4B1E4809373049B
:10CD800090937404A0937504B093760410926B048E
:10CD900010926C0410926D0410926E0410926F0445
:10CDA00010927004109271041092720488E893E15A
:10CDB000A0E0B0E08093110590931205A0931305B5
:10CDC000B093140581E080939A021092650410924A
:10CDD0006604109267041092680410926104109225
:10CDE000620410926304109264048093400580E012
:10CDF00090E0AAE7B3E48093930490939404A09303
:10CE00009504B093960480938B0490938C04A09324
:10CE10008D04B0938E0480E090E0AFE2B3E48093A1
:10CE2000830490938404A0938504B09386041092A5
:10CE30008F04109290041092910410929204109218
:10CE40008704109288041092890410928A04109228
:10CE50007F0410928004109281041092820480E07A
:10CE600090E0A2E8B2E48093EF049093F004A093E2
:10CE7000F104B093F204109260041092CB0510926A
:10CE8000CA050E9463784091EB025091EC026091D8
:10CE9000ED027091EE0280EA96E00E943C868FE6F9
:10CEA0009EE10E9427730E946D830E9451400E9460
:10CEB0002B7F1092750510927605109277051092CF
:10CEC00078051092690510926A0510926B05109210
:10CED0006C051092790510927A0510927B051092DC
:10CEE0007C0510926D0510926E0510926F051092E0
:10CEF000700510927D0510927E0510927F051092AC
:10CF000080051092710510927205109273051092AF
:10CF1000740510928105109282051092830510927B
:10CF2000840510927505109276051092770510927F
:10CF300078050E94B34E0E94AD170E94BB170E9455
:10CF40004D8369E875E085E795E00E9494948AEF47
:10CF500093E00E94BFB590913E05882311F0926046
:10CF600001C09D7F90933E05682F70E085E492E0BC
:10CF70000E94F8738FE593E10E943C1380E00E94C9
:10CF80001B412EE088E190E00FB6F894A8958093BD
:10CF900060000FBE2093600008954F925F926F92E1
:10CFA0007F928F929F92AF92BF92CF92DF92EF9239
:10CFB000FF920F931F93CF93DF93CDB7DEB76497A4
:10CFC0000FB6F894DEBF0FBECDBF4B015C01290147
:10CFD0003A01E982FA820B831C8388E393E00E9482
:10CFE0004A126B017C0180E393E00E944A129B018C
:10CFF000AC01C701B6010E9452AD6D837E838F8361
:10D0000098878CE393E00E944A126B017C0184E3D1
:10D0100093E00E944A129B01AC01C701B6010E9435
:10D0200052AD69877A878B879C87A3019201C501DE
:10D03000B4010E9452AD2B013C0180E493E00E94B8
:10D040004A126B017C0180E393E00E944A129B012B
:10D05000AC01C701B6010E9452AD6D877E878F87F4
:10D06000988B84E493E00E944A126B017C0184E374
:10D0700093E00E944A129B01AC01C701B6010E94D5
:10D0800052AD698B7A8B8B8B9C8B29813A814B813A
:10D090005C81C501B4010E9452AD4B015C019B0152
:10D0A000AC0169857A858B859C850E945FB06B0198
:10D0B0007C0129893A894B895C89C301B2010E94AC
:10D0C0005FB09B01AC01C701B6010E9452AD6983FC
:10D0D0007A838B839C832D853E854F855889C30138
:10D0E000B2010E945FB06B017C01A50194016D81CA
:10D0F0007E818F8198850E945FB09B01AC01C70142
:10D10000B6010E9452AD2B013C0129893A894B8915
:10D110005C896D817E818F8198850E945FB06B01F3
:10D120007C012D853E854F85588969857A858B855B
:10D130009C850E945FB09B01AC01C701B6010E94B3
:10D1400052AD4B015C0129813A814B815C81CA015E
:10D15000B9010E945FB06B017C01A3019201C30180
:10D16000B2010E945FB09B01AC01C701B6010E94F1
:10D1700053AD6B017C01A5019401C501B4010E946E
:10D180005FB09B01AC01C701B6010E9453AD0E9484
:10D19000CCB06B017C0120E030E0A901C501B401F5
:10D1A0000E94B7AD87FF04C0F7FAF094F7F8F09447
:10D1B000A701960169817A818B819C810E94BEAD15
:10D1C0006D837E838F83988760932D0570932E05E2
:10D1D00080932F0590933005A7019601C301B201FA
:10D1E0000E94BEAD2B013C01609331057093320566
:10D1F0008093330590933405A7019601C501B401CE
:10D200000E94BEAD6B017C016093350570933605BD
:10D2100080933705909338051092210510922205CE
:10D220001092230510922405D301C201B0588983BE
:10D230009A83AB83BC83A7019601C701B6010E9404
:10D240005FB06D877E878F87988BA301920169817C
:10D250007A818B819C810E945FB09B01AC016D85BE
:10D260007E858F8598890E9452AD69877A878B87E2
:10D270009C872D813E814F81588569817A818B8180
:10D280009C810E945FB04B015C0120E030E0A9016D
:10D29000C701B6010E945FB09B01AC01C501B4019A
:10D2A0000E9452AD6093190570931A0580931B0577
:10D2B00090931C0520E030E0A901C301B2010E9457
:10D2C0005FB04B015C012D813E814F815885C701C4
:10D2D000B6010E945FB09B01AC01C501B4010E9480
:10D2E00052AD4B015C0129853A854B855C85CA01AD
:10D2F000B9010E945FB02B013C01A5019401C50159
:10D30000B4010E945FB09B01AC01C301B2010E9455
:10D3100053AD0E94CCB02B013C019B01AC0169854F
:10D320007A858B859C850E94BEAD609315057093B0
:10D3300016058093170590931805A3019201C50166
:10D34000B4010E94BEAD60931D0570931E058093CD
:10D350001F059093200529813A814B815C81CA0188
:10D36000B9010E945FB09B01AC016D857E858F8500
:10D3700098890E9453AD0E94CCB04B015C019B0187
:10D38000AC01C701B6010E94BEAD60932505709344
:10D3900026058093270590932805A50194016981AE
:10D3A0007A818B819C810E94BEAD60932905709328
:10D3B0002A0580932B0590932C0526E049E065E132
:10D3C00075E083ED99E164960FB6F894DEBF0FBE69
:10D3D000CDBFDF91CF911F910F91FF90EF90DF9024
:10D3E000CF90BF90AF909F908F907F906F905F9005
:10D3F0004F900C94667508958BE093E10C943E7306
:10D40000E0E3F4E011821082349684E0E035F8071E
:10D41000C9F708954091EB025091EC026091ED0242
:10D420007091EE0281E093E10E9450746FE770E02A
:10D4300084EF92E10E94067461E070E087EE92E171
:10D440000E94067460E070E087ED92E10E9406742D
:10D4500060E070E08CEC92E10E94067460E070E0A5
:10D4600084EC92E10E94067461E070E08FEB92E13F
:10D470000E94067460E070E08AEB92E10E940674FC
:10D4800061E070E085EA92E10E94067461E070E07C
:10D490008BE992E10E94067461E070E081E992E11B
:10D4A0000E94067461E070E087E892E10E940674D1
:10D4B00060E070E088E792E10E94067460E070E04E
:10D4C0008CE592E10E94067460E070E080E592E1F4
:10D4D0000E94067461E070E088E492E10E940674A4
:10D4E00061E070E08DE392E10E94067461E070E01B
:10D4F00085E392E10E94067460E170E085E292E1CA
:10D500000E940674409173045091740460917504F4
:10D510007091760422E08DE192E10E942B7540919A
:10D520008F0450919004609191047091920422E0D4
:10D5300087E192E10E942B75409187045091880405
:10D540006091890470918A0422E081E192E10E9455
:10D550002B7540917F0450918004609181047091FB
:10D56000820422E08BE092E10E942B7520919304CB
:10D5700030919404409195045091960460918F04E9
:10D580007091900480919104909192040E9453AD07
:10D59000AB01BC0122E085E092E10E942B75209155
:10D5A0008B0430918C0440918D0450918E046091D5
:10D5B0008704709188048091890490918A040E9464
:10D5C00053ADAB01BC0122E08FEF91E10E942B75BE
:10D5D0002091830430918404409185045091860405
:10D5E00060917F0470918004809181049091820405
:10D5F0000E9453ADAB01BC0122E089EF91E10E9492
:10D600002B7540919304509194046091950470910E
:10D61000960422E082EF91E10E942B7540918B04E9
:10D6200050918C0460918D0470918E0422E08BEEF9
:10D6300091E10E942B754091830450918404609184
:10D6400085047091860422E084EE91E10E942B759E
:10D650004091AC025091AD026091AE027091AF0268
:10D6600022E087ED91E10E942B754091B00250912C
:10D67000B1026091B2027091B30222E08AEC91E1B2
:10D680000E942B754091B4025091B5026091B60290
:10D690007091B70222E08DEB91E10E942B754091D1
:10D6A0009C0250919D0260919E0270919F0222E027
:10D6B0008FEA91E10E942B754091A0025091A10246
:10D6C0006091A2027091A30222E081EA91E10E949E
:10D6D0002B754091A4025091A5026091A602709111
:10D6E000A70222E083E991E10E942B7581E891E194
:10D6F000B1D768E770E085E791E10E94067488ED94
:10D7000093E18DD761E070E082ED93E10E94EC73CC
:10D710006AE380EA96E00E9444824091230250919D
:10D720002402609125027091260222E08FE691E1A9
:10D730000E94107588ED93E172D761E070E082ED90
:10D7400093E10E94EC736AE380EA96E00E944482CF
:10D7500040911B0250911C0260911D0270911E02AB
:10D7600022E085E691E10E94107588ED93E157D79C
:10D7700061E070E082ED93E10E94EC736AE380EA7D
:10D7800096E00E94448240911F02509120026091D5
:10D7900021027091220222E087E591E10E9410753A
:10D7A00088ED93E13CD761E070E082ED93E10E9467
:10D7B000EC736AE380EA96E00E94448240918A0218
:10D7C00050918B0260918C0270918D0222E08DE469
:10D7D00091E10E94107588ED93E121D761E070E03E
:10D7E00082ED93E1F9D76AE380EA96E00E944482F1
:10D7F00060EF70E084E491E1FBC70F931F93CF9338
:10D80000DF931F921F92CDB7DEB78C01BE016F5F11
:10D810007F4F0E94F6B229813A810217130719F44B
:10D8200060E070E0CB010F900F90DF91CF911F91DE
:10D830000F9108950F931F93CF93DF931F921F9221
:10D84000CDB7DEB78C014AE050E0BE016F5F7F4F7D
:10D850000E945EB429813A810217130719F460E02F
:10D8600070E0CB010F900F90DF91CF911F910F913E
:10D870000895FC014081518140FD02C084E001C057
:10D8800086E043FD8C5F44FD8C5F45FD8C5F46FD6B
:10D890008C5F50FD8C5F51FD8F5F52FD8C5F53FD9F
:10D8A0008C5FDA01A270BB27BA016470772754FF3E
:10D8B00037C022813381AB2B11F48E5F01C08C5FA6
:10D8C000672B09F08E5F20FD8C5F21FD8C5F22FDB0
:10D8D0008C5F23FD8C5F24FD8C5F25FD8C5F26FD16
:10D8E0008C5F27FD8C5F30FD8C5F31FD8C5F32FDDE
:10D8F0008C5F33FD8C5F34FD8C5F35FD8C5F36FDB6
:10D900008C5F37FD8C5F57FF13C0248130E02F5FA1
:10D910003F4F2135310514F020E530E0820F0895A6
:10D92000AB2B09F08F5F672B09F08F5F57FD805F8E
:10D930000895109242068091D3058F5F8093D3059E
:10D9400008958091D305882349F08091430626E508
:10D95000829FC00111248C5B994F089580E090E074
:10D960000895EF92FF920F931F93CF93DF93DC0103
:10D97000EB01FC01EB5AFF4F81E0482740836091A7
:10D98000DD0562507E0120E030E080E090E066231B
:10D9900019F1762F663108F075E1671BA701172F83
:10D9A0001E0DFA010191AF01800F911D8F3F91056E
:10D9B00010F08F5F9109280F391F2F3F310510F0AC
:10D9C0002F5F31091413EDCF7150472F50E04F5F97
:10D9D0005F4FE40EF51EDBCFF7014181241B3109B7
:10D9E0004081841B9109282B392B232B41F08091F6
:10D9F0009B0282FF60C186EC9EE14AD65CC18881B1
:10DA0000998111969C938E938C010027107194FF3D
:10DA10000EC02A813B8113963C932E931297FE01F0
:10DA200097FD02C0349609C03596FC8008C0FE01FF
:10DA3000329613961C921E92129720E1F22E80FFCE
:10DA400010C04191519115965C934E93149760E0EC
:10DA500070E04093D4055093D5056093D60570933C
:10DA6000D705AC01427055279C0124703327012B48
:10DA700089F0452B31F04191519117965C934E936B
:10DA80001697232BC9F02191319119963C932E932F
:10DA9000189712C0452B39F0408150E017965C93DF
:10DAA0004E9316973196232B39F0208130E019964A
:10DAB0003C932E931897319683FF0AC04191519160
:10DAC000619171911A964D935D936D937C931D971F
:10DAD00084FF0AC041915191619171911E964D93BD
:10DAE0005D936D937C93519785FF0AC0419151914D
:10DAF0006191719152964D935D936D937C9355977F
:10DB000086FF0AC0419151916191719156964D9352
:10DB10005D936D937C93599790FF0AC04191519109
:10DB2000619171915A964D935D936D937C935D973E
:10DB300091FF07C040819D012C5A3F4FE901488366
:10DB4000319692FF0AC041915191619171915E9617
:10DB50004D935D936D937C93919793FF0AC0419190
:10DB600051916191719192964D935D936D937C93D8
:10DB7000959712962D913C91139720FF0AC04191E1
:10DB800051916191719196964D935D936D937C93B4
:10DB9000999721FF0AC041915191619171919A9693
:10DBA0004D935D936D937C939D9722FF0AC04191A5
:10DBB0005191619171919E964D935D936D937C937C
:10DBC000D19723FF0AC04191519161917191D296F1
:10DBD0004D935D936D937C93D59724FF0AC041913B
:10DBE000519161917191D6964D935D936D937C9314
:10DBF000D99725FF0AC04191519161917191DA96AF
:10DC00004D935D936D937C93DD9726FF0CC04191FE
:10DC10005191619171918D01025C1F4FE801488320
:10DC200059836A837B8327FF0CC041915191619195
:10DC300071918D010E5B1F4FE801488359836A8300
:10DC40007B8330FF0CC041915191619171918D01A5
:10DC50000A5B1F4FE801488359836A837B8331FF46
:10DC60000CC041915191619171918D01065B1F4FE3
:10DC7000E801488359836A837B8332FF0CC041915A
:10DC80005191619171919D01225B3F4FE901488360
:10DC900059836A837B8397FF0AC0AE5ABF4FED93C7
:10DCA000FC93EF0DF11D108281E08093DC05109252
:10DCB000CE0581E001C080E0DF91CF911F910F91EF
:10DCC000FF90EF9008954F925F926F927F929F9294
:10DCD000AF92BF92CF92DF92EF92FF920F931F937A
:10DCE000CF93DF93EC01B62EA72E198218821B82E8
:10DCF0001A82FC01EB5AFF4F81E048274083662ED1
:10DD0000772E7E0124E5E20EF11C6E0182E5C80E3D
:10DD1000D11C9924939483010F5F1F4FF3018081DD
:10DD2000882309F415C1992787FD9095A92FB92F4C
:10DD3000FC01BA97E135F10508F008C1EE58FF4F34
:10DD40000C949AB1C80176DD6093D4057093D50523
:10DD50008093D6059093D705288139812160398336
:10DD600028837D836C83F2C0C80164DD798768876E
:10DD7000288139816F3F710509F010F4246002C0D9
:10DD80002460306139832883E1C0C80153DDDB01A1
:10DD90007F836E8328813981A9014260598348833A
:10DDA0006F3F710531F028F022603061398328839C
:10DDB00003C06731710579F02B01ECE14E1A51086F
:10DDC000F3E04F16510438F0A032B10521F0A53729
:10DDD000B10509F0BBC0F8010F5F1F4F40814053F0
:10DDE0004A30C8F39F01C9012F5F3F4FFC014081BA
:10DDF0004032C9F3F60191838083FC018F012191A8
:10DE0000222329F0A537B10551F0203241F4F80161
:10DE100010829092DC058881998190687DC02A32B9
:10DE200069F7F5CFC801E9DC6A877B878C879D8716
:10DE300088819981886070C0C801DFDC6E877F8728
:10DE4000888B998B88819981806166C0C801D5DCF7
:10DE50006A8B7B8B8C8B9D8B8881998180625CC067
:10DE6000C801CBDC6E8B7F8B888F998F88819981DD
:10DE7000806452C0C801C1DC6A8F7B8F8C8F9D8FFC
:10DE800088819981916048C0C801D4DCF701608322
:10DE900088819981926040C0C801CCDC6E8F7F8FF1
:10DEA00088A399A388819981946036C0C801C2DC97
:10DEB0006AA37BA38CA39DA38881998198602CC0C1
:10DEC000C8019BDC6EA37FA388A799A78A819B8149
:10DED00081601DC0C80191DC6AA77BA78CA79DA7A4
:10DEE0008A819B81826013C0C80187DC6EA77FA7EF
:10DEF00088AB99AB8A819B81846009C0C8017DDCB5
:10DF00006AAB7BAB8CAB9DAB8A819B8188609B832A
:10DF10008A838881998190619983888317C0C80119
:10DF200089DCEB2DFA2D80E0E615F70519F09191CB
:10DF30008927FACFBE2EAF2E861741F080919B0223
:10DF400082FF25C086EC9EE1A3D321C03801E3CE39
:10DF50008A819B8197FD0AC0888199818670927021
:10DF6000892B21F01092CE0581E012C08091CE0560
:10DF70008F5F8093CE0580919B0282FF03C089EB67
:10DF80009EE186D381E09091CE05933008F480E045
:10DF9000DF91CF911F910F91FF90EF90DF90CF9085
:10DFA000BF90AF909F907F906F905F904F9008953B
:10DFB000FF920F931F93CF93DF93CDB7DEB7C65A6F
:10DFC000D1090FB6F894DEBF0FBECDBF8C0190E033
:10DFD00080E0F801F490FF20B9F0FAE0FF16A1F01C
:10DFE0002BE3F21659F0911109C0E7E5F0E0EC0FD0
:10DFF000FD1FE80FF11DF0828F5F01C091E08F34AB
:10E0000028F40F5F1F4FE5CF8823B1F0E7E5F0E07C
:10E01000EC0FFD1FE80FF11D108240E0BE01695AB0
:10E020007F4FCE0101964FDE882331F089819A819E
:10E0300086709270892B29F4FF2051F090E080E0E7
:10E04000E0CFCE0101960E94373E0E94A953F4CF43
:10E05000CA55DF4F0FB6F894DEBF0FBECDBFDF91BC
:10E06000CF911F910F91FF900895682F80EA96E05D
:10E070000C94448280EA96E00E9436821092E10578
:10E080008091E005882311F08EE101C08EE080933D
:10E09000E8020E94A9184091D8055091D9056091D5
:10E0A000DA057091DB054F5F5F4F6F4F7F4F8BED50
:10E0B0009EE15FD381E09FE1CAC2CF92DF92EF92EF
:10E0C000FF920F931F93CF93DF93EC01888181FF21
:10E0D00037C08E819F818E369105A1F48091D40541
:10E0E0009091D505A091D605B091D7058093D8051C
:10E0F0009093D905A093DA05B093DB0581E09FE109
:10E10000A6D28EC08037910511F40E94AB178E8184
:10E110009F818A399240A1F48091D8059091D905C8
:10E12000A091DA05B091DB050196A11DB11D809388
:10E13000D8059093D905A093DA05B093DB0573C099
:10E14000888180FF65C0C090D805D090D905E09047
:10E15000DA05F090DB05970186010F5F1F4F2F4F07
:10E160003F4F4091D4055091D5056091D6057091EF
:10E17000D705D901C80184279527A627B727AA273D
:10E18000BB27892B8A2B8B2B09F43AC0C41AD50ADA
:10E1900088E2C816D10420F18091E80287FF1DC0F3
:10E1A00080919B0282FF10C0B901A80186E89EE120
:10E1B000C8D24091D4055091D5056091D605709193
:10E1C000D70580E89EE1D5D2DF91CF911F910F91C5
:10E1D000FF90EF90DF90CF904DCF81508093E80279
:10E1E0001092E1058AE79EE1C4D281E09FE1DF91D0
:10E1F000CF911F910F91FF90EF90DF90CF9027C2AA
:10E200004093D8055093D9056093DA057093DB05E8
:10E2100090DB81E09FE11BD28091E0058093DF05D8
:10E220008FEF8093E802DF91CF911F910F91FF90C4
:10E23000EF90DF90CF900895CF93DF93EC0188812A
:10E2400080FF09C08EE411DF6C817D8180E090E069
:10E25000AAD280E20ADF888181FF0BC08DE405DF4E
:10E260006E817F81882777FD8095982F9CD280E2F0
:10E27000FCDE888182FF0BC087E4F7DE6885798544
:10E28000882777FD8095982F8ED280E2EEDE8881F8
:10E29000998191FF0CC084E5E8DEFE01EC5AFF4F46
:10E2A000608170E080E090E07ED280E2DEDE8881F6
:10E2B00083FF08C04A855B856C857D8522E086EBFF
:10E2C0009EE1EBD3888184FF08C04E855F85688915
:10E2D000798922E083EB9EE1E0D3888185FF08C045
:10E2E0004A895B896C897D8922E080EB9EE1D5D3E8
:10E2F000888186FF08C04E895F89688D798D24E00A
:10E300008DEA9EE1CAD38881998190FF08C04A8D29
:10E310005B8D6C8D7D8D22E08AEA9EE1BED3888183
:10E32000998192FF07C04E8D5F8D68A179A187EA20
:10E330009EE184D28881998193FF07C04AA15BA1A5
:10E340006CA17DA184EA9EE179D28A8180FF08C018
:10E350004EA15FA168A579A522E081EA9EE19DD347
:10E360008A8181FF08C04AA55BA56CA57DA522E036
:10E370008EE99EE192D38A8182FF08C04EA55FA5F7
:10E3800068A979A922E08BE99EE187D388819981E8
:10E3900097FF05C0CE5ADF4F8881998183D1DF91E5
:10E3A000CF910C94A918CF93DF93EC0180919B023D
:10E3B00080FF07C085ED9EE132D1CE01DF91CF9184
:10E3C0003BCFDF91CF9108952091D305222381F097
:10E3D000EADF809143068F5F813019F08093430616
:10E3E00002C0109243068091D30581508093D305DB
:10E3F0000895CF92DF92EF92FF921F93CF93DF9316
:10E400008091D305811103C18091DC05882321F01F
:10E410008091D3058111FBC01092DC050E9472AB84
:10E420006B017C0180EA96E00E94F78118161906BC
:10E430000CF441C08091E80287FF04C08091E1059F
:10E440008823A9F08091CF059091D005A091D105A6
:10E45000B091D205A7019601281B390B4A0B5B0B23
:10E46000293C31054105510510F004DE1CC08091A6
:10E47000D305811120C08091CF059091D005A09146
:10E48000D105B091D205A7019601281B390B4A0B83
:10E490005B0BDA01C901893E9340A105B10558F033
:10E4A0008FEA99E1D4D0C092CF05D092D005E09206
:10E4B000D105F092D205DEE111E080EA96E00E94FB
:10E4C000F781181619060CF0A2C0C091E105C036FC
:10E4D00008F09DC0C092CF05D092D005E092D10542
:10E4E000F092D20581E08C0F8093E10580EA96E0FE
:10E4F0000E941D82EC2FF0E0EE51FA4F8083C09114
:10E50000E105C130D9F49091E8028091E20597FDD0
:10E510000DC02091DF05222349F0811104C09150E4
:10E520009093E80243C0D093E80240C0882309F4E6
:10E530003DC0881F8827881F8093E0058091E005F3
:10E540008823F1F0C23008F4B8CF8CEF8C0F823002
:10E5500028F482EE95E08DD98093DD058091DD056C
:10E56000C81348C0C091420646E5C49FE00111248B
:10E57000CC5BD94F41E062EE75E0CE01F2D926C006
:10E58000EC2FF0E0EF51FA4F8081882351F08A3070
:10E5900041F08D3031F09091DE05911120C08A3329
:10E5A000F1F410821092DE05C13019F41092E105E9
:10E5B00084CFC091420656E5C59FE0011124CC5B93
:10E5C000D94F41E062EE75E0CE017DDB882319F082
:10E5D000CE0173DD01C04EDD1092E10518C08B3312
:10E5E00011F41093DE058091DE05882319F0C150E7
:10E5F000C093E1058091E105803609F05ECFDF919F
:10E60000CF911F91FF90EF90DF90CF9033CDDF91AE
:10E61000CF911F91FF90EF90DF90CF900895CF930F
:10E62000DF93FC018491EF012196882319F01DDD11
:10E63000FE01F8CFDF91CF910895CF93DF93EC01E6
:10E6400083EE9EE1ECDFCE01DF91CF91E8CFE7DFF3
:10E650000C94A918CF93DF93EC0188ED93E1DFDFF1
:10E66000CE01DF91CF91F3CFCF93DF93EC0183EE17
:10E670009EE1D5DFCE01DF91CF91E9CFCF93DF933C
:10E68000EC018CEE9EE1CBDFCE01DF91CF91DFCFAD
:10E69000CF93DF93EC0182EF9EE1C1DFCE01DF91EA
:10E6A000CF91D5CFCF93DF93EC018991882311F0DF
:10E6B000DCDCFBCFDF91CF910895BF92CF92DF9248
:10E6C000EF92FF920F931F93CF93DF93CDB7DEB7F7
:10E6D0002B970FB6F894DEBF0FBECDBFB62E1B86AC
:10E6E0008E01055F1F4F2AE0C22ED12CE12CF12CA8
:10E6F0006B2DA70196010E945CB180E38B0D9AE01F
:10E70000299F80191124F80182938F012115310569
:10E710004105510521F0B22E732FCA01E9CFCF0177
:10E72000C1DF2B960FB6F894DEBF0FBECDBFDF91D1
:10E73000CF911F910F91FF90EF90DF90CF90BF90FE
:10E740000895CF93DF9300D01F92CDB7DEB74983F2
:10E750005A836B837C8363DF49815A816B817C811F
:10E76000CB01BA010F900F900F900F90DF91CF91D6
:10E77000A4CFCF93DF9300D01F92CDB7DEB74983EC
:10E780005A836B837C834BDF49815A816B817C8107
:10E79000CB01BA0192DF0F900F900F900F90DF9195
:10E7A000CF910C94A918CF92DF92EF92FF926B0158
:10E7B0007C0197FF0AC08DE258DCF094E094D0947D
:10E7C000C094C11CD11CE11CF11CC701B601FF9013
:10E7D000EF90DF90CF9071CFCF93DF93EB011FDFEE
:10E7E000BE01882777FD8095982FDF91CF91DBCFF1
:10E7F000CF93DF93EB0113DFBE01882777FD809570
:10E80000982FD1DFDF91CF910C94A9180F931F930C
:10E81000CF93DF931F921F92CDB7DEB78C0188EDA7
:10E8200093E169837A83FBDE69817A81C8010F9065
:10E830000F90DF91CF911F910F91DACFCF93DF939C
:10E8400000D01F92CDB7DEB749835A836B837C8398
:10E85000E6DE49815A816B817C81CB01BA010F9040
:10E860000F900F900F90DF91CF919DCFCF93DF93BB
:10E8700000D01F92CDB7DEB749835A836B837C8368
:10E88000CEDE49815A816B817C81CB01BA018BDF5D
:10E890000F900F900F900F90DF91CF910C94A918CB
:10E8A0000F931F93CF93DF9300D01F92CDB7DEB7A6
:10E8B0008C0188ED93E149835A836B837C83AFDEBF
:10E8C00049815A816B817C81C8010F900F900F9014
:10E8D0000F90DF91CF911F910F91C8CF8F929F9290
:10E8E000AF92BF92CF92DF92EF92FF92CF936B01E4
:10E8F0007C01C42F9B01AC010E940AB1882319F04E
:10E900008DEF9EE11AC046015701E894B7F82FEF4A
:10E910003FEF4FE75FE7C501B4010E940AB18111E3
:10E9200016C02FEF3FEF4FE75FE7C501B4010E942C
:10E93000B7AD181664F489EF9EE1CF91FF90EF9088
:10E94000DF90CF90BF90AF909F908F9068CE20E0E7
:10E9500030E0A901C701B6010E94B7AD87FF06C02C
:10E960008DE283DBF7FAF094F7F8F094B12C60E0D5
:10E9700070E080E09FE3BC1641F020E030E040E230
:10E9800051E40E94BEADB394F6CF9B01AC01C70128
:10E99000B6010E9453AD6B017C010E945CAE4B013D
:10E9A0005C010E9488AE9B01AC01C701B6010E94C8
:10E9B00052AD6B017C01C501B4017FDECC2311F0A7
:10E9C0008EE253DBCC2311F120E030E040E251E451
:10E9D000C701B6010E945FB06B017C010E9457AE77
:10E9E0004B01AA2497FCA094BA2CC501B401DBDE2C
:10E9F000C501B4010E948AAE9B01AC01C701B601FA
:10EA00000E9452AD6B017C01C150DCCFCF91FF90D1
:10EA1000EF90DF90CF90BF90AF909F908F90089530
:10EA2000CF92DF92EF92FF92CF93DF931F92CDB7F9
:10EA3000DEB76A017B012983F2DD2981422FC701FC
:10EA4000B6014CDF0F90DF91CF91FF90EF90DF90F8
:10EA5000CF900C94A9180F931F93CF93DF9300D0FE
:10EA60001F921F92CDB7DEB78C0188ED93E12D8305
:10EA700049835A836B837C83D2DD2D8149815A81FE
:10EA80006B817C81C8010F900F900F900F900F90B9
:10EA9000DF91CF911F910F91C3CFCF92DF92EF9271
:10EAA000FF92CF93DF931F92CDB7DEB76A017B0150
:10EAB0002983B5DD2981422FC701B6010F90DF916F
:10EAC000CF91FF90EF90DF90CF9008CFCF92DF9261
:10EAD000FF920F931F93CF93DF931F921F92CDB797
:10EAE000DEB7042FF22E69837A8399DD6981C62E01
:10EAF0007A81D72E10E0101761F0F6014191519103
:10EB0000619171916F012F2D8DE89DE1C6DF1F5F2F
:10EB1000F2CF0F900F90DF91CF911F910F91FF9047
:10EB2000DF90CF900C94A9180895CF93DF9300D075
:10EB30001F92CDB7DEB749835A836B837C8344E051
:10EB400050E0BC01CE0101960E94D1B50F900F900C
:10EB50000F900F90DF91CF9108954DEC5CEC6CE439
:10EB60007EEB88E293E0E1DF40E050E064EB72E4AA
:10EB70008CE293E0DADF40E050E068E472E488E49D
:10EB800093E0D3DF40E050E0BA0180E293E0CDDFD4
:10EB900040E050E0BA0184E293E0C7DF40E050E09B
:10EBA00068E572EC80E393E0C0DF40E050E068EF9E
:10EBB00071EC84E393E0B9DF40E050E068E572E493
:10EBC00088E393E0B2DF40E050E068EF71EC8CE363
:10EBD00093E0ABDF40E050E0BA0180E493E0A5DFD2
:10EBE00040E050E062E872E484E493E09EDF40E0BD
:10EBF00050E0BA0180ED93E098DF40E050E0BA01C8
:10EC000084ED93E092DF40E050E0BA0188ED93E0BC
:10EC10008CDF40E050E060EA71E481EA93E085DF58
:10EC200046E656EE66E073E481E793E07EDF40E07F
:10EC300050E062E872E485E793E077DF68EC70E02B
:10EC400089E793E00E94EDB560E570E08BE793E023
:10EC50000E94EDB561E070E08BE290E00E94EDB5BE
:10EC600060E070E08DE793E00E94EDB560E070E059
:10EC70008FE793E00E94EDB560E070E081E893E0FB
:10EC80000E94EDB540E050E062E573E485E893E072
:10EC90004CDF40E050E065EA73E489E893E045DF4B
:10ECA00040E050E064EB72E48DE893E03EDF40E04A
:10ECB00050E0BA0181E993E038DF40E050E0BA016A
:10ECC00085E993E032DF40E050E0BA0189E993E062
:10ECD0002CDF40E050E062E872E48DE993E025DF4C
:10ECE00040E050E0BA0185EA93E01FDF40E050E0E9
:10ECF000BA0189EA93E019DF40E050E0BA018DEAF9
:10ED000093E013DF40E050E0BA0180ED93E00DDFC7
:10ED100040E050E0BA0184ED93E007DF40E050E0CE
:10ED2000BA0188ED93E001DF60E08CED93E00E9492
:10ED3000DAB540E050E060E470E480EE93E0F5DEA8
:10ED400040E050E060E571E484EE93E0EEDE40E008
:10ED500050E060E272E488EE93E0E7DE40E050E0ED
:10ED6000BA018CEE93E0E1DE40E050E0BA0180EFC2
:10ED700093E0DBDE40E050E0BA0184EF93E0D5DEC3
:10ED800040E050E060EA71E488EF93E0CEDE60E0BE
:10ED90008AEF93E00C94DAB580E990EDA3E0B0E05F
:10EDA0008093EB029093EC02A093ED02B093EE02FD
:10EDB00080EA9BEBADE0B0E08093F3029093F40225
:10EDC000A093F502B093F60280EC97E2A9E0B0E0E0
:10EDD0008093EF029093F002A093F102B093F202BD
:10EDE00080E090E0A0EAB2E48093D8029093D90248
:10EDF000A093DA02B093DB028093DC029093DD02F1
:10EE0000A093DE02B093DF028093E0029093E102D0
:10EE1000A093E202B093E30240E050E060E87FE3B9
:10EE20004093E4025093E5026093E6027093E70298
:10EE300040E050E06AEF72E44093C8025093C90288
:10EE40006093CA027093CB024093CC025093CD02E0
:10EE50006093CE027093CF024093D0025093D102C0
:10EE60006093D2027093D3028093BC029093BD0250
:10EE7000A093BE02B093BF028093C0029093C102E0
:10EE8000A093C202B093C3028093C4029093C502C0
:10EE9000A093C602B093C70280E090E0A0E4B1E482
:10EEA0008093730490937404A0937504B0937604D4
:10EEB00080E090E0AAE7B3E48093AC029093AD02C7
:10EEC000A093AE02B093AF028093B0029093B102D0
:10EED000A093B202B093B3028093B4029093B502B0
:10EEE000A093B602B093B70240E050E068EC73E440
:10EEF00040939C0250939D0260939E0270939F02E8
:10EF00004093A0025093A1026093A2027093A302C7
:10EF10004093A4025093A5026093A6027093A702A7
:10EF20008093930490939404A0939504B0939604D3
:10EF300080938B0490938C04A0938D04B0938E04E3
:10EF400080E090E0AFE2B3E4809383049093840484
:10EF5000A0938504B093860410928F0410929004BD
:10EF600010929104109292041092870410928804D7
:10EF70001092890410928A0410927F0410928004E7
:10EF800010928104109282048DEC9CECA8EBB2E408
:10EF90008093150290931602A0931702B093180263
:10EFA00080E090E0A8ECB2E480931B0290931C02F6
:10EFB000A0931D02B0931E0280E090E0A4E3B2E4AF
:10EFC0008093230290932402A0932502B0932602FB
:10EFD00080E090E2ABECB5E480931F0290932002B6
:10EFE000A0932102B093220281E080934A0228EC90
:10EFF00020934F0288E78093500280E090E0A8ECD5
:10F00000B1E48093510290935202A0935302B093C3
:10F0100054028AE999E9A9E5BFE3809355029093E8
:10F020005602A0935702B093580280E090E0A0E30C
:10F03000B3E48093590290935A02A0935B02B09379
:10F040005C0282ED80935D02109211021092120216
:10F05000109213021092140210920D0210920E02DE
:10F0600010920F021092100283E090E090932C0215
:10F0700080932B0286E990E090932E0280932D02DC
:10F080001092300210922F022093880210923102C7
:10F0900010923202109233021092340280E00E94E9
:10F0A0008E6181E00E94DA6558DD0E94B34EE091E6
:10F0B0001C03F0911D0380810E941B410E94123F9E
:10F0C00087E698E1DBCA80E990EDA3E0B0E08093A9
:10F0D000EB029093EC02A093ED02B093EE0280E07D
:10F0E00090E00E94BFB5813061F48BE490E00E9413
:10F0F000C7B56093EB027093EC028093ED0290939E
:10F10000EE0208951F93CF93DF9310E0C0E0D0E0AC
:10F11000C836D10521F0CE010E94BFB5180F219647
:10F12000C11588E0D807A1F7812FDF91CF911F91FA
:10F130000895FF920F931F93CF93DF93F82E409182
:10F14000EB025091EC026091ED027091EE028BE4C3
:10F1500090E00E94E8B54091F3025091F402609172
:10F16000F5027091F6028FE490E00E94E8B54091BC
:10F17000EF025091F0026091F1027091F20283E58A
:10F1800090E00E94E8B54091D8025091D902609178
:10F19000DA027091DB0283E090E0C7DC4091DC0290
:10F1A0005091DD026091DE027091DF0287E090E015
:10F1B000BCDC4091E0025091E1026091E20270916A
:10F1C000E3028BE090E0B1DC4091C8025091C902AB
:10F1D0006091CA027091CB028FE090E0A6DC409172
:10F1E000CC025091CD026091CE027091CF0283E1AA
:10F1F00090E09BDC4091D0025091D1026091D2020C
:10F200007091D30287E190E090DC4091BC02509174
:10F21000BD026091BE027091BF028BE190E085DC7F
:10F220004091C0025091C1026091C2027091C3022C
:10F230008FE190E07ADC4091C4025091C502609168
:10F24000C6027091C70283E290E06FDC40917304C4
:10F2500050917404609175047091760487E290E097
:10F2600064DC4091AC025091AD026091AE027091AD
:10F27000AF0283E390E059DC4091B0025091B102BB
:10F280006091B2027091B30287E390E04EDC40914E
:10F29000B4025091B5026091B6027091B7028BE34F
:10F2A00090E043DC40919C0250919D0260919E024F
:10F2B00070919F028FE390E038DC4091A002509162
:10F2C000A1026091A2027091A30283E490E02DDC80
:10F2D0004091A4025091A5026091A6027091A702EC
:10F2E00087E490E022DC61E08AE690E00E94DAB5F3
:10F2F0006FEF8BE690E00E94DAB560E58CE790E076
:10F300000E94DAB542E558EB6FEA72E48CE690E0D1
:10F310000CDC47ED53EA60E470E480E790E005DC44
:10F320004BE754E760E274E484E790E0FEDB6FEFC4
:10F3300088E790E00E94DAB540918F0450919004E4
:10F34000609191047091920485E890E0EEDB409129
:10F350008704509188046091890470918A0489E837
:10F3600090E0E3DB40917F04509180046091810440
:10F37000709182048DE890E0D8DB40919304509125
:10F380009404609195047091960481E990E0CDDB3E
:10F3900040918B0450918C0460918D0470918E0487
:10F3A00085E990E0C2DB4091830450918404609130
:10F3B00085047091860489E990E0B7DB4091EF0401
:10F3C0005091F0046091F1047091F20485E793E0AC
:10F3D000ACDB40E050E0BA018DE990E0A6DB40E014
:10F3E00050E0BA0181EA90E0A0DB40E050E0BA01D1
:10F3F00085EA90E09ADB6091400565FB662760F93D
:10F4000080E793E00E94DAB5C5E1D5E000E010E0C6
:10F410004991599169917991C801880F991F880F75
:10F42000991F845B9C4F81DB0F5F1F4F09301105D3
:10F4300079F7A89540911502509116026091170234
:10F440007091180288EC90E070DB40911B025091A3
:10F450001C0260911D0270911E028CEC90E065DB35
:10F46000409123025091240260912502709126025E
:10F4700080ED90E05ADB40911F0250912002609194
:10F4800021027091220284ED90E04FDB60914A02EC
:10F4900088ED90E00E94DAB560914F0289ED90E02E
:10F4A0000E94DAB56091500285EF90E00E94DAB5D3
:10F4B0004091510250915202609153027091540256
:10F4C0008AED90E032DB40915502509156026091F6
:10F4D0005702709158028EED90E027DB409159025F
:10F4E00050915A0260915B0270915C0282EE90E052
:10F4F0001CDB60915D0286EE90E00E94DAB54091DF
:10F500000D0250910E0260910F027091100287EE71
:10F5100090E00E94E8B54091110250911202609172
:10F520001302709114028BEE90E00E94E8B5609196
:10F530002B0270912C028FEE90E00E94EDB560914D
:10F540002D0270912E028AEF90E00E94EDB560913D
:10F550002F02709130028CEF90E00E94EDB5609127
:10F5600088028EEF90E00E94DAB540E050E0BA01E8
:10F5700081EF90E0DADA40913102509132026091ED
:10F5800033027091340286EF90E0CFDAFF2071F001
:10F5900040E050E0BA018DE790E00E94E8B540E01D
:10F5A00050E0BA0181E890E0C0DAD7DA6CE089E691
:10F5B00090E00E94DAB5A6DD682F88E690E0DF9142
:10F5C000CF911F910F91FF900C94DAB58F929F927B
:10F5D000AF92BF92CF92DF92EF92FF921F93CF93A1
:10F5E000DF9389E690E00E94BFB5182F8BE490E08E
:10F5F0000E94C7B56093EB027093EC028093ED021A
:10F600009093EE028FE490E00E94C7B56093F302FE
:10F610007093F4028093F5029093F60283E590E0F4
:10F620000E94C7B56093EF027093F0028093F102DD
:10F630009093F20283E090E00E944A126093D80215
:10F640007093D9028093DA029093DB0287E090E016
:10F650000E944A126093DC027093DD028093DE0206
:10F660009093DF028BE090E00E944A126093E002E8
:10F670007093E1028093E2029093E3028FE090E0C6
:10F680000E944A126093C8027093C9028093CA0212
:10F690009093CB0283E190E00E944A126093CC02E7
:10F6A0007093CD028093CE029093CF0287E190E0D9
:10F6B0000E944A126093D0027093D1028093D202CA
:10F6C0009093D3028BE190E00E944A126093BC02B7
:10F6D0007093BD028093BE029093BF028FE190E0D1
:10F6E0000E944A126093C0027093C1028093C202CA
:10F6F0009093C30283E290E00E944A126093C40296
:10F700007093C5028093C6029093C70287E290E08F
:10F710000E944A126093730470937404809375047A
:10F720009093760483E390E00E944A126093AC02C7
:10F730007093AD028093AE029093AF0287E390E0A6
:10F740000E944A126093B0027093B1028093B20299
:10F750009093B3028BE390E00E944A126093B4024C
:10F760007093B5028093B6029093B7028FE390E056
:10F770000E944A1260939C0270939D0280939E02A5
:10F7800090939F0283E490E00E944A126093A0024B
:10F790007093A1028093A2029093A30287E490E069
:10F7A0000E944A126093A4027093A5028093A6025D
:10F7B0009093A70285E890E00E944A1260938F041C
:10F7C00070939004809391049093920489E890E060
:10F7D0000E944A126093870470938804809389047E
:10F7E00090938A048DE890E00E944A1260937F040F
:10F7F00070938004809381049093820481E990E067
:10F800000E944A1260939304709394048093950429
:10F810009093960485E990E00E944A1260938B04CD
:10F8200070938C0480938D0490938E0489E990E00A
:10F830000E944A1260938304709384048093850429
:10F840009093860485E793E00E944A126093EF0448
:10F850007093F0048093F1049093F204133008F451
:10F8600092C065E1E62E65E0F62EC0E0D0E0CE0164
:10F87000880F991F880F991F845B9C4F0E944A1222
:10F88000F70161937193819391937F012196C93020
:10F89000D10569F7609115057091160580911705DE
:10F8A000909118059B01AC010E940AB1811106C01C
:10F8B000C5E1D5E0C12CD12C76012BC045E1E42E69
:10F8C00045E0F42ECCE4D3E0CE01880F991F880FD9
:10F8D000991F0E944A12F70161937193819391934A
:10F8E0007F012196C535F3E0DF0771F7E1CFA50170
:10F8F0009401C501B4010E945FB09B01AC01C70136
:10F90000B6010E9453AD6B017C0185E0C933D80775
:10F9100089F089909990A990B990A5019401C501A9
:10F92000B4010E940AB1882311F320E030E040E2E4
:10F9300051E4E5CF2DEC3CEC4CE250E4C701B601BC
:10F940000E94B7AD87FD0AC023E333E343E550E4EB
:10F95000C701B6010E94EBAF18161CF480E00E94AC
:10F96000DA6580E793E00E94BFB591E0811101C0A4
:10F9700090E0892F0E948E6126E049E065E175E004
:10F9800083ED99E1A3D8A89588EC90E00E944A12F3
:10F9900060931502709316028093170290931802D9
:10F9A0008CEC90E00E944A1260931B0270931C0240
:10F9B00080931D0290931E0280ED90E00E944A12F7
:10F9C0006093230270932402809325029093260271
:10F9D00084ED90E00E944A1260931F02709320020F
:10F9E000809321029093220288ED90E00E94BFB59F
:10F9F00080934A0289ED90E00E94BFB580934F0248
:10FA000085EF90E00E94BFB5809350028AED90E0B0
:10FA10000E944A12609351027093520280935302E3
:10FA2000909354028EED90E00E944A12609355022A
:10FA300070935602809357029093580282EE90E0A2
:10FA40000E944A126093590270935A0280935B029B
:10FA500090935C0286EE90E00E94BFB580935D02B9
:10FA600087EE90E00E94C7B560930D0270930E027E
:10FA700080930F02909310028BEE90E00E94C7B526
:10FA800060931102709312028093130290931402F8
:10FA90008FEE90E00E94CCB590932C0280932B02C5
:10FAA0008AEF90E00E94CCB590932E0280932D02B5
:10FAB0008CEF90E00E94CCB59093300280932F029F
:10FAC00086EF90E00E944A126093310270933202F6
:10FAD0008093330290933402123048F08EEF90E01E
:10FAE0000E94BFB5809388021C3009F44DC183E4A5
:10FAF00098E10E943E73133008F053C04DEC5CEC6B
:10FB00006CE47EEB88E293E010D840E050E064EBD8
:10FB100072E48CE293E009D840E050E068E472E4DB
:10FB200088E493E002D840E050E0BA0180E293E03C
:10FB30000E94957540E050E0BA0184E293E00E9493
:10FB4000957540E050E068E572EC80E393E00E9438
:10FB5000957540E050E068EF71EC84E393E00E941B
:10FB6000957540E050E068E572E488E393E00E9418
:10FB7000957540E050E068EF71EC8CE393E00E94F3
:10FB8000957540E050E0BA0180E493E00E949575DD
:10FB900040E050E062E872E484E493E00E949575EE
:10FBA00002C01330A9F546E656EE66E073E481E73D
:10FBB00093E00E94957540E050E062E872E485E7CA
:10FBC00093E00E94957561E070E08BE290E00E9406
:10FBD000EDB568EC70E089E793E00E94EDB560E573
:10FBE00070E08BE793E00E94EDB560E070E08DE798
:10FBF00093E00E94EDB560E070E08FE793E00E9433
:10FC0000EDB560E070E081E893E00E94EDB502C0E0
:10FC10001430C9F440E050E062E573E485E893E015
:10FC20000E94957540E050E065EA73E489E893E04E
:10FC30000E94957540E050E064EB72E48DE893E03B
:10FC40000E94957502C01530B1F440E050E0BA0151
:10FC500081E993E00E94957540E050E0BA0185E9A2
:10FC600093E00E94957540E050E0BA0189E993E085
:10FC70000E94957502C01630F1F440E050E062E851
:10FC800072E48DE993E00E94957540E050E0BA017E
:10FC900085EA93E00E94957540E050E0BA0189EA58
:10FCA00093E00E94957540E050E0BA018DEA93E040
:10FCB0000E94957502C0173049F440E050E060EAB8
:10FCC00071E481EA93E00E94957502C01A30B0F4A5
:10FCD00040E050E0BA0180ED93E00E94957540E06D
:10FCE00050E0BA0184ED93E00E94957540E050E049
:10FCF000BA0188ED93E00E94957502C01A3031F484
:10FD000060E08CED93E00E94DAB502C01B30D1F5C3
:10FD100040E050E060E470E480EE93E00E9495756E
:10FD200040E050E060E571E484EE93E00E94957558
:10FD300040E050E060E272E488EE93E00E94957546
:10FD400040E050E0BA018CEE93E00E94957540E0EF
:10FD500050E0BA0180EF93E00E94957540E050E0DA
:10FD6000BA0184EF93E00E94957540E050E060EAAC
:10FD700071E488EF93E00E94957560E08AEF93E06C
:10FD80000E94DAB580E0D5D90E94B34EDF91CF91C1
:10FD90001F91FF90EF90DF90CF90BF90AF909F901A
:10FDA0008F900C94123FCF93DF931F92CDB7DEB7A5
:10FDB000FC01808191819C0122273A7021153A40F3
:10FDC00071F4DF01AC5ABF4F2C91213009F148F595
:10FDD00092FF05C0668D82A193A10E94DAB592D9E7
:10FDE000682F88E690E069830E94BFB56981681733
:10FDF00021F088E690E00E94DAB5E8DBE0911C0390
:10FE0000F0911D0380810F90DF91CF910C941B41E5
:10FE100092FFE5CF668D778D82A193A10E94EDB50B
:10FE2000DECF223059F492FFDACF468D578D60A194
:10FE300071A182A193A10E94E8B5D1CF233079F6B8
:10FE400083FFCDCF428553856485758582A193A1BB
:10FE50000E949575C4CFCF93DF9354D9C82F88E6FD
:10FE600090E00E94BFB5D82F80E090E00E94BFB51F
:10FE7000813011F4DC1771F061E080E090E00E94C5
:10FE8000DAB50E94AD7581E0DC1301C080E0DF913E
:10FE9000CF914FC9DF91CF9199CBCF93DF931F9231
:10FEA000CDB7DEB72FD9682F88E690E069830E942E
:10FEB000BFB56981681739F088E690E00F90DF914F
:10FEC000CF910C94DAB50F90DF91CF910895CF9236
:10FED000DF92EF92FF9220E030E0A901609161048F
:10FEE0007091620480916304909164040E94B7ADA4
:10FEF000882309F45DC00E9472ABC0906504D09065
:10FF00006604E0906704F09068046C197D098E091E
:10FF10009F0928EE33E040E050E00E945CB16901A7
:10FF20007A018DE790E00E94C7B5AB01BC014C0D92
:10FF30005D1D6E1D7F1D8DE790E00E94E8B581E894
:10FF400090E00E944A126B017C012FE632E143E807
:10FF50005AE360916104709162048091630490910E
:10FF600064040E945FB09B01AC01C701B6010E940E
:10FF700053ADAB01BC0181E890E00E9495751092F1
:10FF800061041092620410926304109264040E944F
:10FF900072AB6093650470936604809367049093DA
:10FFA00068047BDFFF90EF90DF90CF900C94791581
:10FFB000FF90EF90DF90CF900895885C910988358D
:10FFC00022E0920768F464E670E00E9435B16F5F4A
:10FFD0007F4F82ED93E10E94EC7380E20C943570C8
:10FFE0000895EF92FF920F931F93CF93DF931F9289
:10FFF000CDB7DEB77C018B01BC0187E298E1498374
:020000021000EC
:100000000E94EC7380E20E943570C7010E944A1280
:1000100049810E946E7480E20E943570C701CDDF75
:10002000C8010F90DF91CF911F910F91FF90EF903A
:100030000C9427730F931F93CF93DF93EC018B01E5
:10004000BC018EE298E10E94EC7380E20E94357060
:10005000CE010E94C7B50E94D37380E20E94357022
:10006000CE01ABDFC801DF91CF911F910F910C94AE
:1000700027730F931F93CF93DF93EC018B01BC0188
:1000800085E398E10E94EC7380E20E943570CE0116
:100090000E94CCB5BC01882777FD8095982F0E94DF
:1000A000D37380E20E943570CE0187DFC801DF91F3
:1000B000CF911F910F910C9427730F931F93CF93A0
:1000C000DF93EC018B01BC018CE398E10E94EC739F
:1000D00080E20E943570CE010E94BFB5682F70E0AB
:1000E00080E090E00E94D37380E20E943570CE01E0
:1000F00064DFC801DF91CF911F910F910C9427739A
:100100006EE178E18BE490E095DF60E178E18BE2ED
:1001100090E0AFDF43E06BEF77E181E890E061DFF3
:1001200068EE77E18DE790E085DF6AEC77E18FE4B8
:1001300090E080DF61EA77E183E590E07BDF44E0F7
:100140006AEE76E18BE090E04CDF43E065ED76E12E
:1001500087E190E046DF43E06EEB76E183E290E0FA
:1001600040DF43E06AE277E187E290E03ADF43E094
:1001700061E977E185E890E034DF43E061E877E129
:1001800089E890E02EDF43E061E777E18DE890E0D9
:1001900028DF43E06FE577E181E990E022DF43E08B
:1001A0006DE477E185E990E01CDF43E06BE377E104
:1001B00089E990E016DF43E064E177E18BE390E0CA
:1001C00010DF43E067EF76E187E490E00ADF43E089
:1001D00065EA76E181E793E004DF43E063E876E1F6
:1001E00085E793E0FEDE43E06EED75E18DE993E097
:1001F000F8DE65E576E18BE793E03BDF6BE676E1E1
:1002000089E793E036DF66E376E18DE793E031DF5F
:1002100067E176E18FE793E02CDF68EF75E181E835
:1002200093E027DF43E068EB7CE185E893E0D9DEEB
:1002300043E06AEA7CE189E893E0D3DE43E06DE9DC
:100240007CE18DE893E0CDDE43E06AE87CE181E982
:1002500093E0C7DE43E067E77CE185E993E0C1DE38
:1002600043E064E67CE189E993E0BBDE43E068ECCF
:1002700075E185EA93E0B5DE43E062EB75E189EA7A
:1002800093E0AFDE43E06CE975E18DEA93E0A9DE2F
:1002900043E06BE979E188E293E0A3DE43E06DE7B8
:1002A00079E181EA93E09DDE43E06CE379E18CE261
:1002B00093E097DE43E063E279E188E493E091DE46
:1002C00043E067E679E180E293E08BDE43E061E5BD
:1002D00079E184E293E085DE43E068E179E180E35F
:1002E00093E07FDE43E06DE079E184E393E079DE43
:1002F00043E062E079E188E393E073DE43E067EF97
:1003000078E18CE393E06DDE43E06CEE78E180E42D
:1003100093E067DE43E061EE78E184E493E061DE40
:100320006AEC78E180E793E0C8DE43E06FE875E1CE
:1003300088EC90E056DE43E06AE775E18CEC90E0F3
:1003400050DE43E064E675E180ED90E04ADE43E094
:100350006EE475E184ED90E044DE6BE375E188EDD9
:1003600090E0ABDE6DE275E189ED90E0A6DE6FE135
:1003700075E185EF90E0A1DE44E06AE075E18AED89
:1003800090E02FDE44E06FEF74E18EED90E029DE27
:1003900044E064EF74E182EE90E023DE6EED74E100
:1003A00086EE90E08ADE6DEC74E187EE90E042DE4E
:1003B0006CEB74E18BEE90E03DDE63EA74E18FEE6E
:1003C00090E057DE6DE774E18AEF90E052DE67E57A
:1003D00074E18CEF90E04DDE69E374E18EEF90E024
:1003E0006CDE43E067E274E186EF90E0FACDFC0159
:1003F00024813581F901E058FF4F808131962081B9
:1004000090E080589F4F821B91098F77992708951C
:10041000FC0184819581FC01E058FF4F30813196C9
:100420002081321739F02081FC01E20FF11D80811B
:1004300090E008958FEF9FEF0895FC0184819581EE
:10044000FC01E058FF4F308131962081321759F07E
:100450002081DC01A20FB11D8C9190819F5F9F775D
:10046000908390E008958FEF9FEF0895FC018681BF
:100470009781FC01E05CFF4FDC01AF5BBF4F308137
:100480002C913213FCCF0895CF93DF93FC0186812A
:100490009781DC01A05CBF4F2C912F5F2F73EC0183
:1004A000CF5BDF4F38812317E9F33C91DC01A30FC9
:1004B000B11D6C93A681B781A05CBF4F2C93A6851C
:1004C000B7852C9181E090E0058802C0880F991FC4
:1004D0000A94E2F7282B2C9381E090E0DF91CF91F2
:1004E0000895EF92FF920F93EE24FF189923A1F441
:1004F000882309F012C001E1661F771F0A9509F4ED
:1005000031C0EE1CFF1CE41AF50A20F4E40EF51EBF
:100510008894F2CF0894F0CF12C009E1661F771FCC
:10052000881F0A9509F41EC0EE1CFF1CE41AF50A88
:1005300020F4E40EF51E8894F1CF0894EFCF01E289
:10054000661F771F881F991F0A9509F40BC0EE1CC0
:10055000FF1CE41AF50A20F4E40EF51E8894F0CF8F
:100560000894EECF0F91FF90EF90089530EC222782
:10057000B0E4AA1B18F08A179B0720F08A1B9B0B7C
:10058000A22BB32B36952795B327A227661F771F7B
:10059000881F991F60FFEECF18F0A817B90720F445
:1005A000730B8A0B9B0BA395770F881F991F10F075
:1005B000A817B907A31FB31F9B2F8A2F08954F9227
:1005C0005F92811520E2920708F03CC0811522E07D
:1005D000920768F48A30910510F48AE090E0AC014B
:1005E00060E074E284EF90E05F904F907ACFAC01CE
:1005F000E2E5FFE1242F2F715695479556954795D3
:1006000056954795569547954E7FE40FF51F659192
:1006100075912B010590401805905008249DA0016C
:10062000259D500DE12D440F551FEE1F440F551F02
:10063000EE1F440F551FEE1F651B7E0B8827992761
:10064000112428C0AC01E4E5F1E29A013F7056950F
:10065000569556955E7FE50FF11D659175912B01BD
:100660000590401805905008249DA001359DE02D6F
:10067000259D500DE11D349D500DE11D507F52957B
:10068000E2954E2F407F542BEF70651B7E0B882721
:10069000992711245F904F90089514BCEEE6F0E086
:1006A00080818260808314BC80E488BD8081846006
:1006B00080831092800010928200EFE6F0E01082BA
:1006C00089E0809381008CED9FEF90938900809367
:1006D00088008081826080830895CF93C4B7C0FF73
:1006E00004C087E69EE10E943E73C1FF04C088E516
:1006F0009EE10E943E73C2FF04C088E49EE10E9416
:100700003E73C3FF04C089E39EE10E943E73C5FFB0
:1007100004C08AE29EE10E943E7314BECF91089508
:100720001F93CF93DF931FB7F89484E090E00E946B
:10073000CFB1EC010E9467B28DB79EB71FBF8C1B73
:100740009D0BDF91CF911F910895E0918107F0916A
:100750008207199480E480937C0010922C041092FC
:100760002B0410922A04109228041092270487EC7C
:1007700080937A0080917A0086FDFCCF809178008A
:1007800090917900E0912904F0E0ED5BFE4EE49158
:1007900080917B00E3FF02C0886001C0877F809367
:1007A0007B0080917C00E770807EE82BE0937C00EA
:1007B00080917A00806480937A000895DC01CB01F7
:1007C000F894AA23E1F49F3FD1F010927C07109295
:1007D0007D0710927E07A0918400B091850024E6E9
:1007E000A20FB11D8A179B0728F4B0938900A0932C
:1007F000880012C090938900809388000DC09058A3
:10080000A04080937C0790937D07A0937E07B0E87B
:10081000B09389001092880008951F920F920FB62E
:100820000F9211240BB60F922F933F934F935F9328
:100830006F937F938F939F93AF93BF93EF93FF93A8
:1008400080918007811179C080E070917E077723C5
:1008500081F470917D07772319F460917C0791F002
:10086000709389006093880010927C0710927D0736
:1008700008C060917D076058704060937D07709359
:100880007E0781E0811159C081E08093800788E470
:100890009EEE909389008093880080919207882330
:1008A00019F00E9495A00EC080918705882361F001
:1008B0000E94C15660911105709112058091130537
:1008C000909114057BDF37C08091E6189091E7186E
:1008D000892BD1F4209107053091080521153105A8
:1008E00071F08091CA059091CB05821B930B909378
:1008F000CB058093CA0510920805109207058091D8
:10090000CA059091CB0509C08091E6189091E7182F
:1009100001979093E7188093E61810927C07109245
:100920007D0710927E0710927F078CED9FEF9093CA
:1009300089008093880010928007FF91EF91BF910A
:10094000AF919F918F917F916F915F914F913F9167
:100950002F910F900BBE0F900FBE0F901F90189508
:100960001F920F920FB60F9211240BB60F922F9376
:100970003F934F935F938F939F93AF93BF93CF9387
:10098000DF93EF93FF9388B5805C88BD80919F06CD
:10099000811106C08091E81880939B068111759A99
:1009A00080919A06811116C08091EA1880939D0665
:1009B000882329F080910201886080930201809150
:1009C000EB1880939E06882329F0809102018062B3
:1009D0008093020180919B0690919F06891303C02A
:1009E0008F3F09F0759880919D0690919A06891322
:1009F00007C08F3F29F080910201877F8093020119
:100A000080919E0690919A06891307C08F3F29F026
:100A1000809102018F7D80930201789480912E0451
:100A200090912F040196863821E0920728F4909344
:100A30002F0480932E0407C010922F0410922E04CE
:100A400081E080932D0480917A0086FD43C08091DF
:100A5000780090917900E0912904F0E09F01220F45
:100A6000331FD901A65DBB4F4D915C911197840F47
:100A7000951F11969C938E93E45DFB4F40814F5FD1
:100A80004083403210F143E0969587954A95E1F70F
:100A9000E901C95DDB4F998388831D921C92108206
:100AA00010922904E3E4F1E1E49180917B00E3FFFB
:100AB00002C0886001C0877F80937B0080917C00AA
:100AC000E770807EE82BE0937C0080917A00806460
:100AD00080937A0080919A068F5F80939A06809126
:100AE0009F068F5F80939F06FF91EF91DF91CF91DB
:100AF000BF91AF919F918F915F914F913F912F91B6
:100B00000F900BBE0F900FBE0F901F901895109274
:100B10007B0708951F920F920FB60F9211242F9307
:100B20003F938F939F9327B58091400581FF41C0EC
:100B30008091CA059091CB05181619065CF4809136
:100B40007B07813039F080910B018F7B80930B0103
:100B500081E010C08091CA059091CB0597FF12C02B
:100B600080917B078F3F71F080910B0180648093AF
:100B70000B018FEF80937B07285D8091CC05820F5E
:100B800087BD17C08091CA059091CB05892BA9F329
:100B9000439A8091CA059091CB0530917B07831BC6
:100BA000910937FD93959093CB058093CA0543989F
:100BB000E4CF9F918F913F912F910F900FBE0F9097
:100BC0001F9018951F920F920FB60F9211240BB61B
:100BD0000F922F938F939F93EF93FF939091C60063
:100BE000809179078F5F8F7720917A07821741F084
:100BF000E0917907F0E0E750F94F9083809379070F
:100C0000FF91EF919F918F912F910F900BBE0F90BD
:100C10000FBE0F901F9018951F920F920FB60F9254
:100C200011240BB60F928F939F93EF93FF939091A4
:100C3000F7068091F806981306C08091C1008F7D59
:100C40008093C1000EC0E091F806F0E0E954F94F3E
:100C500090818091F8068F5F8F738093F806909350
:100C6000C600FF91EF919F918F910F900BBE0F9057
:100C70000FBE0F901F901895CF92DF92EF92FF92C8
:100C8000CF93DF93EC016A017B01411581EE580798
:100C900061057105F9F0EC85FD8581E090E00E8835
:100CA00002C0880F991F0A94E2F7808360E079E020
:100CB0008DE390E0A70196010E945CB121503109BB
:100CC000410951095695479537952795211580E19A
:100CD000380798F0EC85FD85108260E874E88EE1B5
:100CE00090E0A70196010E945CB1215031094109B1
:100CF00051095695479537952795E885F9853083AD
:100D0000EA85FB852083EE85FF85408181E090E0C8
:100D10009C010A8802C0220F331F0A94E2F7422B7B
:100D20004083EE85FF8540819C010B8802C0220F25
:100D3000331F0A94E2F7422B4083EE85FF85408102
:100D40009C010C8802C0220F331F0A94E2F7422B49
:100D50004083EE85FF8520810D8802C0880F991F92
:100D60000A94E2F7809582238083DF91CF91FF90F0
:100D7000EF90DF90CF9008951092A3061092A206F4
:100D800080E093E09093A1068093A00689EF96E01F
:100D90009093A5068093A40687EB96E09093A70610
:100DA0008093A60685EC90E09093A9068093A80610
:100DB00084EC90E09093AB068093AA0680EC90E0E0
:100DC0009093AD068093AC0681EC90E09093AF06D3
:100DD0008093AE0686EC90E09093B1068093B006C7
:100DE00084E08093B20683E08093B30687E080932B
:100DF000B40685E08093B50681E08093B606089539
:100E00009C01229FB001339FC001239F2227700DB8
:100E1000811D921F700D811D921F11240895CF9284
:100E2000DF92EF92FF920F931F936B017C01890178
:100E30009A01D09E812DD29E902DC12CD19E800DE5
:100E4000911DC31EE09E800D911DC31EE19E900D5D
:100E5000C11CF09E900DC11CE29EC00CF19EC00C06
:100E6000C69497958795C6949795879511241F9159
:100E70000F91FF90EF90DF90CF9008958091400503
:100E800086FB882780F908954098419842980895F4
:100E9000813E2EE2920790F0813C2DE5920740F0D2
:100EA00024E020939A0296958795969587950895C4
:100EB00022E020939A0296958795089521E0209349
:100EC0009A0208952091400521FF55C0FC01E15F81
:100ED000FE4F408151812227579FC001649F312DD1
:100EE000659F300D811D921F749F300D811D921FD3
:100EF0001124F8944091CA055091CB052091070523
:100F000030910805FC01E21BF30B4E0F5F1F50935D
:100F1000CB054093CA051816190694F41216130649
:100F20002CF12091CA053091CB05E0911C03F09182
:100F30001D0341A552A5440F551F240F351F12C094
:100F40000097A1F037FD12C02091CA053091CB0562
:100F5000E0911C03F0911D0341A552A5440F551FBC
:100F6000241B350B3093CB052093CA0590930805BD
:100F70008093070578940895809191078F5F803161
:100F800018F48093910702C0109291071092950770
:100F900010929407F8948091920781508093920761
:100FA00080919207811105C080913D058F7E8093CD
:100FB0003D050895809193078F5F803118F48093E9
:100FC000930702C01092930780913D058061809342
:100FD0003D059FB7F894809192078F5F80939207A9
:100FE0009FBF0895FC0120812F3011F02F5F01C0B9
:100FF00020E0FC01208308954F925F926F927F92D0
:101000008F929F92AF92BF92CF92DF92EF92FF9218
:101010000F931F93CF93DF93EC01888180FDCDC0A8
:10102000898180FDCAC0FE01FD9680809180A280EA
:10103000B38070962081318142815381C501B40112
:101040000E945FB02B013C01FE01E75FFE4F008173
:101050001181B80180E090E00E9488AE6B017C01B4
:10106000FE01E75BFF4F2081318142815381C50141
:10107000B4010E945FB09B01AC01C701B6010E94A0
:101080005FB00E945CAE5E01F5EFAF1AFEEFBF0AE3
:10109000D5016D937C93A3019201C701B6010E9413
:1010A0005FB00E945CAE6E01B3EFCB1ABEEFDB0AFD
:1010B000F60171836083C801A3DE2B013C01D501D9
:1010C0008D919C919DDE8E0103501F4FA3019201D3
:1010D000261B370B480B590BCA01B9017E0131E0C1
:1010E000E30EF31ED7012D913D914D915C91220F9E
:1010F000331F441F551F0E945CB12F5F3F4FF80103
:1011000031832083D6018D919C917ADEA3019201D7
:10111000261B370B480B590BCA01B901D7012D917A
:101120003D914D915C91220F331F441F551F0E942A
:101130005CB1B9016F5F7F4F7E01BFEFEB0EF11C19
:10114000F70171836083D801ED91FC911197AB0198
:101150004E0F5F1F54968D919D910D90BC91A02DC7
:101160004A01A12CB12C88169906AA06BB0614F1D7
:101170009A012E5F3F4F4901A12CB12C881A990A80
:10118000AA0ABB0AB594A79497948794C401E8155A
:10119000F90508F4CF01E81BF90BD801ED93FC9396
:1011A00094016815790508F49B01621B730BF70124
:1011B00071836083888181608883DF91CF911F91E3
:1011C0000F91FF90EF90DF90CF90BF90AF909F90E6
:1011D0008F907F906F905F904F9008952F923F92E5
:1011E0004F925F926F927F928F929F92AF92BF9237
:1011F000CF92DF92EF92FF920F931F93CF93DF93E3
:1012000000D01F92CDB7DEB7582E6A8385E191E0FA
:10121000589E9001599E300D11242A56384F3C8318
:101220002B83F901E35BFF4F9080818072806380A4
:10123000FA815F1609F452C1552011F05A9402C088
:10124000BFE05B2E85E191E0589E8001599E100D14
:1012500011240A56184FF801E65AFF4F9081EB818E
:10126000FC81E65AFF4F8081D801AB5BBF4F6D0117
:10127000F801E35BFF4F7F012B813C81275B3F4FF0
:101280005901981340C02D913D914D915C91692D6C
:10129000782D872D962D0E94B7AD811134C0892DF0
:1012A000982DA72DB62DF70180839183A283B38358
:1012B000EB81FC81EF5AFF4F4080318022802381F7
:1012C0002983292D382D472D562D642D732D822DE0
:1012D00099810E94B7AD87FF04C0492C382C272C78
:1012E0006982842D932DA22DB981F501808391838C
:1012F000A283B383D8018C918E7F8C93EB81FC8188
:1013000080818E7F8083AB81BC8111968C911197F7
:1013100081FF0CC0D9969C90D997DA968C90DA9779
:10132000DB967C90DB97DC966C901AC0292D382DCB
:10133000472D562D692D782D872D962D0E945FB053
:10134000EB81FC81EF5BFF4F208131814281538132
:101350000E9453AD0E94CCB0962E872E782E692E17
:10136000F601208031804280D3809101442D5D2D93
:10137000692D782D872D962D0E94EBAF87FD65C0D6
:101380009101442D5D2DD7016D917D918D919C91A1
:101390000E94B7AD882311F1F80180818E7F808390
:1013A000EF5AFF4F708081809280C3809101442D5D
:1013B0005D2D672D782D892D9C2D0E94B7AD87FF5F
:1013C00004C0722C832C942CCD2C872D982DA92D04
:1013D000BC2DF70180839183A283B3839101442DB7
:1013E0005D2DD5016D917D918D919C910E94B7AD40
:1013F000882329F1EB81FC81EF5AFF4F70808180B7
:101400009280C3809101442D5D2D672D782D892D0B
:101410009C2D0E94B7AD87FF04C0722C832C942CA6
:10142000CD2C872D982DA92DBC2DF501808391837E
:10143000A283B383AB81BC818C918E7F8C93F701A7
:10144000908081807280638046C0EB81FC81EF5A7E
:10145000FF4F30804180C280D380292D382D472D09
:10146000562D632D742DC6010E94B7AD87FF04C0B1
:10147000392C482CC72CD62C832D942DD601F50160
:1014800080839183A283B383F801EF5AFF4FC0801A
:10149000D180B280A38096014B2D5A2D692D782DD5
:1014A000872D962D0E94B7AD87FF03C09C2C8D2CF5
:1014B0003501892D982DA72DB62DF70180839183B5
:1014C000A283B383D8018C918E7F8C93EB81FC81B6
:1014D00080818E7F80831C830B83AACE0F900F9018
:1014E0000F900F90DF91CF911F910F91FF90EF9090
:1014F000DF90CF90BF90AF909F908F907F906F9034
:101500005F904F903F902F9008952F923F924F926F
:101510005F926F927F928F929F92AF92BF92CF9283
:10152000DF92EF92FF920F931F93CF93DF93CDB78C
:10153000DEB72A970FB6F894DEBF0FBECDBF898302
:1015400025E131E0829F1001839F300C112491012D
:101550002A56384F1901F901E75BFF4FA080B1808F
:10156000C280D3809981809193079101275B3F4F7F
:101570003F832E83981709F474C1CE01019632DDA2
:101580008981A5E1B1E08A9F20018B9F500C112435
:10159000F201EA56F84F2F01E65AFF4FD101A65A41
:1015A000BF4F9C9180819101235B3F4F3B832A83F6
:1015B0005597BD83AC83F1019080981323C0D90166
:1015C000EC901196FC90119712960C91129713962D
:1015D0001C91EC81FD812081318142815381B701D1
:1015E000C8010E94B7AD81110DC0C501D601EE81C1
:1015F000FF8180839183A283B383892D8260D1018F
:101600008C9327C1D10111968C91119781FF0CC049
:10161000D996EC90D997DA96FC90DA97DB960C91F4
:10162000DB97DC961C9113C09501A601B501C6019C
:101630000E945FB0F101EF5BFF4F20813181428159
:1016400053810E9453AD0E94CCB07B018C01EA8192
:10165000FB812081318142815381B701C8010E9401
:10166000EBAFF101EF5AFF4F18160CF083C0E0808A
:10167000F180028113819701A801B501C6010E9482
:10168000B7AD87FF1AC09701A801B701C8010E9432
:101690005FB0F101EF5BFF4F2081318142815381C7
:1016A0000E9453AD0E94CCB0AA81BB816D937D9303
:1016B0008D939C93139757016801C501D601EE8164
:1016C000FF8180839183A283B383F201EF5AFF4F9E
:1016D00020812E83318138878281898793819A87FF
:1016E000AC81BD816C9011967C90119712968C9074
:1016F000129713969C90EA81FB81A080B180C280F2
:10170000D3809301A401B501C6010E94B7AD87FF44
:1017100003C07501860102C0730184012E813885E2
:1017200049855A85B701C8010E94B7AD87FF04C03B
:10173000EE80F88409851A85C701D801F201E75BBC
:10174000FF4F80839183A283B3839301A401B501EA
:10175000C6010E94B7AD811108C0D1018C91826091
:101760008C93F201808184608083D1018C918E7F83
:101770008C9373C0892D8E7F8660D1018C9360809D
:101780007180828093809501A601B301C4010E94FB
:10179000EBAF1816ACF49301A401B301C4010E948D
:1017A0005FB0F101EF5BFF4F2081318142815381B6
:1017B0000E9453AD0E94CCB07B018C0153016401A7
:1017C000C501D601EE81FF8180839183A283B3831B
:1017D0009701A801B301C4010E94B7AD87FF02C001
:1017E00037014801C301D401EA81FB8180839183E1
:1017F000A283B383F201EF5AFF4FA080B180C28071
:10180000D380AC81BD81EC901196FC90119712961B
:101810000C91129713961C919701A801B301C40172
:101820000E94B7AD87FF02C0730184019501A60134
:10183000B701C8010E94B7AD87FF02C075018601DC
:10184000C701D801F201E75BFF4F80839183A28338
:10185000B383F201808184608083570168011201A3
:1018600081CEF101EF5AFF4FE080F18002811381B8
:101870009501A601B701C8010E94B7AD87FF02C05C
:1018800075018601C701D801EE81FF8180839183B4
:10189000A283B3832A960FB6F894DEBF0FBECDBFE6
:1018A000DF91CF911F910F91FF90EF90DF90CF903C
:1018B000BF90AF909F908F907F906F905F904F9070
:1018C0003F902F9008952F923F924F925F926F9288
:1018D0007F928F929F92AF92BF92CF92DF92EF92C0
:1018E000FF920F931F93CF93DF93CDB7DEB72D9762
:1018F0000FB6F894DEBF0FBECDBF209193072A83A9
:1019000085E191E0289F8001299F100D11240A563E
:10191000184F2FB72E83F894809191078983909167
:101920009307891719F0CE0101965CDBC12CD12CED
:10193000760135E1A32EBB24B3948981909193075E
:101940008917C9F08A9DF0018B9DF00D1124EA568C
:10195000F84F83819481A581B681C80ED91EEA1EF5
:10196000FB1ECE0101963EDB38ECC3163FEAD306E0
:10197000E104F10410F339812A8185E191E0231714
:1019800081F0289FF001299FF00D1124EA56F84FAD
:10199000408141FD06C0222311F02150F0CF2FE0FD
:1019A000EECF2A8380919307281761F085E191E0BB
:1019B000289FF001299FF00D1124EA56F84F8081ED
:1019C00081FDA5C12A818091930728130EC0F801DB
:1019D000818180688183FE81FFBFF80180818460FE
:1019E0008083C80109DBF8014FC185E191E0289FA0
:1019F000A001299F500D11244A56584F5D834C83F6
:101A0000FA01818180688183FE81FFBF2091930765
:101A1000222311F0215001C02FE085E191E0289FA1
:101A20001001299F300C112491012A56384F1901B9
:101A300080914005F901F085FA87F801F085FB8770
:101A40002B5B3F4F3987288781FF10C08F2F881F5E
:101A50008827881F9A85991F9927991F981731F011
:101A60008F2F3A85832B807309F055C1F101E65A17
:101A7000FF4F9081F801E65AFF4F8081F801F1ADE8
:101A8000FB83F801F2ADFF83F801F3ADFC87F801A9
:101A9000F4ADFD87F10198131AC0C1ACD2ACE3AC30
:101AA000F4AC2B813F814C855D85C701B6010E9456
:101AB000EBAF18162CF48B819F81AC85BD85C4C01B
:101AC000E885F985C082D182E282F382C3C021A574
:101AD00032A543A554A5F80161A572A583A594A5D7
:101AE0000E9452AD2B013C01F10125A536A547A569
:101AF00050A9F80165A576A587A590A90E9452ADC9
:101B00004B015C01F10121A932A943A954A9F801B3
:101B100061A972A983A994A90E9452AD6B017C01AD
:101B2000A3019201C301B2010E945FB02B013C01ED
:101B3000A5019401C501B4010E945FB09B01AC01F5
:101B4000C301B2010E9453AD4B015C01A701960194
:101B5000C701B6010E945FB09B01AC01C501B40191
:101B60000E9453AD0E94CCB04B015C01C090730445
:101B7000D0907404E0907504F0907604A70196016B
:101B80000E94EBAF18164CF4A5019401C701B601F1
:101B90000E94BEAD2B013C0106C0412C512C90E8A7
:101BA000692E2FE3722EF10125A936A947A950AD60
:101BB000F80165A976A987A990AD0E9452AD4B01A5
:101BC0005C01E894B7F8E0911C03F0911D03C7880D
:101BD000D08CE18CF28CA7019601C501B4010E9462
:101BE000EBAF181694F4A5019401C701B6010E9449
:101BF000BEAD6B017C019B01AC01B201C3010E942F
:101C0000B7AD87FD02C026013701EB80DF80CC84B1
